:100000000C94083B0C94B23B0C94B23B0C94B23B66
:100010000C94B23B0C94B23B0C94B23B0C94B23BAC
:100020000C94B23B0C94B23B0C94B23B0C94B23B9C
:100030000C94B23B0C949D520C94B23B0C94B23B8A
:100040000C94B23B0C94B23B0C94B23B0C94B23B7C
:100050000C94B23B0C94B23B0C94B23B0C94B23B6C
:100060000C94B23B0C94B23B0C94B23B0C94B23B5C
:100070000000000000000000000000000000000080
:100080000000000000000000000000000000000070
:100090000000000000000000000000000000000060
:1000A0000000000000000000000000000000000050
:1000B0000000000000000000000000000000000040
:1000C00000000049000000495252000052525C2DCD
:1000D0000000000000000000000000000000000020
:1000E0000040000000494A52004952525B1C5253E2
:1000F0001C25241B2425251B0A0A2D1C12120A0A62
:100100000000000000000000404949494949525B95
:100110005B5B525B1C1C1312241C12090909120997
:100120000909090A0A0A0A0A0A13120A0A12130A10
:100130000000000000009252525252521312130952
:10014000001C0A1212401B65090A0009241B120038
:1001500000251C1C010025241C1C0024252424240B
:100160000000000000005249494000001B135249A2
:100170004900641C1C5B4A481C651C2552491C1C18
:10018000652464491C1C652564491C1C6D2E5C4952
:100190000000000000000000000000490000000016
:1001A000535200000053522500004A5225250000FA
:1001B0005B251300005B53000A1C095B1C657F373D
:1001C0004052522E2E1C525C2E251B1324251C1C23
:1001D00012002525120000121B0000132E37001BF1
:1001E00037372E2E37372E2E2E2E2E2E6E6E6E1C5D
:1001F0001313120009131200001213130012251C0E
:1002000013132E371C131313361C131B1B1B251320
:100210001C1C1B1B1B1C1C1C1C1C1C1C1C1C1C132A
:100220001312121313001313131C000913131C01D0
:100230000037131C13002E2E1C1C001C772E2500CB
:10024000137F251C010A37241C1C0A2E25250900B2
:10025000132E242525252E252525252525252D2E3E
:10026000251B2E2E251C1325251C1C1C1C011C1CAB
:100270001300011C0A000165775C016E7F6E521B42
:1002800025256D1C524925251C1353001C1C1C528E
:100290004A001B135B5B000009525C0000005B5CC2
:1002A000000000001B000000000000000000000033
:1002B000135B7F776E6E136577766E6E1B65777650
:1002C00076761B5BBF76B67609136DBFB7B6001B9B
:1002D000125C76BF0000121B125B00000000090ACE
:1002E0006E6E6E77241C6E6E77251C1C6E776E1CEE
:1002F0001C1C76761C1C2425B765646D6D1B766D01
:100300006D5B09125B5C5B125B641213131B1212B0
:100310001C1C1C1C1C241C1C242525242425251BDA
:1003200000002513000064BF00096EBFBF6D6EBFE3
:100330006D5B12135B12131209000901000000002B
:100340002E1C0900096E010009767F7F12777F7FDE
:100350006412BF775B121B095B121B0900001B09AB
:10036000000000000000000000000000000000008D
:100370007F7F5313130064121B0100001B12000047
:10038000000000000000000000000000000000006D
:10039000000000000000000000000000000000005D
:1003A0000000000000002600000026002F000000D2
:1003B0002F00370000003700FF000000FF00BF00E3
:1003C0000000BF00370000370000002626000000B4
:1003D000000000000000262626262600000000005F
:1003E0002F000000003700000000FF00000000BFE9
:1003F0000000000037000000000026262626260008
:100400000000000000002626262626002F000000FF
:100410000000370000000000FFFFFFFF0000BF00EA
:1004200000000000370000000000262626262600D7
:100430000000000000002626262600002F000000F5
:100440002F00370000003700FFFFFFFF0000BF0054
:100450000000BF00370000003700262626260000D7
:10046000000000000000000026262600002F0000EB
:100470002F00370000003700FF000000FF00BF0022
:100480000000BF00370000370000262626000000CD
:100490000000000000002600000026002F000000E1
:1004A0002F000037003700000000FF00000000BFF1
:1004B00000BF0000370000003700260000002600C3
:1004C000000000000000000000000000000000002C
:1004D000000000000000000000000000000000001C
:1004E0000000009B000000529BA400005B9B6D7706
:1004F00000000000000000000000000000000000FC
:10050000005B000000E4F6FF099BEDF6FFBFA4AD21
:10051000BFBFBFBF767F7FB7B7BF7F766EB7B7BFAE
:1005200000000000000000005BB6F6F6F6FFFFFFDB
:10053000FFBFFFFFFFBFBFAEFFFFFFB7AD65FFFF10
:10054000B7B6AD65FFFFBFB7AE6EFFFFBFB7B7650C
:10055000000000000000F6F6EDEDADA4B66D6D5C98
:10056000526E6565655265765C5C52536E246552C9
:10057000526E25255B52772D2525526E6E2D252531
:10058000000000000000A49B9B4900006564A49B40
:1005900092006D2525649349656E652E9B52242536
:1005A0006D25655225246D2D655225256E2E6452CC
:1005B00000000000000000000000004A00000000F1
:1005C0005B9B0000005B5B2D0000525B2E2E000148
:1005D0005B2D1C01005C5B014A654A5B1C6E7F77EA
:1005E000495B9B77776D5B65776E65656D2D25251E
:1005F0005C522E25130949641C09095C7F7F091C84
:100600007F7F777F777F77777F7F7776777F7F6E44
:10061000656E6EA4B6FF655BA4B7BFFF526DBFBF2A
:10062000BFFF7FBFBFBFBFFFBFBFB7BFFFFF7FB76A
:10063000BFBFFFFF6EB7BFBFFFFF77BFBFBFFFFFEB
:10064000FFFFBFBFB75BFFFFBFBFA464FFFFBFAD2E
:10065000A47FFFFFBFA4BF7FFFBFADBFBFBFFFB67B
:10066000BFBFBF77F7BFBFBF7777FFBFBFBF6452C2
:100670006D7F6E2E2D2D7F766E6E6E2E7777777650
:100680002E1C7F776E251C25776525251C096E6E2F
:100690001C0949255B494A6E7F645377BF775B5CD1
:1006A000256E6E255B4A25651C1B5B002524245B9B
:1006B00053001C1B5B5C00000A5B64000000646468
:1006C000000000005C0000000000000000000000CE
:1006D0005B5C7FBF77765C6D7FB777775C6D7FBF44
:1006E00077775C64BFBFBFBF0A5C6EBFBFBF0065EA
:1006F000646DBFBF00005B6D646D00000000125BA5
:100700007777777F6E6E77777F766D7677BF776D49
:100710006E76BF7F6D6E767FBF7676BFBF76BFBFCA
:10072000BFB664ADADB6B6ADBFFF646DADB6AD647A
:1007300077BFBFBFFFFF77BFBFBFFFFF7FBFBFBF99
:10074000FFF6BFB7ADF6FFFFA4ADFFFFFFFFFFFF52
:10075000FFFFFFFFFFFFFFF6A4005B520000000059
:10076000BFBFAD5B64BFB6ADADBFFFBFFFFFFFFF57
:10077000BF64FFFFBFB6765BFFBFBF5B0000FF5CDF
:100780000000000000000000000000000000000069
:10079000BFBF645C5C006E5C654900006D5B00007F
:1007A0000000000000000000000000000000000049
:1007B0000000000000000000000000000000000039
:1007C0000600040000000100020003000400050010
:1007D00006000700080009000A000B000C000D00CD
:1007E0000E000F0010000000110012001300140092
:1007F000150016000600030000001700180019007D
:100800001A001B001C001D001E001F0020002100FC
:10081000220023002400250026000000000208001A
:10082000085504085A0000F8000990000A1E320515
:100830000000FF0000001C08000000007E548C54E3
:100840006A55375923598F549E54AD540B59BB5494
:10085000C95400000001000200030004000501006B
:10086000010101020103010401050200020102026B
:10087000020302040205030003010302030303044D
:100880000305040004010402040304040405050034
:10089000050105020503050405050600060106021B
:1008A00006030604060507000701070207030704FD
:1008B00007050800080108020803080408050900E4
:1008C000090109020903090409050A000A010A02CB
:1008D0000A030A040A050B000B010B020B030B04AD
:1008E0000B050C000C010C020C030C040C050D0094
:1008F0000D010D020D030D040D050E000E010E027B
:100900000E030E040E050F000F010F020F030F045C
:100910000F05100010011002100310041005110043
:10092000110111021103110411051200120112022A
:10093000120312041205130013011302130313040C
:1009400013051400140114021403140414051500F3
:1009500015011502150315041505160016011602DA
:1009600016031604160517001701170217031704BC
:1009700017051800180118021803180418051900A3
:10098000190119021903190419051A001A011A028A
:100990001A031A041A051B001B011B021B031B046C
:1009A0001B051C001C011C021C031C041C051D0053
:1009B0001D011D021D031D041D051E001E011E023A
:1009C0001E031E041E051F001F011F021F031F041C
:1009D0001F05FFFFFFFFFFFFFFFFFFFFFFFFFFFF01
:1009E000FFFFFFFFFFFFFFFFFFFFFFFFFFFFFFFF17
:1009F000FFFFFFFFFFFFFFFFFFFFFFFFFFFFFFFF07
:100A0000FFFFFFFFFFFFFFFFFFFFFFFFFFFFFFFFF6
:100A1000FFFFFFFFFFFFFFFFFFFFFFFFFFFFFFFFE6
:100A2000FFFFFFFFFFFFFFFFFFFFFFFFFFFFFFFFD6
:100A3000FFFFFFFFFFFFFFF7FFFFFFA70F0FFFFF06
:100A4000670F0F0FFFF70F0F0F0FFFAF0F0F0F0FF6
:100A5000FFA70F0F0F0FFFF70F0F0F0FFFFF570F1E
:100A60000F0FF7FFFFFFFFFF0F17F7FFFFFF0F5FEE
:100A7000AFFFFFFFA7FFFFFFFFFFF7FFFFFFFFFF36
:100A8000AFFFFFFFF7FF17F7FFF70FF70F0FAF5F8E
:100A90000F5FFFFFFFFFFFFFFFFFFFFFFFFFFFFFF6
:100AA000FFFFFFFFFFFFFFFFFFFFFFFFFFFFFFFF56
:100AB000FFFFFFFFFFFFFFFFFFFFFFFFFFFFFFFF46
:100AC000FFFFFFFFFFFFFFFFFFFFFFFFFFFFFFFF36
:100AD000FFFFFFA7FFFFFFFF570FFFFFFF670F0F8E
:100AE000FFFFFF570F0FFFFFF70F0F0FFFFFF70F6E
:100AF0000F0FFFFFAF0F0F0FFFFFFF5F0F0F5FAF76
:100B0000FFFF570F57FFFFFFA70FA7FFFFFFAF0F15
:100B10005FFFFFFF5F0F0F5FA7570F0F0F0F0F0F45
:100B20000F0F0F0F0F0F0F0F0F0F0F0F0F0F0F0FD5
:100B30000F0F0F0F0F0F0F0F0F0F0F0F0F0F0F0FC5
:100B40000F0F0F0F0F0F0F0F0F0F0F0F0F0F0F0FB5
:100B50000F0FFFFFFFFFFFFFAFFFFFFFFFFF5FFF75
:100B6000FFFFFFFF5FFFFFFFFFFF5FFFFFFFFFFFD5
:100B70005FFFFFFFFFFF5FFFFFFFFFFF67FFFFFF5D
:100B8000FFFFFFFFF70F0F0FFFFFF70F0F0FFFFF25
:100B9000F70F0F0FFFFFF70F0F0FFFFFF70F0F0FED
:100BA000FFFFF70F0F0FFFFFF70F0F0FFFFFF70FFD
:100BB0000F0F0F0F0F0F0F0F0F0F0F0F0F0F0F0F45
:100BC0000F0F0F0F0F0F0F0F0F0F0F0F0F0F0F0F35
:100BD0000F0F0F0F0F0F0F0F0F0F0F0F0F0F0F5FD5
:100BE0005F5F0F0F0F0F0F0F0F0F0F0F0F0F0F0F75
:100BF0000F0F0F5F0F0F0F0F0FF70F0F0F0FA7FF45
:100C00000F0F0F5FFFFF0F0FA7FFFFFFA7FFFFFFF4
:100C1000FFFFAFFFFFFFFFFFFFFFFFFFFFFFFFFF34
:100C2000FFFFFFFFFFFFFFFFFFFFFFFFFFFFFFFFD4
:100C3000FFFFFFFFFFFFFFFFFFFFFFFFFFFFFFFFC4
:100C4000FFFFFFFFFFFFFFFFFFFFFFFFFFFFFFFFB4
:100C5000FFFFFFFFFFFFFFFFF6F6FFFFFF5B09ADA2
:100C6000FFF6520009ADFF5B000909ADFF5B00090B
:100C700009ADFFFFF70F0F0FFFFFF70F0F0FFFFF7C
:100C8000F70F0F0FFFFFF70F0F57FFFFF70F0FF7CC
:100C9000FFFFF70FA7FFFFFFF75FFFFFFFFFFFF764
:100CA000FFFF0F17F7FFFFFF0FB7FFFFFFFFA7FFC4
:100CB000FFFFFFFFFFFFFFFFFFFFFFFFFFFFFFF64D
:100CC000FFFFFFFFFF52FFFFFFFFF609FFFFFFFFE0
:100CD000AD09FFFFFFFFFFFFFFFFFFFFFFFFFFFF6C
:100CE000FFFFFFFFFFAD5B52A4FF5200090009F6B2
:100CF0000009090009F60009090009F6090052FF78
:100D0000FFFFFFFFFFFFFFFFFFFFFFFFFFFFFFFFF3
:100D1000FFFFFF52FFFFFFFF5200FFFFFFAD000983
:100D2000FFFFFF5B0009FFFFFF520009FFFFFF52BB
:100D30000009FFFFFFFFFFFFADA45B52A4AD000958
:100D4000090909000909090909090909525209098A
:100D500009ADFFFFF60909F6FFFFFF5B0052F6FF42
:100D6000FFFFFFFFFFFFFFFFFFFFFFFFFFFF09F692
:100D7000FFFFF65B0909FFFFAD090900A4FFAD09FC
:100D8000000052FFAD09000009FFAD09FFFFFFFFA2
:100D9000AD09FFFFFFFFFFFFFFFFFFFFAD5B52004D
:100DA000AD5B00090900520009090909090909098F
:100DB00009090009ADF6090909F6FFFF090052FF0C
:100DC000FFFFFFFFFFFFFFFF5BA4F6FFFFFF090927
:100DD00009A4FFFF09090909ADFF0909090009F67E
:100DE000A400090900ADFFA40009005BFFFF090092
:100DF0000009FFFFFFFFFFFFFFFFFFFFFFADFFFF4A
:100E0000FFAD0909FFFFAD000909FFFF520009000E
:100E1000FFF600090052FFAD000900A4FFFFF6F63F
:100E2000F6FFFFFFFFFFFFFFA4525BA4ADFF090920
:100E300009090009090909090900095252000909AB
:100E4000FFFFFFA40009FFFFFFF60900FFFFFFAD52
:100E50000900FFFFFFFFFFFFFFFFFFFFFFFFF6FFA0
:100E6000FFF65B0909F6FFA4000000ADFFA400092E
:100E7000005BFFA40009005BFFA40009005BFFA466
:100E80000009FFFFFFFFFFFFFFFFFFF65B5B09F6B7
:100E9000AD090900095B09000900090909090900F0
:100EA000090909090900090052F6FFFF0009F6FFC8
:100EB000FFFFFF5B000909ADFF5B000909ADF65BB1
:100EC000000909ADF65B000909ADF65B000909AD43
:100ED000F65B000909F6FF5B000909ADFF5B00093D
:100EE0000909FFFFFFFFFFFFFFFFFFFFF6F6FFFF10
:100EF000FF520009FFFFA4000900FFAD000900092F
:100F0000F609090900AD52000900A4FF0009005BC1
:100F1000FFFFFFFFFFFFAD09F6F6FFFFA409005B2F
:100F2000FF09000952FF52000909FFA4000909093D
:100F3000FFF6F6F6A409FFFFFFFFAD09FFFFFFFF75
:100F4000AD090900A4FFFFFF09005BF6F6FF0909E0
:100F5000090052AD0909090052AD0909090052AD55
:100F600009005BF6F6AD0900A4FFFFF60900A4FF37
:100F7000FFF6FFFFFFFFFFFFF6F6F6F6FFFF0900A3
:100F8000005BFFFF0900005BFFFF0900005BFFFF44
:100F90000900005BFFFF0900005BFFFF0900005B29
:100FA000FFFFFFFFFFFFFFFFFFFFFFF6F6F6FFFF6C
:100FB000A4000900FFFFA4000900FFFFA40009002E
:100FC000FFFFA4000900FFFFA4000900FFFFA40029
:100FD0000900FFFFFFFFFFFFFFFFF6F6F6F6ADFF8C
:100FE00009090052ADFF09090052ADFF09090909BD
:100FF000ADFF09090909ADFF09090900ADFF09099C
:101000000909FFFFFFFFFFFFFFFFAD5B5BA4F609D0
:101010000009090952000909090909090909090909
:10102000095BF6A409095BFFFFFFA400F6FFFFFFC1
:10103000F600FFFFFFFFFFFFFFFFFFFFFFFF09F6C7
:10104000FFFFFFFF0052FFFFFFFF0009ADFFFFFFA3
:101050000900A4FFFFFF09005BFFFFFF00005BFF2B
:10106000FFFFFFFFFFA40009FFFFFFFF0900FFFFD5
:10107000FFFFF652FFFFFFFFFFFFFFFFFFFFFFFF36
:10108000FFFFFF525252FFFFFF090900FFFFFF520F
:101090000009090900095BAD0909090909000009EE
:1010A00009090909F65B09000909FFFFFFF65B0062
:1010B000ADFFFFFFFF5B52FFFFFFFFA409A4FFFF8F
:1010C000F609FFFFFFFFAD0909ADFFFFAD090900FC
:1010D000A4FFAD09090009F6AD09090009ADAD0984
:1010E000000009ADAD09000009ADAD09000009F629
:1010F000AD090900A4FFFFFF0900ADFFFFFF0900D4
:10110000ADFFFFFF0900ADFFFFFF0900A4FFFFFFD8
:10111000090052FFFFFF090909F6FFFF090900094D
:10112000A4F6FFFF52000900FFFF5B000900FFFF6C
:101130005B000900FFFF5B000900FFFF5200090090
:10114000FFFF09000009FFA40009005B5B09090912
:1011500000ADFFFFFFFFFFFFF6FFFFAD5209FFFFEE
:101160005B000909FFAD00090900F65B000900A456
:10117000FF52000009FFFF52000009FFFF52000963
:1011800009ADF6F6A40900090909090909090909BF
:1011900009090909095BA4AD0900FFFFFFF6090071
:1011A000FFFFFFAD0900FFFFFFA40009FFFFF609E5
:1011B0000009005BFFA40009005BFFA40009005BBD
:1011C000FFA40009005BFFA40009005BFFA4000965
:1011D000005BFFA40009005BFFA40009005BFFA403
:1011E0000009005BFFFFFFFF00A4FFFFFFFF09AD49
:1011F000FFFFFFFF09ADFFFFFFFF09ADFFFFFFFF8F
:1012000009ADFFFFFFFF09ADFFFFFFFF09ADFFFFC6
:10121000FFFFFF5B00090909FF5B00090909FF5B8C
:1012200000090909FF5B00090909FF5B0009005279
:10123000FF5B000909ADFF5B000909ADFF5B000919
:1012400009AD090900ADFFFF09090052FFFF0909B7
:101250000900ADFF0909090009FFF609000900A40A
:10126000FF5B00090009FFF609090900FFFF5B00A9
:101270000900FFFFFFFFAD09FFFFFFFFAD09FFFF03
:10128000FFFFAD09FFFFFFFFAD09FFFFFFFFAD0946
:10129000FFFFFFFFAD09ADFFFFFFAD0952FFFFFFED
:1012A000AD090900A4FFFFF60900A4FFFFF609003D
:1012B000A4FFFFF60900A4FFFFF60900A4FFFFF654
:1012C0000900A4FFFFF60900A4FFFFF60900A4FF30
:1012D000FFFF0900005BFFFF0900005BFFFF090043
:1012E000005BFFFF0900005BFFFF0900005BFFFFE1
:1012F00009000052FFFF09000909FFFF0900090961
:1013000009A4FFFFA4000900FFFFA4000900FFFFDC
:10131000A4000900FFFFA4000900FFFFA4000900CA
:10132000FFFF52000900FFF600090900A40909099E
:101330000900ADFF09090909ADFF09090909ADFF58
:1013400009090909ADFF09090909ADFF09090909D9
:10135000ADFF09090909ADFF09090909ADFF09092F
:101360000909FFFFFFFFF609FFFFFFFFF609FFFF77
:10137000FFFFF609FFFFFFFFF609FFFFFFFFF6097A
:10138000FFFFFFFFF609FFFFFFFFF609FFFFFFFF6B
:10139000F60900005BFFFFFF00005BFFFFFF00009E
:1013A0005BFFFFFF00005BFFFFFF00005BFFFFFF35
:1013B00000005BFFFFFF00005BFFFFFF00005BFF23
:1013C000F6F6FFFFFFFFFFFFFFFFFFFFFFFFFFFF3F
:1013D000FFFFFFFFFFFFFFFFFFFFFFFFFFFFFFFF1D
:1013E000FFFFFFFFFFFFFFFFFFFFFFFFFFFFFFFF0D
:1013F000FFFFFFFFFFAD0009FFFFFFFF5B00FFFFE7
:10140000FFFFFFA4FFFFFFFFFFFFFFFFFFFFFFFF47
:10141000FFFFFFFFFFFFFFFFFFFFFFFFFFFFFFFFDC
:10142000FFFF090009520909090909090909090900
:1014300009090900FFADA4A4A4F6FFFFFFFFFFFF09
:10144000FFFFFFFFFFFFFFFFFFFFFFFFFFFFFFFFAC
:10145000FFFF090052FFAD090909F6FFAD0909F6C2
:10146000FFFFAD09FFFFFFFFAD09FFFFFFFFAD0964
:10147000FFFFFFFFAD09FFFFFFFFAD09FFFFFFFF0C
:10148000AD090909090909090900520009090900FA
:10149000A4A409000900A4FFF6A40900A4FFFFFF0B
:1014A0000900A4FFFFFF0900A4FFFFFF0900A4FF3C
:1014B000FFFF0909090052FF09090909ADFF0909E0
:1014C00009ADFFFFA4A4FFFFFFFFFFFFFFFFFFFF2A
:1014D000FFFFFFFFFFFFADA4A4A4A4F6AD09090917
:1014E00000F6FFA400090900FFF609000909FFFF43
:1014F000AD090009FFFFFFFFA4A4FFFFFFFFFFFFEF
:10150000FFFFFFFFFFFFFFFFFFAD5BFFFFFFFF528E
:1015100009FF09090909090909090909090909004E
:1015200052F65200A4F6FFFFFFFFFFFFFFFFFFFF91
:10153000FFFFFFFFFFFFFFFFFFFFFFADFFFFFFFF0D
:10154000FFAD005BFFA400090052FFA400090009E1
:10155000FFA40009FFFFFFFFFFFFFFFFFFFFFFFFEB
:10156000FFFFFFFFFFFFA4A4A4A4F6FF00090900EA
:10157000F6FF09ADFFFFFFFF09ADFFFFFFFF09AD5C
:10158000FFFFFFFFFFFFFFFFFFFFFFFFFFFFFFFF6B
:10159000FFFFFFFFFFFFFFFFFFFF5B52FFFFFF5259
:1015A0000009FF5B000909ADFF5B000909ADFF5BA6
:1015B000000909ADFFFFFFFFFFFFFFFFFFFFFFFF78
:1015C000FFFFFFFFFFFF5BF6FFFFFFAD0009FFFF1F
:1015D000FF5BFFFFF6090009FFFFFF5B0009FFFF4C
:1015E000FFF60900FFFFFFFFFFFFFFFFFFFFFFFF09
:1015F000FFFFFFFFFFFFA4A4A4A4A4FF00090909A3
:1016000000F600ADFFFFAD090009FFFFAD090900BD
:10161000A4FFAD09FFFFFFFFFFFFFFFFFFFFFFFF7D
:10162000FFFFFFFFFFFFFFFFFFA4A4A4FFFFF600E3
:1016300009090900A4FFFFFF0900A4FFFFFF09003B
:10164000A4FFFFFFFFFFFFFFFFFFFFFFFFFFFFFF05
:10165000FFFFFFFFFFFFA4F6FFFFFFFF0009F6FFFC
:10166000FFFF520009090909AD0009090909FFA492
:1016700000090909FFFFFFA4A4A4FFFFFFFFFFFF6C
:10168000FFFFFFFFFFFFFFAD5B52A4FFAD000909A5
:10169000005B09090909090009095B00090009A49F
:1016A000F6000900FFFFFFFFFFFFFFFFFFFFFFFF47
:1016B000FFFFFFFFFFFFFFFFFFFFA45BFFFFFFFF39
:1016C0005200ADFF09090909ADFF09090909ADFF7C
:1016D00009090909FFFFFFFFFFFFFFFFFFFFFFFFF2
:1016E000FFFFFFFFFFFFFFFFAD5BFFFFADFFA400AC
:1016F000F6FFFFFFFFFFF609FFFFFFFFF609FFFF01
:10170000FFFFF609FFFFFFFFFFFFFFFFFFFFFFFFE8
:10171000FFFFFFFFFFFFFFFF5BADFFFFFFF6095B72
:10172000FFFF00005BAD095200005BFF5BAD0000F6
:101730005BFF5BADFFFFFFFFFFFFFFFFFFFFFFFF53
:10174000FFFFFFFFFFFFFFFFFFA4525BFFFF5B00F8
:1017500009005B52ADFFFFFF5209ADFFFFFF525B77
:10176000ADFFFFFFFFFFFFFFFFFFFFFFFFFFFFFFDB
:10177000FFFFFFFFFFFFF6FFFFFFFFF609F6FFFF8A
:10178000FF09FFFFFFFFFFFFFFFFFFFFFFFFFFFF5F
:10179000FFFFFFFFFFFFFFFFFFFFFFFFFFFFFFFF59
:1017A000FFFFFFFFFFFF5B52A4FFFFFF0909005B84
:1017B000FFFFFFFFFFFFAD09FFFFFFFFFF09FFFF77
:1017C000FFFFFFF6FFFFFFFFFFFFFFFFFFFFFFFF32
:1017D000FFFFFFFFFFFFFFFFFFFFFFFFFFFFFFFF19
:1017E000FFFF0900A4FFFFFF0000A4FFFFFF0900A7
:1017F000A4FFFFFFAD00A4FFFFFFFFADA4FFFFFFAD
:10180000FFFFFFFFFFFFFFFFFFFFFFFFFFFFFFFFE8
:10181000FFFFAD09A4FFFFFFAD09A4FFFFFFAD0966
:10182000090009F6AD09A4A4A4F6AD09A4FFFFFFC1
:10183000AD09525252F6AD00090900F6FFFFFFFF55
:10184000FFFFFFFFFF5209FFFFFFFF5209FFFFFFEE
:10185000FF5209FFFFFFFF5209FFFFFFFF5209FF81
:10186000FFFFFF520052FFFFFF5B0009FFFFFFFF7A
:10187000FFFFFFFFFFFFFFADFFFFFFFFFFADFFFF1C
:10188000FFFFFFADFFFFFFFFFFADFFFFFFFFFFAD5E
:101890005252FFFFFFAD0909FFFFFFADFFFFFFFF42
:1018A000FFFF00A4FFFFFFFF00A4FFFFFFFF0009F1
:1018B0000900F6FF00A4A4A4F6FF00A4FFFFFFFFA9
:1018C00000525252F6FF00090900F6FFFFFFFFFF2A
:1018D000FFFFFFFFAD005BFFFFFF5B09F6FFFFFFB0
:1018E0005B09FFFFFFFF5B09FFFFFFFFA400A4FFF1
:1018F000FFFFF609095BFFFFFFAD0909FFFFFFFFCF
:10190000FFF6A400ADFFFFFFFFADFFFFFFFFFFFFEE
:10191000FFFFFFFFFFF6FFFFFFFFAD09ADFFFFFF7A
:101920000909F6FFFFFF09A4FFFFFFFFFFFFFFFF0D
:10193000FFFFF65209ADF6FFFF5B09F6FFFFFF5B05
:1019400009F6FFFFFF5B09F6FFFFFF5B09F6FFFFEC
:10195000FF5B09F6FFFFFF5B09FFFFFFFFFFFFFFD4
:10196000FFFFFFFFF600ADFFFFFFF600ADFFFFFF3B
:10197000F6000909FFFFF6005252FFFFF600ADFF27
:10198000FFFFF600ADFFFFFFF609F6FFFFFFFFFFC9
:10199000FFFF5B00ADFFFFFFA400F6FFFFF6005264
:1019A000FFFFFFF60052FFFFFFF6A400F6FFFFFF68
:1019B000AD00F6FFFFFFAD00F6FFFFFFFFFFFFFFEB
:1019C000FFFF0909F6F65209095BFFFFF60009FF60
:1019D000FFFFFF0009F6FFFFF6000952FFFFA4001A
:1019E0005B0052520052FF52000009F6FFFFF6F66C
:1019F000FFFFF6FFFFFF5200ADFFFFFF5200A4FF05
:101A0000FFFF5200ADFFFFFF5200ADFFFFFF52008E
:101A1000FFFFFFFF5200FFFFFFFF0909FFFFFFFF6E
:101A2000FFFF52FFA400F6FF00ADA400F6FF5252E4
:101A3000A400F6FFAD005200F6FFFF520000F6FFD3
:101A4000FFA40000F6FFFFFF0952FFFFFFFFFFFFAB
:101A5000FFFFFFF6095BFFFFFFF6095BFFFFFFF6E5
:101A6000095BFFFFFFF6095BFFFFFFF6095BFFFF66
:101A7000FFF6095BFFFFFFFF095BFFFFFFFFFFFFB3
:101A8000FFFFFFF60052FFADFFAD00F6FFFFFFA422
:101A900000F6FFFFFFAD00F6FFFFFFAD00A4FFF66D
:101AA000FFF609095B09FFFFAD090000FFFFFFFF1B
:101AB000F6FF00ADFFFFAD00A4FFFFFFAD00FFFF8D
:101AC000FFFFFF52F6FFFFFFFFFF00ADFFFFF6092C
:101AD00000F6FFFFAD00A4FFFFFFFF5BFFFFFFFF6E
:101AE000FFFFA4FF5B52FFFF52ADFFFFFFFF0009A6
:101AF00000A4FFFFAD520009F6FFF6FFA400ADFF02
:101B000052A40909FFFF090909A4FFFFFFF6FFFF1F
:101B1000FFFFFF0900000000FF0900000000FF09AF
:101B200000000000FF0900000000FF0900000000A5
:101B3000FF0900000000FF0900000000FF0900008D
:101B40000000000000000000000000000000000095
:101B50000000000000000000000000000000000085
:101B6000000000000000000000000009000000006C
:101B7000000A00000000000000000000000000005B
:101B80000000000000000000000000000000000055
:101B9000000000000A130900011C666E5C12126648
:101BA000AE6E00000000B6FF0000001366FF0000EC
:101BB0000A656EFF00000A656EFF000000095D6E99
:101BC000135C5C13656E6E6E6E6EAEB7B7AEAEAE86
:101BD000AEB7FFFFFFFFFFFFFFFFFFFFFFFFFFFFAE
:101BE000FFFFFFFFFFFFFFFFFFFFFFFFFFFFFFFF05
:101BF000FFFFFFFFFFFFFFFFFFFFFFFFAEFFFFFF46
:101C0000FFFFFFFFFFFFFFFFFFFFFFFFFFFFFFFFE4
:101C1000FFFFFF5BFFFFFFFFFF5BFFFFFFFFAD006D
:101C2000FFFFFFFFAD00FFFFFFFFAD00FFFFFFF66F
:101C30000000520000000000520000000000000000
:101C40000000000000000000000000000000000094
:101C50000000000000000000000000000000000084
:101C6000001200000000091300000009656E00006A
:101C70000165AEB700126666AFB7001CAEAFB7B76E
:101C80000A66AEB7B7B75DAEB7B7B7B766AFB7B7A7
:101C9000B7B76E5C1C6E6E6EB765656EAEB7B76E2D
:101CA0006EB7AFB7B7AEB7B7B7B7B7B7B7B7B7B71E
:101CB000B7B7B7B7B7B7B7B7B7B7B7B7B7B7B7F774
:101CC000B7B7AEAEAEB7AEAEB7B7B7AEAEB7B7B7E3
:101CD000B7B7AEAEB7B7B7B7B7B7B7B7B7B7B7B7A6
:101CE000F7B7B7B7B7B7F7F7B7B7B7B7B7F7F7B744
:101CF000B7B7AEFFFFFFFFFFB7AEFFFFFFFFB7AE07
:101D0000FFFFFFFFB7B7B7FFFFFFB7B7FFFFFFFF4B
:101D1000B7B7B7FFFFFFB7B7B7FFFFFFB7B7B7FF5B
:101D2000FFFFFFFFFFF60000FFFFFFF60000FFFFD1
:101D3000FF000000FFFFFF000000FFFFFF000000AA
:101D4000FFFFFF000000FFFFFF000000FFFFFF009C
:101D50000000000000000965000000015C6E00004A
:101D6000000A66B70000005DAEB700005C6EAFB75A
:101D7000000A6EB7B7B7000AAEB7B7B700136EB7B1
:101D8000B7B76EB7B7B7B7F7AEB7B7B7B7F7B7B7B5
:101D9000B7B7B7B7B7B7B7B7B7B7B7B7B7B7B7B7D3
:101DA000B7B7B7B7F7AEB7B7B7B7B713B7B7B7F7F0
:101DB0006E00B7B7F7F7B7B7B7B7B7B7B7B7B7B733
:101DC000B7B7B7B7B7B7B7B7B7B76E6EB76EB7B77E
:101DD0001CAEB75CB7B712AE6613B7B70A650A1286
:101DE0006EAEB7B7B7B7B7B7B7B7B7B7B7B7B7B7D5
:101DF000B7B7B7B7B7B7B7B7B7B7B7B7B7B7B7B773
:101E0000AEB7B7B7B7B7AEB7B7B7B7B7B7B7B7B774
:101E1000B7B7B7B7B76EFFFFB7B7B76EFFFFB7B7C4
:101E2000B7B7FFFFB7B7B7B7FFFFB7AFB7AFFFFFA2
:101E3000AFB7B7B7FFFFB7AFB7AFFFFFB7B7AFB732
:101E4000FFFFFFFFFF000000FFFFFF000000FFFF9C
:101E5000FF000000FFFFFF000000FFFFFF00000089
:101E6000FFFFFF000000FFFFFF000000FFFFFF007B
:101E700000000066B7B7B7B70966AFB7AFB70A6675
:101E8000B7AFB7B70A66B7B7AFAF0966AEB7B713A4
:101E90000166AEAE6501005DAEB76501000A6EB7C2
:101EA000AE09B7B7B7B71300B7B7AE650000B76EE6
:101EB0006E0A0000665C660A0000125C6E5C000040
:101EC000015C6E130000000A5C09000000000100C4
:101ED0000000090A00095D660A5C09000A65011232
:101EE00009000012000000000000000000000000D7
:101EF00000000000000000000000000000000000E2
:101F00000000B7B7B76EAEAF6E6E6665B7B7651354
:101F10005DAEB7B7130165B7B7B700005CB7AEB732
:101F200000001365091200000A660A5D000009AE90
:101F30005C65B7B7B7B7FFFFB7AFB7B7FFFFB7AFCE
:101F4000B7B7FFFFB7B7B7B7FFFFB7B7B7B7AEFFC2
:101F50001C656EB76EFF6EB7B7B76EFFB7B7B7B792
:101F6000FFFFFFFFFF000000FFFFFF000000FFFF7B
:101F7000FF000000FFFFFF000000FFFFFF00000068
:101F8000FFFFFF000000FFFFFF000001FFFFFF0059
:101F9000001300000A656E0A000000001413000020
:101FA0000000091300000000011300000101136587
:101FB000015C5D5D65665DB7B7B76E666EB7B7B756
:101FC000AF660000000000000000000000000000FC
:101FD000000A00000100126E5C00660A5CAE661327
:101FE000AE6666B7AE656EB7B7B7B76E66AEB7B773
:101FF000B7AE0000000100000000005C0A00000015
:102000005CB75C001366B7F7AE5D6EB7B7B7B7B72E
:10201000B7B7B7B7B7AFAFB7B7B7B7AFAFB7B7B770
:10202000B7AF000009AE656500005CB76666005C8E
:10203000B7B7B7AF6EB7B7B7B766F7B7B7B7B665E5
:10204000B7B7B7B7B7AFB7B7B7B7B7B7AFB7B7B730
:10205000B7B7B7AEB7B7FFFFB7B7B7B7FFFFF7B7B9
:10206000B7B7FFFF66B7B7B7FFFF136EB7B7FFFF8E
:1020700066B7B7AFFFFFAEB7B7FFFFFFB7AFAFFFB2
:10208000FFFFFFFFFF000965FFFFFF000A6EFFFF74
:10209000FF00095DFFFFFF000113FFFFFF00005C71
:1020A000FFFFFF00005CFFFFFF00005CFFFFFF0081
:1020B0000013B7B7B7B7B75DB7AFB7B76E65B7B708
:1020C0006E6E6E66AEAE6E6E5C13AE656E1C00001C
:1020D000AE65660A00016E6E660A00096E6E6E5C81
:1020E00009136566AEB7B7AF65AEAEB7B7AF66AF4B
:1020F000B7AFB7AF5DB7B7B7B7AF126EB7AEB7B7D9
:102100000A65B7AEB7B71365B7B7B7B75C6EAFAE12
:10211000B7B7B7B7B7B7B7AFB7B7B7B7B7B7B7B757
:10212000AFB7B7B7AFB7B7B7B7B7AFB7B7B7B7B757
:10213000AFB7B7B7B7B7AFB7B7B7B7B7B7B7B7B73F
:10214000B7B7B7B7B7B7B7B7AFB7B7B7B7B7B7B727
:10215000B7B7B7B7B7B7B7B7B7B7B7B7B7B7B7F7CF
:10216000B7AFB7B7B7B7B76EB7B7B7FFB7FFFFFF30
:10217000FFFFB7B7B7FFFFFFB7B7B7FFFFFFB7F76F
:10218000FFFFFFFFB7AEFFFFFFFFB7FFFFFFFFFF40
:10219000FFFFFFFFFFFFFFFFFFFFFFFFFFFFFFFF4F
:1021A000FFFFFFFFFF000000FFFFFF000000FFFF39
:1021B000FF000009FFFFFF000009FFFFFF00001301
:1021C000FFFFFF00001CFFFFFF000165FFFFFF0096
:1021D000096613656E661C5D091365B7666E135C50
:1021E0006EB76EAE666EB7B76E6666B7B7B76EB7E8
:1021F0006EAFB7B7FFB6B7AFB7B7FFFFB7AFB7B7F9
:10220000FFFF6EB7B7B7B7B7B7B76EAFB7B7B76EB1
:102210006EB7B7B76E6EAFB7AFB7B7AFAFAFAFB759
:10222000B7B7B7B7AFFFAEB7AF6EFFFFFFFFFFFFA8
:10223000FFFFB7B7B7B7B7B7B7B7B7B7B7B76EAFEF
:10224000B7B7B7F7FFB7AEB7FFFFFFFFFFFFFFFF5F
:10225000FFFFFFFFFFFFFFFFFFFFFFFFFFFFFFFF8E
:10226000FFFFAFFFFFFFFFFFFFFFFFFFFFFFFFFFCE
:10227000FFFFFFFFFFFFFFFFFFFFFFFFFFFFFFFF6E
:10228000FFFFFFFFFFFFFFFFFFFFFFFFFFFFFFFF5E
:10229000FFFFFFFFFF0013AEFFFFFF005CB7FFFF74
:1022A000FF00136EFFFFFF000965FFFFFF00136EC5
:1022B000FFFFFF0013AEFFFFFF0012AEFFFFFF00A6
:1022C000126EB7AFB7B7FFFFB7B7B7B7FFFF6E6E06
:1022D000AEB7FFFF666E6EB7FFFF6E6EAFB7FFFF64
:1022E000B7B7B7B7FFFFB7B7B7B7FFFFAFB7B7B766
:1022F000FFFFFFFFFF0013AEFFFFFF0013AEFFFF66
:10230000FF0012AEFFFFFF000A66FFFFFFF6011C91
:10231000FFFFFFF6015DFFFFFFF60165FFFFFFF620
:102320000965B7AFB7B7FFFFB7B7B7B7FFFFB7B725
:10233000B7B7FFFF6E6E6EB7FFFF66666EAFFFFF4B
:102340006E6EAFB7FFFFAEB7B7B7FFFFAEB7B7B7A9
:10235000FFFFFFFFFFF60966FFFFFFF6096EFFFFB5
:10236000FFF60A6EFFFFFFFFAD66FFFFFFFFF6659A
:10237000FFFFFFFFF665FFFFFFFFF7AEFFFFFFFF69
:10238000FFB7B7B7B7B7FFFFB7B7B7B7FFFFB7B775
:10239000B7B7FFFFB7B7B7B7FFFFB7B7B7B7FFFF1D
:1023A000B7B7B7B7FFFFB7B7B7B7FFFFB7B7B7FF55
:1023B000FFFFFFFFFFFFFFFFFFFFFF77FFFFFFFFB5
:1023C000FF1D00FFFFFFFF1D7700FFFFFF141D7FB4
:1023D000FFFFFF5B141DFFFF5BFFFFFFFFFF5BFFC6
:1023E000FFFFFF00FFFFFFFFFF001DFFFFFF007F5C
:1023F0001DFFFFFF007714FFFFFF771D14FFFFFF96
:102400001D145BFFFFFFFFFFFF5BFFFFFFFFFF5B95
:10241000FFFFFFFFFFFFFFFFFFFFFFFFFFFFFFFFCC
:10242000FFFFFFFFFFFFFFFFFFFFFFFFFFFFFFFFBC
:10243000FFFFFFFFFFFFFFFFFFFFFFFFFFFFFFFFAC
:10244000FFFFFFFFFFFFFFFFFFFF005B00FFFFFF3E
:1024500000F65BFFFFA400F600FFA4FF00F6005BA0
:10246000A4FF00F60000A4FFFFFFFFFFA4FFFFFF93
:10247000FFFFFFFFFFFFFFFFFF005B00FFFFFFFF0E
:102480000000FFFFFF5B0000A4FFFF000000FFA4AF
:102490005B000000FFA4FFFFFFFFFFA4FFFFFFFFA3
:1024A000FFA4FFFFFFFFFFFF54FFFFFFFFFF54FFED
:1024B000FFFFFFFF155EFFFF54FFFF15FF5EFFFFED
:1024C000A4FFFFFFA4FFA4FFFFFFA4FFA4FFFFFFE3
:1024D000A4FFFFFFFFFFFFFFFFFF1300FFFFFFFF52
:1024E000131F00FFFFA413370AFFA4FF137F13007D
:1024F000A4FF137F1342A4FFFFFFFFFFA4FFFFFF12
:10250000FFFFFFFFFFFFFFFFFFFF0013FFFFFFFFC6
:102510000A13FFFFFF000A13A4FF00041313FFA414
:102520000A061313FFA4FFFFFFFFFFA4FFFFFFFF37
:10253000FFA43030303030302020202020201818E8
:10254000181818181818181818181010101010103B
:10255000101010101010000000000000000000001B
:102560000000FFFFFFFF7777FFFFFF777F7FFFFF11
:10257000FF777F00FFFFFF777F00FFFFFF777F7F01
:10258000FFFFFF5B777FFFFF5BFFFFFFFFFF5BFF4F
:10259000FFFF7777FFFFFFFF7F7F77FFFFFF007F62
:1025A0007FFFFFFF7F7F77FFFFFF7F776FFFFFFFDB
:1025B000776F5BFFFFFFFFFFFF5BFFFFFFFFFF5B2F
:1025C000FFFFFFFFFFFFFFFFFFFF00F60000FFFF21
:1025D00000F60000FFA400F60000A4FF00F60000D3
:1025E000A4FF00F60000A4FFFFFFFFFFA4FFFFFF12
:1025F000FFFFFFFFFFFFFFFF00000000FFFF0000E5
:102600000000FFFF00000000A4FF00000000FFA486
:1026100000000000FFA4FFFFFFFFFFA4FFFFFFFF7C
:10262000FFA4FF5E5E5EFFFF5E275D275EFF5E5DCF
:1026300027275EFF5E2727275EFFFF5E5E5EFFFFA8
:10264000A4FFFFFFA4FFA4FFFFFFA4FFA4FFFFFF61
:10265000A4FFFFFFFFFFFFFFFFFF137F138CFFFFB0
:10266000137F138CFFA4137F138CA4FF137F138C91
:10267000A4FF137F138CA4FFFFFFFFFFA4FFFFFF46
:10268000FFFFFFFFFFFFFFFF13061313FFFF1306FC
:102690001313FFFF13061313A4FF13061313FFA452
:1026A00013061313FFA4FFFFFFFFFFA4FFFFFFFFAD
:1026B000FFA4FFFFFFFFFFFFFFFFFFFFFFFFFFFF85
:1026C000FFFFFFFFFFFFFFFFFFFFFFFFFFFFFFFF1A
:1026D000FFFFFFFFFFFFFFFFFFFFFFFFFFFFFFFF0A
:1026E000FFFFFFFF0000FFFFFFFF0000FFFFFFFFF6
:1026F0000000FFFFFFFF00FFFFFFFFFF00FFFFFFE6
:10270000FFFFFFFFFFFFFFFF00FFFFFFFFFFFFFFD8
:10271000FFFFFF00FFFF00FF0000FF0000FF00FFC2
:10272000FF00FFFFFFFFFFFFFFFFFFFFFFFFFFFFB8
:10273000FFFFFFFFFFFFFFFFFFFFFFFFFFFFFFFFA9
:10274000FFFFFFFF0000FFFFFF00FFFF00FF00FF94
:102750000000FF0000FF00FFFF0000FF00FFFF0080
:1027600000FF0000FF00FF00FFFF00FFFFFF000071
:10277000FFFFFF00FFFFFFFFFF000000FFFF00FF64
:10278000FFFFFFFFFF0000FFFFFFFFFFFF00FFFF56
:10279000000000FFFFFFFFFF00FFFFFFFFFFFFFF45
:1027A000FFFFFF00FFFF00FF0000FFFF00FFFFFF34
:1027B000FF00FFFFFFFF00FFFFFFFF00FFFFFFFF26
:1027C00000FFFF0000FF00FFFF00FFFFFFFFFFFF14
:1027D000FFFFFF00FFFFFFFF00FF00FFFFFF00FF05
:1027E00000FFFFFFFF00FFFFFFFF00FF00FF00FFF4
:1027F00000FFFF00FFFFFF0000FF00FFFFFFFFFFE4
:10280000FFFFFFFF00FFFFFFFF0000FFFFFFFF00D4
:10281000FFFFFFFFFFFFFFFFFFFFFFFFFFFFFFFFC8
:10282000FFFFFFFFFFFFFFFFFFFFFFFFFFFFFFFFB8
:10283000FFFFFFFF00FFFFFFFF00FFFFFFFFFF00A5
:10284000FFFFFFFFFF00FFFFFFFFFF00FFFFFFFF96
:10285000FF00FFFFFFFFFFFF00FFFFFFFFFFFFFF86
:10286000FFFFFF00FFFFFFFFFFFF00FFFFFFFFFF76
:1028700000FFFFFFFFFF00FFFFFFFFFF00FFFFFF65
:10288000FFFF00FFFFFFFF00FFFFFFFFFFFFFFFF56
:10289000FFFFFFFFFFFFFFFFFF00FF00FFFFFF0045
:1028A0000000FFFF0000000000FFFF000000FFFF2E
:1028B000FF00FF00FFFFFFFFFFFFFFFFFFFFFFFF26
:1028C000FFFFFFFFFFFFFFFFFFFF00FFFFFFFFFF17
:1028D00000FFFFFF0000000000FFFFFF00FFFFFF01
:1028E000FFFF00FFFFFFFFFFFFFFFFFFFFFFFFFFF7
:1028F000FFFFFFFFFFFFFFFFFFFFFFFFFFFFFFFFE8
:10290000FFFFFFFFFFFFFFFFFFFFFFFFFFFFFFFFD7
:10291000FFFF00FFFFFFFF0000FFFFFFFF00FFFFC3
:10292000FFFFFFFFFFFFFFFFFFFFFFFFFFFFFFFFB7
:10293000FFFFFFFF0000000000FFFFFFFFFFFFFFA2
:10294000FFFFFFFFFFFFFFFFFFFFFFFFFFFFFFFF97
:10295000FFFFFFFFFFFFFFFFFFFFFFFFFFFFFFFF87
:10296000FFFFFFFFFFFFFFFFFFFFFFFFFFFFFFFF77
:10297000FF0000FFFFFFFF0000FFFFFFFFFFFFFF63
:10298000FFFFFFFFFFFFFFFFFFFFFFFF00FFFFFF56
:10299000FF00FFFFFFFF00FFFFFFFF00FFFFFFFF44
:1029A00000FFFFFFFFFFFFFFFFFFFFFFFFFFFFFF36
:1029B000FFFFFF0000FFFFFF00FFFF00FFFF00FF22
:1029C000FFFF00FF00FFFFFF00FF00FFFFFF00FF12
:1029D00000FFFFFF00FFFF000000FFFFFFFFFFFF02
:1029E000FFFFFFFF00FFFFFFFF0000FFFFFFFFFFF4
:1029F00000FFFFFFFFFF00FFFFFFFFFF00FFFFFFE4
:102A0000FFFF00FFFFFFFF000000FFFFFFFFFFFFD2
:102A1000FFFFFF0000FFFFFF00FFFF00FFFFFFFFC2
:102A2000FFFF00FFFFFF0000FFFFFF00FFFFFFFFB2
:102A300000FFFFFFFFFF0000000000FFFFFFFFFFA0
:102A4000FFFFFF0000FFFFFF00FFFF00FFFFFFFF92
:102A5000FFFF00FFFF000000FFFFFFFFFFFF00FF81
:102A600000FFFFFF00FFFF000000FFFFFFFFFFFF71
:102A7000FFFFFFFF00FFFFFFFF00FF00FFFF00FF62
:102A8000FF00FFFF00FFFF00FFFF0000000000FF4E
:102A9000FFFFFF00FFFFFFFFFF00FFFFFFFFFFFF44
:102AA000FFFF00000000FFFF00FFFFFFFFFF00002F
:102AB00000FFFFFFFFFFFF00FFFF00FFFFFF00FF22
:102AC000FF00FFFF00FFFFFF0000FFFFFFFFFFFF12
:102AD000FFFFFFFF0000FFFFFF00FFFFFFFF00FF02
:102AE000FFFFFFFF000000FFFFFF00FFFF00FFFFF1
:102AF00000FFFFFF00FFFF000000FFFFFFFFFFFFE1
:102B0000FFFF00000000FFFFFFFFFFFF00FFFFFFD0
:102B1000FF00FFFFFFFF00FFFFFFFF00FFFFFFFFC2
:102B2000FF00FFFFFFFFFF00FFFFFFFFFFFFFFFFB3
:102B3000FFFFFF0000FFFFFF00FFFF00FFFF00FFA0
:102B4000FFFF00FFFF000000FFFF00FFFFFF00FF8F
:102B500000FFFFFF00FFFF000000FFFFFFFFFFFF80
:102B6000FFFFFF0000FFFFFF00FFFF00FFFF00FF70
:102B7000FFFF00FFFF00000000FFFFFFFFFF00FF5F
:102B800000FFFFFF00FFFF000000FFFFFFFFFFFF50
:102B9000FFFFFFFFFFFFFFFFFFFFFFFFFFFFFFFF45
:102BA00000FFFFFFFF0000FFFFFFFFFFFFFFFFFF32
:102BB000FFFF00FFFFFFFF0000FFFFFFFFFFFFFF22
:102BC000FFFFFFFFFFFFFFFFFFFFFFFFFFFFFFFF15
:102BD00000FFFFFFFF0000FFFFFFFFFFFFFFFFFF02
:102BE000FFFF00FFFFFFFF0000FFFFFFFF00FFFFF1
:102BF000FFFFFFFFFFFF00FFFFFFFF00FFFFFFFFE3
:102C000000FFFFFFFF00FFFFFFFFFFFF00FFFFFFD1
:102C1000FFFFFF00FFFFFFFFFFFF00FFFFFFFFFFC2
:102C2000FFFFFFFFFFFFFFFFFFFFFFFFFFFF0000B2
:102C3000000000FFFFFFFFFFFFFFFFFFFFFFFFFFA1
:102C40000000000000FFFFFFFFFFFFFFFFFFFFFF8F
:102C5000FFFFFF00FFFFFFFFFFFF00FFFFFFFFFF82
:102C6000FF00FFFFFFFFFFFF00FFFFFFFF00FFFF71
:102C7000FFFF00FFFFFFFF00FFFFFFFFFFFFFFFF62
:102C8000FFFFFF000000FFFF00FFFFFF00FFFFFF4F
:102C9000FFFF00FFFFFFFF00FFFFFFFF00FFFFFF41
:102CA000FFFFFFFFFFFFFFFF00FFFFFFFFFFFFFF33
:102CB000FFFFFF000000FFFF00FFFFFF00FF00FF1E
:102CC000FF0000FF00FF00FF00FF00FFFF00FFFF0D
:102CD00000FFFFFFFFFFFF000000FFFFFFFFFFFF00
:102CE000FFFF000000FFFFFF00FFFF00FFFF00FFEE
:102CF000FFFF00FF00FFFFFF00FF0000000000FFDC
:102D000000FFFFFF00FF00FFFFFF00FFFFFFFFFFCF
:102D1000FFFF000000FFFFFF00FFFF00FFFF00FFBD
:102D2000FFFF00FF00000000FFFF00FFFFFF00FFAC
:102D300000FFFFFF00FF00000000FFFFFFFFFFFF9D
:102D4000FFFFFF0000FFFFFF00FFFF00FFFF00FF8E
:102D5000FFFF00FF00FFFFFFFFFF00FFFFFFFFFF80
:102D600000FFFFFF00FFFF000000FFFFFFFFFFFF6E
:102D7000FFFF000000FFFFFF00FFFF00FFFF00FF5D
:102D8000FFFF00FF00FFFFFF00FF00FFFFFF00FF4E
:102D900000FFFFFF00FF00000000FFFFFFFFFFFF3D
:102DA000FFFF000000FFFFFF00FFFFFFFFFF00FF2E
:102DB000FFFFFFFF00000000FFFF00FFFFFFFFFF1E
:102DC00000FFFFFFFFFF0000000000FFFFFFFFFF0D
:102DD000FFFF000000FFFFFF00FFFFFFFFFF00FFFE
:102DE000FFFFFFFF00000000FFFF00FFFFFFFFFFEE
:102DF00000FFFFFFFFFF00FFFFFFFFFFFFFFFFFFE1
:102E0000FFFFFF0000FFFFFF00FFFF00FFFF00FFCD
:102E1000FFFF00FF00FFFFFFFFFF00FFFF0000FFBD
:102E200000FFFFFF00FFFF00000000FFFFFFFFFFAC
:102E3000FFFF00FFFFFFFFFF00FFFFFF00FF00FF9E
:102E4000FFFF00FF0000000000FF00FFFFFF00FF8A
:102E500000FFFFFF00FF00FFFFFF00FFFFFFFFFF7E
:102E6000FFFF00000000FFFFFFFF00FFFFFFFFFF6D
:102E700000FFFFFFFFFF00FFFFFFFFFF00FFFFFF5F
:102E8000FFFF00FFFFFF0000000000FFFFFFFFFF4C
:102E9000FFFFFFFFFF0000FFFFFFFFFF00FFFFFF3F
:102EA000FFFF00FFFFFFFFFF00FF00FFFFFF00FF2E
:102EB000FF00FFFF00FFFFFF0000FFFFFFFFFFFF1E
:102EC000FFFF00FFFF00FFFF00FFFF00FFFF00FF0D
:102ED00000FFFFFF0000FFFFFFFF00FF00FFFFFFFD
:102EE00000FFFF00FFFF00FFFFFF00FFFFFFFFFFEE
:102EF000FFFF00FFFFFFFFFF00FFFFFFFFFF00FFDF
:102F0000FFFFFFFF00FFFFFFFFFF00FFFFFFFFFFCF
:102F100000FFFFFFFFFF0000000000FFFFFFFFFFBB
:102F2000FFFF0000FF00FFFF00FF00FF00FF00FFAA
:102F300000FF00FF00FF00FF00FF00FFFFFF00FF9A
:102F400000FFFFFF00FF00FFFFFF00FFFFFFFFFF8D
:102F5000FFFF000000FFFFFF00FFFF00FFFF00FF7B
:102F6000FFFF00FF00FFFFFF00FF00FFFFFF00FF6C
:102F700000FFFFFF00FF00FFFFFF00FFFFFFFFFF5D
:102F8000FFFFFF0000FFFFFF00FFFF00FFFF00FF4C
:102F9000FFFF00FF00FFFFFF00FF00FFFFFF00FF3C
:102FA00000FFFFFF00FFFF000000FFFFFFFFFFFF2C
:102FB000FFFF000000FFFFFF00FFFF00FFFF00FF1B
:102FC000FFFF00FF00000000FFFF00FFFFFFFFFF0B
:102FD00000FFFFFFFFFF00FFFFFFFFFFFFFFFFFFFF
:102FE000FFFFFF0000FFFFFF00FFFF00FFFF00FFEC
:102FF000FFFF00FF00FFFFFF00FF00FF00FF00FFDB
:1030000000FFFF00FFFFFF0000FF00FFFFFFFFFFCB
:10301000FFFF000000FFFFFF00FFFF00FFFF00FFBA
:10302000FFFF00FF00000000FFFF00FFFF00FFFFA9
:1030300000FFFFFF00FF00FFFFFF00FFFFFFFFFF9C
:10304000FFFFFF0000FFFFFF00FFFF00FFFFFF008B
:10305000FFFF00FFFFFF00FFFFFFFFFFFF00FFFF7D
:1030600000FFFFFF00FFFF000000FFFFFFFFFFFF6B
:10307000FFFF0000000000FFFFFF00FFFFFFFFFF5A
:1030800000FFFFFFFFFF00FFFFFFFFFF00FFFFFF4D
:10309000FFFF00FFFFFFFFFF00FFFFFFFFFFFFFF3E
:1030A000FFFF00FFFFFF00FF00FFFFFF00FF00FF2B
:1030B000FFFF00FF00FFFFFF00FF00FFFFFF00FF1B
:1030C000FF00FFFF00FFFFFF0000FFFFFFFFFFFF0C
:1030D000FFFF00FFFFFF00FF00FFFFFF00FF00FFFB
:1030E000FFFF00FF00FFFFFF00FF00FFFFFF00FFEB
:1030F000FF00FF00FFFFFFFF00FFFFFFFFFFFFFFDD
:10310000FFFF00FFFFFF00FF00FFFFFF00FF00FFCA
:1031100000FF00FF00FF00FF00FF00FF00FF00FFB7
:1031200000FF00FF00FFFF00FF00FFFFFFFFFFFFAA
:10313000FFFF00FFFFFF00FFFF00FF00FFFFFF009A
:10314000FF00FFFFFFFF00FFFFFFFF00FF00FFFF8B
:10315000FF00FF00FFFF00FFFFFF00FFFFFFFFFF7B
:10316000FFFF00FFFFFF00FF00FFFFFF00FFFF006A
:10317000FF00FFFFFFFF00FFFFFFFFFF00FFFFFF5C
:10318000FFFF00FFFFFFFFFF00FFFFFFFFFFFFFF4D
:10319000FFFFFF000000FFFFFFFFFF00FFFFFFFF3B
:1031A00000FFFFFFFF00FFFFFFFF00FFFFFFFFFF2C
:1031B00000FFFFFFFFFF00000000FFFFFFFFFFFF1A
:1031C000FFFFFFFF0000FFFFFF00FFFFFFFFFF000B
:1031D000FFFFFFFF00FFFFFFFFFFFF00FFFFFFFFFD
:1031E000FF00FFFFFFFFFFFF0000FFFFFFFFFFFFEC
:1031F000FFFFFFFF0000FFFFFF00FFFF00FF00FFDA
:103200000000FF0000FF00FFFF0000FF0000FF00C4
:10321000FF00FFFF00FFFFFF0000FFFFFFFFFFFFBA
:10322000FFFFFF0000FFFFFFFFFFFF00FFFFFFFFAB
:10323000FF00FFFFFFFFFFFF00FFFFFFFF00FFFF9B
:10324000FFFFFF00FFFFFF0000FFFFFFFFFFFFFF8B
:10325000FFFFC7C7C7C7C7C7C7C7C7C7C7C7C7C78E
:10326000C7C7C7C7C7C7C7C7C7C7C7C7C7C7C7C7EE
:10327000C7C7C7C7C7C7C7C7C7C7C7C7C7C7C7C7DE
:10328000C7C740010102030405060708090A0B0C21
:103290000D0E0F101112131415161718191A1B1CE6
:1032A0001D1E1F202122232425262728292A2B2CD6
:1032B0002D2E2F303132333435363738393A3B3CC6
:1032C0003D3E0001FFFFFFFFFFFFFFFFFFFFFFFF8E
:1032D000FFFFFFFFFFFFFFFFFFFFFFFFFFFFFFFFFE
:1032E000FFFFFFFFFFFFFFFFFFFFFFFFFFFFFFFFEE
:1032F000FFFFFFFFFFFFFFFFFFFFFFFFFFA4F6FF42
:10330000FFFFADADADF6FFFF5AEDADADFFF6A35A31
:10331000ACF6FFFFADA4ADA4FFFFAD9BF6ADFFFF84
:10332000FFF65AA4FFFFFFFFFFFFFFFFFFFFFFFFB6
:10333000FFFFFFFFFFFFF6F55BEDFFFFFFFF5BA465
:10334000FFFFA4A35BADFFFFA39BA4FFFFFFAC5B4C
:10335000ADFFFFFFFFFFFFFFFFFFFFFFFFFFFFFFCF
:10336000FFF6F6FFFFFFFFADA4FFFFFFFFFFADADD0
:10337000ADA4FFFFF6A3A4A4FFFFFFAD52A4FFFF7F
:10338000F6F6A4ADFFFFFFFFFFFFFFFFF6F6F6FF27
:10339000FFFFAD5BF6FFADA39BA4FFFF5BA3ADFFFB
:1033A000FFFFA45AACFFFFFFFEA45AFEFFFFFFADD4
:1033B0005AA3FFFFFFFFFFFFFFFFFFFFFFFFFFFF1E
:1033C000FFF5FFFFF6ADFFF6F6FFF5ACFFFFFF5B85
:1033D000A4A3FFFFFFACA4ADFFFFF6FFACACFFFF63
:1033E000F6A35A5BFFFFFFFFFFFFA4F6F6FFFFFF08
:1033F000ACF6ADFFFFFFFF5BACFFFFFFFFF69BF5F9
:10340000FFFFFFFFF6F5FFFFADF6ADA4FEFF5A9BF1
:10341000ADADFFFFFFFFFFFFFFFFFFFFFFFFF6ADBB
:10342000FFFFF6F6F5ADFFFFF5A4ADADFFFFACACC9
:10343000ACA4FFFF5A5AA4A4FFFFAD5B5A9BFFFF49
:10344000F5ADA45BADFFFFFFFFFFFFACF6FFFFFF95
:10345000FFFEEDFFFFFFFFFFF6FFFFFFA4FFF6FFFC
:10346000FFFF52A4EDFFFFFFA4A3ADFEF6FF5B5BE1
:103470005AA3FFFFFFFFFFFFFFFFFFFFF6F6FFFF6F
:10348000FFFF9BADF6F6FFFFA45BA39BFFFFAD9B89
:10349000A3A4FFFFF5A35B9BFFFFADA45B5BFFFF56
:1034A000F6A3A49BFFFFFFFFFFFFFFFFFFFFFFFF50
:1034B000FFFFFFFFFFFFEDFFFFFFFFFFADA4ADFF2D
:1034C000FFFFA3A3ACACF6FF5B5BA4A4ADFFA3F628
:1034D000AD5BACFFFFFFF6FFFFFFFFFFF6ADACF605
:1034E000FFFFF5FFAD9BFFF6F6F6A3ACFFFF5AA377
:1034F000A49BFFFFA3A4FFA3FFFFACA4AD5BFFFF52
:10350000FFAD5B9BFFFFFFFFFFFFFFFFFFFFFFFF25
:10351000EDFFFFFFFFFFADF5FFFFFFFFF6ADA3F6E9
:10352000FFFFA39B52A3F6FF5BADA49BA4F6A3A44D
:10353000F5ADFFFFFFFFFFFFFFFFFFFFF5FFFFED13
:10354000FFF6ADFFF6ACFFFFACFFEDADFFFFF6A45D
:10355000ADA3FFFFFE9B9BADFFFFFF5BA3A4FFFF9F
:10356000FFAC5BA4FFFFFFFFFFFFFFFFFFFFFFFFBD
:10357000FFFFF6FFFFFFFFFFF6F6FFFFADFFADA376
:10358000F6FFFFFFFFACEDFFA4A4ACA4ADFFADF6CA
:103590009BADFFFFFFFFFFFFA35BFFFFFFF6A4A4B0
:1035A000FFFFFFFFAD9BFFFFFFFFF6ADFFFFFFFF3C
:1035B000FFF6FFFFFFFFFFFFFFFFFFFFFFFFFFFF24
:1035C000FFFFFFADA45AACFFFFFFF6ADA3FFFFFF67
:1035D0009BADF6FFFFFF5AA3FEFFFFFF9BADFFFF72
:1035E000FFFFA4F6FFFFFFFFADFFFFFFFFFFF6FFAA
:1035F000FFFFFFFFFFFFF6A4A35BFFFFFFFE5B9B48
:10360000FFFFFFFF5B9BFFFFFFFFF6A4FFFFFFFF36
:10361000FFF6FFFFFFFFFFFFFFFFFFFFFFFFFFFFC3
:10362000FFFFFFAD5BF6F5F6FFFF9B5B5BFFFFFF68
:103630009BA3EDFFFFFF5A9BF6FFFFFFA3ADFFFF2C
:10364000FFFFA4FFFFFFFFFFADFEFFFFFFFFF6FF41
:10365000FFFFFFFFFFFFFFA4A39BFFFFFFFEAC5B8D
:10366000FFFFFFFFF5A3FFFFFFFFFFACFFFFFFFF23
:10367000FFF6FFFFFFFFFFFEFFFFFFFFFFFFFFFF64
:10368000FFFFFFAD5B5B52A4FFFF5BA3A4FFFFFF47
:10369000A3A4A4FFFFFF5BA3F6FFFFFF9BF5FFFFC3
:1036A000FFFFA3FEFFFFFFFFACFFFFFFFFFFF6FFE3
:1036B000FFFFFFFFFFFFFEF6A49BFFFFFFFFAD5BD9
:1036C000FFFFFFFFF6A4FFFFFFFFFFADFFFFFFFFC0
:1036D000FFF5FFFFFFFFFFF6FFFFFFFFFFFFFFFF0D
:1036E000FFFFFFAD9B5B5AACFFFFA3FFADFEFFFFEB
:1036F0005BACADFFFFFF529BF6FFFFFF5AADFFFF34
:10370000FFFFA3FEFFFFFFFFACFEFFFFFFFFF6FF83
:10371000FFFFFFFFFFFFFFED5B9BFFFFFFFFAD5BC9
:10372000FFFFFFFFF65BFFFFFFFFFFA4FFFFFFFFB1
:10373000FFF6FFFFFFFFFFFFFFFFFFFFFFFFFFFFA2
:10374000FFFFFFADA3F6F6ADFFFF5A9BA3FFFFFF00
:103750009B5BACFFFFFF529BF6FFFFFF5BEDFFFFA4
:10376000FFFFA4F6FFFFFFFFACFFFFFFFFFFF6FF29
:10377000FFFFFFFFFFFFFFF65B5AFFFFFFFFA4AD58
:10378000FFFFFFFFAD9BFFFFFFFFFFACFFFFFFFF52
:10379000FFF6FFFFFFFFFFFEFFFFFFFFFFFFFFFF43
:1037A000FFFFFFAD5B5A52ACFFFFFFA4A4FFFFFF7A
:1037B000A4A3EDFFFFFF529BF6FFFFFF5AADFFFFF3
:1037C000FFFF9BF6FFFFFFFFACFFFFFFFFFFF6FFD2
:1037D000FFFFFFFFFFFFFFF6A3EDFFFFFFFFAC9B27
:1037E000FFFFFFFFF6A3FFFFFFFFFFA4FFFFFFFFA9
:1037F000FFF6FFFFFFFFFFFEFFFFFFFFFFFFFFFFE3
:10380000FFFFFFADACA45BF6FFFFA3ADADFFFFFF75
:103810005BA3F6FFFFFF5AA3F6FFFFFF5AADFFFFC2
:10382000FFFFA3F6FFFFFFFFADFFFFFFFFFFF6FF68
:10383000FFFFFFFFFEFED0FEFEFEFEFED0FEFEFE00
:10384000FEFEFEFEFEFED0FED0FED0FEFEFEFEFE22
:10385000FEFEFEFED0FEFEFEFEFED0FEFEFEFEFEE4
:10386000FEFEFEFEFEFE90FEFEFEFEFEFEFEFEFEE6
:10387000FE909090FEFEFEFEFEFEFEFE909090906A
:1038800090FEFEFE90FEFEFEFEFE90FEFEFEFEFEA2
:1038900090FEFEFEFEFEFE37FEFEFEFE37FEFEFE44
:1038A000FE373FFEFEFE373F3F3F3F3F3F3FFEFEBE
:1038B0003F37FEFEFE3F37FEFEFEFE37FEFEFEFEFB
:1038C00037FEFEFEFEFEFEFEFEFEFEFEFEFEFEFEDF
:1038D000FEFEF6F6FEFEFEA4F6A4FEFEFEFEA4F636
:1038E000FEFEFEFEF6FEFEFEFEFEFEFEFEFEFEFE00
:1038F000FEFEFEFEFEFEFEFEFEFEFEFEF6FEFEFEF0
:10390000FEA4F6F6A4FEFEF6F6F6FEFEFEFEA4F615
:10391000FEFEFEFEFEFEFEFEFEF6FEFEFEFEFEFECF
:10392000FEFEFEFEFEFEFEFEFEFEFEFEF6FEFEA419
:10393000FEFEFEF6FEFEA4F6FEFEF6FEFEFEFEF621
:10394000FEFEFEFEFEA4FEFEFEFEFEFEFEFEF6FEF9
:10395000FEFEFEFEFEFEFEFEFEFEFEFEFEFEFEFE87
:10396000FEFEFEFEFEFEFEFEFEFEFF52FEFEFEFE22
:10397000FF01FEFEFEFEFEFFFEFEFEFEFEFEFEFE62
:10398000FEFEFEFEFEFEFEFEFEFEFEFEFEFEFEFE57
:10399000FEFEFEFEFEFEA6FEFEFEFEFE04FFFEFE98
:1039A000FEFEFFFFFEFEFEFEFEFEFEFEFEFEFEFE35
:1039B000FEFEFEFEFEFEFEFEFEFEFEFEFEFEFEFE27
:1039C000FEFEFEFEFFFFFEFEFEFE6605FEFEFEFFA5
:1039D000150EFEFEFEFEFFAFFEFEFEFEFEFEFEFE2E
:1039E000FEFEFEFEFEFEFEFEFEFEFEFEFEFEFEFEF7
:1039F000FFFEFEFEFEFE0FAFFEFEFEFE0717FEFE02
:103A0000FEFEAFF7FEFEFEFEFEFEFEFEFEFEFEFE2C
:103A1000FEFEFEFEFEFEFEFEFEFEFEFEFEFEFEFEC6
:103A2000FEFEFEFF5D5EFEFEFEAE0E06FEFEFEA686
:103A3000171FFEFEFEF71E27FEFEFEFEFFFFFEFE28
:103A4000FEFEFEFEFEFEFEFEFEFEFEFEFEFEFEFE96
:103A50001CADFFFEFEFE2715FFFEFEFE3717F7FE2C
:103A6000FEFE0E05F7FEFEFEF7FFFEFEFEFEFEFE6C
:103A7000FEFEFEFEFEFEFEFEFEFEFEFEFEFFEEF77C
:103A8000FEFEFF5D160EFEFEFF041705FEFEFF1490
:103A90002F0FFEFEFF042737FEFEFEFFAE5EFEFE8A
:103AA000FEFEFEFEFEFEFEFEFEFEF7FFFEFEFEFE3C
:103AB0000D15FFFEFEFE371F0DFFFEFE371F05FF33
:103AC000FEFE2F0705FFFEFE5FAFFFFEFEFEFEFEC1
:103AD000FEFEFEFEFEFEFEFFFFFEFEFEFF650DA5E6
:103AE000FEFF5C03170BFEFE5D05AEA4FEFEF604B2
:103AF000160BFEFF4B051704FEFFF7B76F04FEFE23
:103B0000FEFEFFFFFEFEFEFEFEFEAD66FFFEFEFEBB
:103B10000406A6FFFEFE050503F7FEFE060E0DFFDA
:103B2000FEFE0504035EFEFE0567AEAFFEFEFFFF70
:103B3000FEFEFEFEFEFEFFFFFFFFFEFEFF1505FF81
:103B4000FEFF1EAFB7FFFEFE045EFEF7FEFEF705AA
:103B5000AFFFFEFEAE0C0D66FEFFAE66165CFEFE0F
:103B6000FEFEFFF7FFFFFEFEFEFE6505F7FEFEFE12
:103B7000150EF7F7FEFE150DB6A7FEFE0D0D16FF8E
:103B8000FEFE15AEF7F6FFFE0C5EF75DF7FEF7FFE3
:103B9000FEFEFEFEFEFEFEFFFFFFFEFFFFF6B6FF8F
:103BA000FEFF65FFFFFEFEFEB6F7FEFEFEFEFF65B2
:103BB000FFFEFEFFFFB6F6FFFEFFFFAE5CFFFEFE60
:103BC000FEFFFFFFFEFFFFFFFEFEFF5C5CFFFEFE51
:103BD000FFF6FFFFFFFEF6F7F6FFFFFEFFAEAEAE0D
:103BE000FFFEAEF7FFFFFFFFF6FFFFFFF7FFFFFF50
:103BF000FEFEFFFFFEFEFE0707FEFEFEFE07FEFEC8
:103C0000FE07FEFE070707FEFE0707070707070771
:103C100007070707070707FE0707FEFEFEFE07FE6A
:103C2000FEFEFEFEFEFEFE1707FEFEFEFE07FEFE89
:103C3000FE17FEFE070717FEFE0707070707070721
:103C400007070707070707FE0707FEFEFEFE07FE3A
:103C5000FEFEFEFEFEFEFE1F17FEFEFEFE17FEFE31
:103C6000FE1FFEFE07071FFEFE07070717070707D1
:103C700007070707070707FE0707FEFEFEFE07FE0A
:103C8000FEFEFEFEFEFEFE2F1FFEFEFEFE1FFEFEE1
:103C9000FE2FFEFE07072FFEFE0707071F17070769
:103CA00007071707070707FE0707FEFEFEFE07FECA
:103CB000FEFEFEFEFEFEFE1F2FFEFEFEFE2FFEFEA1
:103CC000FE1FFEFE17071FFEFE1707072F1F170711
:103CD00007071F17070707FE1707FEFEFEFE07FE72
:103CE000FEFEFEFEFEFEFE171FFEFEFEFE1FFEFE99
:103CF000FE17FEFE1F1717FEFE1F17071F2F1F17A9
:103D000007072F1F170707FE1F17FEFEFEFE17FEF1
:103D1000FEFEFEFEFEFEFE0717FEFEFEFE17FEFE88
:103D2000FE07FEFE2F1F07FEFE2F1F17171F2F1F58
:103D300017071F2F1F1707FE2F1FFEFEFEFE1FFE79
:103D4000FEFEFEFEFEFEFE0707FEFEFEFE07FEFE78
:103D5000FE07FEFE1F2F07FEFE1F2F1F07171F2F38
:103D60001F17171F2F1F17FE1F2FFEFEFEFE2FFE11
:103D7000FEFEFEFEFEFEFE0707FEFEFEFE07FEFE48
:103D8000FE07FEFE171F07FEFE171F2F0707171F50
:103D90002F1F07171F2F1FFE171FFEFEFEFE1FFE01
:103DA000FEFEFEFEFEFEFE0707FEFEFEFE07FEFE18
:103DB000FE07FEFE071707FEFE07171F0707071778
:103DC0001F2F0707171F2FFE0717FEFEFEFE17FE09
:103DD000FEFEFEFEFEFEFE0707FEFEFEFE07FEFEE8
:103DE000FE07FEFE070707FEFE0707170707070780
:103DF000171F070707171FFE0707FEFEFEFE07FE39
:103E0000FEFEFEFEFEFEFEFEFEFEFEFEFEFEFEFED2
:103E1000FEFEFEFEFEFEFEFE0707FEFEFEFE07079E
:103E2000FEFEFEFEFEFEFEFEFEFEFEFEFEFEFEFEB2
:103E3000FEFEFEFEFEFEFEFEFEFEFEFEFEFEFEFEA2
:103E4000FEFE1717FEFEFE17FEFE17FEFE17FEFE15
:103E500017FEFEFE1717FEFEFEFEFEFEFEFEFEFE37
:103E6000FEFEFEFEFEFEFEFEFEFEFEFE2727FEFE20
:103E7000FE27FEFE27FE27FEFEFEFE2727FEFEFE95
:103E8000FE27FE27FEFE27FEFEFE2727FEFEFEFE85
:103E9000FEFEFEFEFEFE2F2FFEFEFE2FFEFE2FFE7E
:103EA0002FFEFEFEFE2FFEFEFEFEFEFEFEFEFEFED0
:103EB000FEFE2FFEFEFEFE2FFE2FFEFE2FFEFEFE5E
:103EC0002F2FFEFEFE7FFEFE7FFE7FFEFEFEFE7FAC
:103ED000FEFEFEFEFEFEFEFEFEFEFEFEFEFEFEFE02
:103EE000FEFEFEFEFEFEFEFE7FFEFEFEFE7FFE7F6F
:103EF000FEFE7FFEBFFEFEFEFEBFFEFEFEFEFEFEDF
:103F0000FEFEFEFEFEFEFEFEFEFEFEFEFEFEFEFED1
:103F1000FEFEFEFEFEFEFEFEFEFEFEFEFEFEBFFE00
:103F2000FEFEFEBFFEFEFEFEFEFEFEFEFEFEFEFEF0
:103F3000FEFEFEFEFEFEFEFEFEFEFEFEFEFEFEFEA1
:103F4000FEFEFEFEFEFEFEFEFEFEFEFEFEFEFEFE91
:103F5000FEFEFEFEFEFEFEFEFEFEFE30FEFEFEFE4F
:103F6000FE30FEFEFEFEFE30FEFEFEFEFE30FEFEDB
:103F7000FEFEFE30FEFEFEFEFE30FEFEFEFEFEFEFD
:103F8000FEFEFEFEFEFEFEFEFEFEFE303FFEFEFEDE
:103F9000FE303FFEFEFEFE303FFEFEFEFE303FFEE8
:103FA000FEFEFE303FFEFEFEFE303FFEFEFEFEFE4B
:103FB000FEFEFEFEFEFEFEFEFEFEFE303F1FFEFE8D
:103FC000FE303F1FFEFEFE303F1FFEFEFE303F1F55
:103FD000FEFEFE303F1FFEFEFE303F1FFEFEFEFED9
:103FE000FEFEFEFEFEFEFEFEFEFEFE303F1F07FE54
:103FF000FE303F1F07FEFE303F1F07FEFE303F1F13
:1040000007FEFE303F1F07FEFE303F1F07FEFEFE8D
:10401000FEFEFEFEFEFEFEFEFEFEFE07070303FEA4
:10402000FE07070303FEFE07070303FEFE03030765
:1040300007FEFE03030707FEFE03030707FEFEFE5F
:10404000FEFEFEFEFEFEFEFEFEFEFE03030707FE74
:10405000FE03030707FEFE03030707FEFE07070331
:1040600003FEFE07070303FEFE07070303FEFEFE33
:10407000FEFEFEFEE8E8E5E8E8E8DEE2E2E8E2E28D
:10408000DBE893800431088934171EACF144E2A6C2
:10409000341B11A61431C8BC411EA2EB44EB93346F
:1040A000241B8F0E54C296502AA2DB50F1A911177F
:1040B0008C270E3799F8319CEB50E59F1147C2C20F
:1040C0003A27860B2E892A14EB937A89B9631B80D1
:1040D0003434CC9067C5BC2A249F0B1BF5AF37EB5B
:1040E000895024AFCF5D018C08478C1424F2A63D83
:1040F0000BC8F22ADBDF1424BCF241EBB6113AC83C
:10410000CF2BFEC8FB41C8BF2E1B14A6F84AD8B956
:10411000343A80FB4A1EB6B9571B89F254F59C1BF2
:104120002E2E804A2E14961837E5A92B27FECFD8BD
:1041300054CCC211509FD82E3199441160800B3E4F
:10414000058063F283372EB9BF60E2B22127B6E55E
:104150002B11991437800154DFA344DFA32B34BC07
:10416000B9609FEF2B0B9F34EF8360DF9F3141C21B
:10417000B967E5AF210E805118DF867F80FE2E24BF
:10418000801B37E2935A11BFBF60DCCFEB44BCF217
:10419000FE37F2C2143E960E1E31C5CC3E1B990E60
:1041A000214A86B94708992E0241B9E22B21F8909D
:1041B000641502993727BCD25708EB935D1518890F
:1041C0003A08E5C53E080EAF2B18CFBC5AFE96053F
:1041D00070A6A94D3190E241F5961E4AB3BC5A082B
:1041E0008D1151DF866ACCA93ECFC244EBC9FB4199
:1041F000803124EB9C64BCBC372BA9D85A93EF4781
:10420000A3E23BFE9C31F299311EDF9C1B11B315DA
:1042100015E8BC4402BCF54ECCB9244A89E23461AD
:10422000A3BF3E3789F83E1EE5A3541B08903131E9
:10423000D2B361E57083EC372880312B2402A62E9F
:104240001524AC082405934E022B8051111B9611A6
:104250001E2BE8A35DFB189C4AFBCFD53EE2C60BA4
:104260003BAFEF1B18A30541DFA62B24D5AF57FFAB
:10427000A01B15807FF5803B34C6A66A9CE21E31E8
:104280008D0B2883243E803E18901834E28A679D67
:10429000EC1B15A90B25801E44D2BC1E34A6EF25AD
:1042A00005963E28ACD95AE5A36D0B18BCD941122E
:1042B000930E283793FB1E51B9B0510E12805DF852
:1042C00064A3F215250EA33BF531CCDC1E0E6D80E8
:1042D000281E5A800E2831CFC9280E34864131213C
:1042E000961815FF9647052E900B38E29D4A1B083D
:1042F0008A540EC3B95A99FF0825A31221F5AC447C
:10430000A9D270D59D1B3883FF4B801E418AE55191
:10431000FB8005088D67BFCF2515C3D644A9FF1BB9
:10432000F8C63BBFAC6DBC994E28A3D661F8803B64
:104330002EA9EF380290212528ACDC3E08B60E0BE2
:104340003493121534C3F85AC67F802BF241C9CC7E
:104350003BFF1E8D4B0531ECA631084EBCB93B1E10
:104360001B803412388D1231EC4E8047E251A3F598
:104370000E3ED6BC2B3B80F82E41B68077F2B9E9D1
:1043800041FCA947B6A96412A3D264029D050B8A19
:1043900067D6B31244B0CF4B9AFF22A6FC349305E4
:1043A0002E871838D2B33EF88051CFC331189D2ED6
:1043B0005A8DEF38B3D24EF29D1EF8B91E3BEF8DE9
:1043C0004E18801B511E8AF257E99351F822A91802
:1043D000FC38C0DC3EEC61900831EF31AD41DF2E9E
:1043E000D6D648FC4BA6121B1218259A2B151B9DDE
:1043F00031051231A3F83B083B80221844F880486D
:1044000048A3C62E4BDC873E2E18801B57A9C92512
:104410002EBCC94EDCC0084BC0DC54A9B36D90D98A
:10442000312B802E0B901B2E8031F8C6FF31DC9D86
:104430007FB98A4EE2DF289D08358DF5519A022515
:104440008A2B1802A348E2B92B22BCD64EECCCD959
:104450007FC69A54359DD674DC9D48022B8A48FC51
:104460003BADE238153E87F2541808A90F25221EED
:1044700093181B2E31ADB974E638D9B32831221BFD
:10448000A031FF353B8008312215804B1E25840C5E
:10449000222BD3C02EF922933EFFDCBC51CFDFE6A6
:1044A00038CFE20518C0FC18FCA061B3B64BD68427
:1044B0007AA6D62E448022ECB93218A0FF38804B61
:1044C000A0F20F2B9A1B12A32205B03205A02ED00A
:1044D000D65EADC04515C0EC3E803E0C28D9CC451B
:1044E000B0F232FC159A5B0F35803B454E80FF5E83
:1044F000F248AA02351FC6E625154E18841F321F42
:1045000035D9C648F557C9C03E0C3B2E84086EDC31
:104510003BFFA0442BFC4E9308442B9DE954C664FA
:10452000AAEC320C804EFC2EC0EF44ECAA154412CB
:10453000A0FC35933B15CCCC57B6CC223E97022835
:10454000C01205A3221BAA25ADEC2508D302B0DFBB
:104550006A90222E0C9D4B97EF5ED69D54E3D0259A
:10456000CCE33EC6BD3818C30832DCC63E0CD6C00C
:104570005105BD150845A30F32FFF2B974FF2E9DFA
:1045800035D93E22874E0F0232B3121212352ED683
:10459000CC380C4B28802B2B2B2EC0DC2B1848FF43
:1045A000B3EF321854E2843B3BF941C3D61B3EDCE7
:1045B000E20F0F18B0053EDFA34E22D6C03B15AD6B
:1045C000E257F99D220FA31F05C30C08D6EF1FADBC
:1045D000EF48A0EC0F904BD3D025D3D632D0B63EC7
:1045E000E9A351B6E628C9CC459D052802B3F615C6
:1045F000B035E99A323BBDCC45A3FF251597123E55
:10460000FF9A480905DFC3352B059A3B0F38D0C602
:10461000450F0C1BC90FF63525F697451B0C3EC000
:10462000C6282B38FFD0D638092522ECD312F254F5
:104630000C12C9FC151835029A381228E6C0410F31
:104640000C904B121F9A2E1228C6E33EFFC3022B7A
:10465000E9C64BC6B93E32B9E91BBD0528BD15FCFC
:10466000B91B22B028C0F228AD0F1FCCF628AAFF34
:1046700038B915F6B9320CC90209BD3EDCC054E6A2
:104680009A4B25A30C54810C2EF2CC58E3FCC31298
:1046900025FCAA410F259A1548020FAD320CF9549A
:1046A000ECAA3B220F18D9FC1C09380CE6D338FFC2
:1046B0004522D3AA4B1B28051BD6D34525FC25F242
:1046C000B04B151B0CE3DC281F15FCCC32F625D3B0
:1046D000E9283EEFC60228FFD01BF9FCD948EFC0FD
:1046E0001238D6D048AD092E029A4B12844515AA2D
:1046F00038ADEC61872E18B0221B8061C3EF329772
:10470000124EA6E635E9D918C31522A31218C61F02
:10471000FF9A4828C6B64E22B6E648F6C60525D00A
:10472000EC1F1FFCB9321C0FD00225E93BE6B03B61
:104730002E092EEFB3281832DC61E6C932F618458F
:104740000CD6DF3BFC2E152515A041EC382812C9EC
:10475000E3353EE61FFCDC38FC3505AA222538BDD2
:10476000CC38122EB90232FC8A1B58BDD054E9D085
:10477000EF1508CC08F2B948C3BD58C6C628F9BD24
:1047800002D925BDC348ECB312D6F6EFC33ECCB078
:1047900032B0092EAD0C1C9A0C2F8A48C6D628F9C7
:1047A000A702259A2B35C0BA3BFFB02825F2DFD0EF
:1047B0003E22CDD045C654D9D32FF23EBDE35BF99E
:1047C000F23B5187F63835FC1838942812320C2504
:1047D000FC61DCC041FC41152E2E90410C122B3E99
:1047E00035C6D05825FC1BE6EF452225D9F21B2BF8
:1047F00012C905252EE6E9FC45F2B658BDD954FF8D
:10480000A31241C6F63EADC654A315E9B635F6A3CC
:1048100067D6AD05CC2BEFA025C6DC12DCE61CA7C5
:1048200012BDE62FC0C312C9FF12C6F2E6BD181FA3
:10483000971F2BE6D312DFF6F9DF25D0C938189D74
:10484000D667D605D3F6FF48F6E3AD183EE6180F57
:10485000BA22FC152FEF3525A3F22509152825329C
:104860009DEC282F051F25F232B3FF3B0CF2510CB3
:10487000FC0CD318221818B6152F1F09D9DC2FF9F4
:1048800045D6C64B0C8048150FD0EC2FE6D02B0533
:10489000813E41803B228D32F6803EC6FF18814228
:1048A000EFBD22AA2B22802FE9C60FE3FFD9BA5B06
:1048B000ADE30C873809975BD6B342EF8D45CDE663
:1048C0002215BDFC1FD9B63E22BDCD1C3BEFA31C5B
:1048D000181809B3FC42251F9ADC450C1838E6AAC3
:1048E0001235150C32EF1FDCE62505094505220CB3
:1048F000D9D03B15FC0238122522F6AD1F2528120F
:104900000F12E09D28182209AAE92F2225C6D309F3
:104910004E058A152FC0FF0CE9D6DC4EE0C625F601
:104920009D122FC6C328AD12E9B61FDCD61F8045E5
:10493000F3B042C9E6158009A0F94280060C9D55E6
:10494000BDEC0C8D1C12C91FB7E648C6C94BECADB7
:104950003BD9C0350CE309FC09B31245EFBD191270
:104960001F25E9B342153802ADFC3BFF220955D3A0
:10497000B71C2C122F1535FC0CC6F63B150F28F969
:104980001C15352F15CDD32F0F02351828FCD9094A
:10499000121C061F22E3F3090C2F15E0D33B18C0AD
:1049A000EC252FEFAA2F2FDCE03EF9A31C229A352D
:1049B000F6AA350FA72FEFCD35F6B028C0FC15D0DD
:1049C0000FD9D935B319DCD32BC0060CA02FBD0FDE
:1049D0001FAD32BD9A45A7F622C0F9ECEF1C06D3F5
:1049E000D03BF9BA2219C0D04EFCC315FF1C06B744
:1049F0003FEF22429DE94BF32FF31F0CD3E6450214
:104A0000222C2FF338C3C6421FF92519193215F984
:104A1000482FD3F338EC2B1922062B0C45FFCD1F62
:104A20002F0C1C1F06E9F902424EE9B025090C457E
:104A3000A0183825A7F65EEFB60CD3D042EFFCD90C
:104A400009E9E306945EC002D6B61CE9D909AAFCBE
:104A500009BD28B0EFD3BD2CB01CC0CD22B302CD10
:104A6000F919841525A4FFE0C0289D15F31C06BA8A
:104A7000F3EF2528E0BD42020CA028193BE3AA2F42
:104A800015061CE3E35BF9F91C152FD9DD3202484A
:104A900009FC4B0CFC3F06BA0F4E1FF625EF151C08
:104AA0003BEC153E1FFF1FBAFC45DC0C2528E31C20
:104AB000EFE9FF1525C038F6A74ED01CE6E0192215
:104AC000FFB6EC0915C309F6E3020FE6CDF9ECD306
:104AD0004EBAECEFBD4BC3E0E6C01212A73887090F
:104AE000ECD345B025E306F6D04884E648804ED99D
:104AF0000F12AD22B31C2CB32815B3F91CFFCA3B0F
:104B0000D9F00219CDE64E0225A425FF1C358025DB
:104B1000F9E33F02ADE6123F0CE64BFCE9D3E92591
:104B2000F928E90CFF0C19022CF30FFC28F622E0FF
:104B30009725DD28220202FF19EC451C15F68A3262
:104B4000DD3522F925CDD30C023245941C0206C076
:104B50002232E912D32FE3EC062CBA1F15BD1F2811
:104B6000A438E0CA5EAA22E3DD38A7221FAD25C61D
:104B70001CCD091FBD388D6BC00F09D019BA22BAE0
:104B8000320CAA2CD6D048B7FF3FE6CD1C22AA286B
:104B90000FF0AD4206D6250906DDEC35F0220CC635
:104BA00012FF1C1235280FA4F055E93512251528DF
:104BB000EC251F190F2F021902AA3512FF3525DD2A
:104BC0003815FC4BE3350CFF2228FC28ECD9F609FC
:104BD000121512FF25CDD935FC2FD9D0F91928A7E8
:104BE000DC1CEFC0EC3BBDF30919C309F9971FC3E7
:104BF000E90FAA1CD6E6EC9D19CD060F875E9AF048
:104C0000E6DD228AFFCA3FA703F99D588042CADD2C
:104C100019BA55B7C30FBA12FFCAF33FCDC36EE03E
:104C2000F0030616CD1F28ECCD1C0C163828C6FC48
:104C3000281619352809F6BA2842122225FC322FE7
:104C40000C2C192C0628154E020645192512EFE3E7
:104C5000420C0C252F2FFC252F0F152F062F1F1F61
:104C6000D3EF06323BF62CC315FF1F28B3F935E905
:104C7000BA2F190CC61912BA06E9E01902AD4BCDCC
:104C8000D32CC02CB7F9198A2CE0D9CD0215A73B3B
:104C9000D3B0D012D6C652A7ECCDE92FCAE9EC09A1
:104CA000D3AD4EE0D006AA3FE3B72C12F3B742B320
:104CB0001FFF0FE9B0350C1FE0D91CF935FC2CD9CA
:104CC000E025151C0C250C1C09280F22C3F9250F03
:104CD00025061C191F1525062515190C220F191F4D
:104CE0001C120C25190F1C19120C0F1F1C0F091276
:104CF0001C121F09AD280C190225AA190F25C3E3A0
:104D00002506B01C0FAA1C1CE0D31F9D4BD9CD1546
:104D1000BA0C1FA438AA06E6CD25B0159A02BA2C03
:104D2000A719D0EC09AD3B9A35AD09F3CA22A428E6
:104D3000F9BD25BDFF1FAA1506B71C32DDCD1C2508
:104D4000BDEC2C12D9CA38032509C0FF2F0328FF58
:104D500038FF22D6D925151C0F151F121519190C4D
:104D600022191F0C1C0F1F19151F191925151C15A9
:104D7000221C220F2215250C25151F1C1F0F25098B
:104D8000250935ECD93519152FB3F92222E6BA3B9E
:104D90000615B02FECBD28F3BA35E3C928A728C9FA
:104DA000E638A702AD35AD0CE6D61CA73B9735AD6E
:104DB00002F6C622A035BDE6B7E9C6EF35A025CA82
:104DC000F302B03BE0D02CE3C33FCDE02506CDF6A7
:104DD00035E6CD1C0F1F1FC0F3280C1F0C250CB08F
:104DE000221512151C191C121219280C15221F1F2E
:104DF000191922121F1F1C191F151F15221C121210
:104E00001F1219190C1F1509191512121F0F19124B
:104E100022FC28E9C32B0F121CBA0F1C15E0CD325F
:104E20000CC91F1FA0220CB00F1CAD2FB3F93BA75C
:104E30000FE3E00FBAEFCD25A04E804EA022D3D3D2
:104E4000D90FE0CD1FAA3BA01CD6E9CAF928AD2C8A
:104E5000AD0206B035D3023FBAFC1215B70C1219D9
:104E6000D3DD2C0625C0FC1C0F220C2202C01C1F07
:104E7000151F15191215280C2C0C191C12220F15B0
:104E800019280619190F220F121C121C090F1919C3
:104E900006191212090F190C0C0F1FFC150C0F1517
:104EA0000F0C12120C120C22FF32FF1FF6C01F153E
:104EB000D6D648A00625BAEC35B00FD6D622A077B4
:104EC000A028C6F90CB338A4FCBA329D42A402ADA6
:104ED00045AA22CD02FCC9F3E309B05EBAF612B0CE
:104EE00022C60225BDFF2FAD1F15BD1C19F9C33801
:104EF0000628DCE0061F1522F6BD32062CFF22191B
:104F00001C0619221212151215151F061F0C22124B
:104F1000151519121C121F1212181518181C0C182E
:104F2000151512151C12181512150C1F180C0C1C37
:104F300012180F150C150F1F12180C12150FB31C99
:104F40000CF2C045C6E30CBA2FF6BD329D38B6FC54
:104F5000B62BB009ECD912C3E6D60FC6C39D359463
:104F6000489718AA4287489A19D9E319AA35B31560
:104F7000E3D042BAFC19D9E042AD0C0928D3E025B0
:104F800015FFBD25191C121525C6EC250F1F0C1F7A
:104F9000121912191C0F1F0F180C18150F121812C6
:104FA00015151C0C150F180F18151C0C1C180C12BD
:104FB000180C0F0C12091509150C120C0F09150508
:104FC0000C0C0C0C120C0F050F09120512050F0228
:104FD000120C1209180918091F091F0C18AA35BD4F
:104FE00002C02FBDF9BD32AA22D3E6D3E6C925A35C
:104FF0002BB3EFB025A70CD3D0D01CDCC342A7F94C
:10500000F3B335D3CD35E0D335C9E62218FCB3224E
:10501000150C1CBDE91C0222F322FF1502120F150C
:10502000091F0C2212151C28121F151C280C281FE2
:1050300012280C1F0F350C0F1F0F18180FF6151222
:10504000051C021FFC1209FF25EF2FF91815FC158E
:105050000C09180F0C1CF93EF928FF1C0F05151C34
:10506000EF1F18090CD3FCDCFC2EAD18A03BB022BE
:10507000D6E3D309DFE6D005E3CCE6F6E3C0F2C918
:10508000E60FC3DCE909B3429738B015F2C0359A90
:1050900038FFD02212B63B0CD01525D9F2250C1CB6
:1050A00009C6151FFF2B091C0F15151FDCD92F056D
:1050B0001F0F121518181218151815150F1518FFAF
:1050C0001209120F0C050F0F09020C050C0C050C30
:1050D0000F0212050909020209050C0C05020C0554
:1050E000FF0205FF09020502050209FF0CFC05028B
:1050F00005050502050209FF0C020F0212FC150549
:10510000150512021F05220225022EE6DFCCEFFC58
:10511000CCDCEC02C3E3E30CB0389445A31FD6E625
:105120000FB335E9D3221FD0EC2818F2C92F091F7D
:105130000FCCF22FF9180C1F0C1C0C1C09180C1C9E
:1051400009180918091B09180F151218091BFF1B4C
:105150000F150C120F0C0F120C1208080C080C0C77
:1051600005080C0F0512FC12020FFF08FF0C080CBB
:10517000FC0F0802FC0F0508F90CFF0F0502080CD4
:10518000050C0505FF0C0C0C050F020F080F0F1581
:1051900012121505C3EFC3E9C3E3FCDCC905CCFF5C
:1051A000E6D9D0FFECD0D3F9F2C3289D3BA322056A
:1051B000C60C1FAD32F9C30C2BD6E3280F121BB956
:1051C00005180C120F150F1512121215121B0F15C0
:1051D00012121812150F12150F120C0F0F121212B5
:1051E000180C0C0C0F08080F0C0C050C0C0C080804
:1051F0000C050805FF0C0C080805FC080202FF025C
:10520000FC02FFFC0202FFFF05FF05FF020505058A
:10521000020502050C080C08080F0C0F080C0F12F1
:1052200012120F0C150F18EFCFE2D6D6FFE2C9F518
:10523000C6F2F5D3DFECFFC6E3DF028D45D3DC1504
:10524000B91FFCC91B1BDCDF280505B62BFF1F0C93
:10525000180C18B322081812180C1B0F150F180F72
:105260001212150F150F120F120F0F0C0F0F0C0C3F
:105270000C080C080C080C020C080C0208020502B1
:10528000080208FFFF0502020202FFFCFFF902FF0D
:10529000FFF9FFFCFCFCFFFC02F9FC0202FCFFFF33
:1052A000FFFC02FC02FFFF0205FC020502050202F0
:1052B00008050508080808080F0C0C0F120F08183D
:1052C0000C22ECD9E2E615B03B9741AD1BDFDF12B3
:1052D000B9221BDCDF2E05C6E2181215B01F0F180D
:1052E0000F120F15121515120F180F151212151592
:1052F0000C12120F150F12120C0F12080F0F0C0CBC
:10530000050F0F0C08080C08050C0C050505050811
:1053100005020505050502050205FC05FF02F9FF6A
:10532000FC02F9FFFCFCFCFFFFFFFCFCFC02F902A5
:10533000F50BFCFF02FFFF05020205080208050B42
:10534000080F02150215081808150B1B02D3DFE61B
:10535000D3EFC61EC305ECD6DFEC02B94EB005F59F
:10536000D31222CCF2220CB91F0C150C1BC0FF1853
:105370000C0F0C15081508120F12120C0F0F120F3C
:10538000150B0B120F0B0F120B120F050F0B0B0847
:105390000F0508080208080208050BFC0502FF02B9
:1053A00002FF02FFFFFF02FCFC02FCFCF8FCF8FC21
:1053B000F8FCF8F8FCF5F5F8F5F5FFF9FCFCFCF560
:1053C00002F9FCFFFFF2FFF505F905FC02FF0202FE
:1053D0000505080208020F020B020F081502150549
:1053E00018021ECCE905C3E9DC15B031A925FFCCB4
:1053F0000815B322051EBC0215150B25D6DF2205A4
:105400002205180B0B08150F0F0F0B0F0F0B1215A2
:105410000F0F0F0F0F080F05080F0B0F0B050B0BCE
:10542000050B05080202020208FFFC05FC02F8FC5D
:10543000FFF8FFF5F5F8F202F5F8FCFCF502F5FCD3
:10544000FCFCF8F8F5F8FCFCF8F5F502F8FCF5FFC3
:10545000FFF8FCFCFCFFF8FFFF020205FC02FC0564
:1054600005FF080B0808080F080B050F0B150F1296
:10547000081208120812C01ED3E231BCF8F5CC386D
:10548000CCEC180FC60512180F18CFEC2505120228
:10549000150F120F150B1205150F15120F120B1207
:1054A00012081208080B0F0208FC08080BFF080876
:1054B000050B08FF050202FFFF050202FCFFFCFFCF
:1054C00005FFFFFFFCFFFFF8FCFCFCF8F8FFF8FC11
:1054D000FCF5FCF5FCF5FCF5F8F8FCFC02F8020222
:1054E000FCF8FFF8FFF5FFFFFCFCFCFFFFFF0202EA
:1054F0000505FFFF05080B08080B080B0805080B3E
:105500000808150815FFCCF2CC25D2E908CC18EC18
:10551000D90BF508D308050BFF05DFFF0FF81505BC
:10552000150F12051208150B120F0B150F05120897
:105530001212120B0F1505020F050F0508FF0505C6
:1055400005080505050505080202080808050805FF
:105550000F050F0B080B0B05050205FCFCFFFC08F3
:10556000D2CCD9CCD9C9D2C6CCC3C9C3CFC0CFB68F
:10557000DFE9DFDFB902C628B61ED9E928C9FF1B5B
:1055800008120F180B1812121518150F120F120F00
:105590000F0F0F120B120F0F080B0F0B0F0F0B0833
:1055A0000B0B080F0805050208FF0FC308180515A7
:1055B0000B150B0F0F0F0B0F0B0F0B12080B0B0F15
:1055C000080F080B0B050B0B0F0B0B08080B0F0B31
:1055D0000B0F080B080B080F0B0F0F1212150B15F2
:1055E0000812EFB3C9BCCCB9E905FF0BFF02050BEC
:1055F0000205080B080B08080F0B0F0B0B120B15FD
:105600000F120B0F0B0F12120B121805180821DFC7
:10561000E9250B180E150E120B1508180B080B05B3
:105620000512080B0B0BFF050B0E05050BFB020B00
:105630000508050B0508FF0BF2CC210E1808121205
:105640000E050B08120E0E0B08150B0E050B0202B1
:105650000B0B0512020E0E120E080B12FF18080893
:10566000120B12F805FFFF0B0505020508121512B3
:105670001B081EE2BCC9C6E2BFE80202020208081B
:1056800008120805080B050E0B0B0E150B0E0E0E5F
:105690000E081805080B0E12080E0E0E0E15121528
:1056A0001B15150B1E08020E1512081218121B05E9
:1056B000150B0E0B080E08150B08050E020505024A
:1056C0000E0BFB050811D50B0B0B020B1B0E081163
:1056D000051108080B0B08080B0505080B02110B38
:1056E0000B0B02020808050B02020208080B08084F
:1056F0000B0E0B0B080B080B0B0E050E080E0B11F7
:105700000B0E0818F8C2CFCCC9E511FB05FE080244
:105710000B0808050B080B0B0B080B0B0E0B0B0BE8
:105720000E0E0E0B0E0E0B0E0B0B110E110E0E0BA2
:105730000E0E0E110E0E0E110B0B0E0E0E0B0B0E8F
:105740000B0B0E0B080808080B08080808050505D0
:10575000050205080E0B0B0B0E0E0E0B0E0B0B0BA2
:105760000B0B0B0B0B080B0E08080B08080B08059E
:10577000080808080808080B0808080808050508AC
:105780000505080B0808080B080B080E08110E0E7B
:10579000080E0511EFC5D2D2C9E80EFB0B050B02AE
:1057A0000B050E0508050505080508050B0B0E0B76
:1057B0000B0B0B0B080B0E0B0B0B0E0B0B0E0E0E2D
:1057C0000E0B0E0B0B080E0E0B0E0E0E0B080B0B1A
:1057D000080B0808080B0B08050808050505050552
:1057E000FECC140E0E0E080B0E08080E0B080B0B49
:1057F000080B08080B080B05050508050505050538
:105800000505050801050805050808080805080B31
:1058100008080108080808080B0B080B080B0B0EFA
:105820000B0B0B0E0B11FEC5E20E05080805050853
:1058300008080B080B0808080B08080B080B0B0ED0
:105840000E0B0B0E0B080B0B0B0E0B0B0B0B0B0BA2
:105850000B0B0B0E0B080B0B0B0B0B0B0B0B08089E
:105860000B0E08080B080808080B040404040804BD
:105870000B0B0B080B080B0B0B0B0B0B080B0B0884
:10588000080B0804040408080404040804040804B9
:1058900008040104040104040404040404040404CA
:1058A0000804040408080808080B0B04080B08087F
:1058B000080B0B0E0BDED8DB0108040401080408FA
:1058C00004040804040804080808080B0B0B0B0B5D
:1058D0000B0B0B0B0B080B0E0B0B0E0E0B0B0B0B12
:1058E0000E0B0B0B080B0B0B0B0B0B0B08080B0811
:1058F000080B080B0404080408080408080BF8DE69
:1059000011080E080B080B040B0808080808080803
:10591000080808080808040B080808080808080808
:10592000040104040404040408040404080404082E
:10593000080808040808080408080B070704070BF0
:10594000070B0B070BE8D50104010404040704044A
:105950000707040707070B0B0B070707040B0B0BC5
:105960000B0B0E0B0B0B0B0B0B0B0B0B0B070B078C
:10597000070B0B0B0B070B07070B0B0707070B0797
:105980000B070B0407070B04070407010BE8F814C7
:10599000070E070B040E070B07070404040707078D
:1059A000040B0404040704070404040407070404A4
:1059B0000707040407040404040404040407070498
:1059C0000407040407070707070707070B0B070B64
:1059D000070B070BF8DBF8070407070707070404A2
:1059E0000707070707070707070707070707070747
:1059F0000707070B07070B07070B0707070707072B
:105A00000B0B0B070B0707070B0707070707070415
:105A1000070707040707040704040404070A0A0A1F
:105A20000A07070707070707070707070707070703
:105A30000407040407040102010201020203020533
:105A400004050302FF01010401030002F8FAC8CFB4
:105A5000FAFB0A090F0C0F0B111017182427595DB8
:105A60002F26160D0B030401F7F2E6DFB18AAEBD57
:105A7000D5E9F410413A1DF6F1E8E7ECEDF0EFF06E
:105A8000EEE9E1DBE1E0E0E3E6E6EBEAF0F6FBFA83
:105A900001FFF4F7F0ECF4FF060A0F0F1214161BC7
:105AA000211F1C2B262428282923211529262124BF
:105AB00030292522261A1F1712053E2B2A3A2522A5
:105AC0001213151C08120B080400F8F7FAFCF9F879
:105AD000FDFEF9FAFAFAFBFC010C04FEFBF6F3E218
:105AE000ED04F0020C03F8E1D3CEC8C3C3CAD4C995
:105AF000BFBAACA9A1B5BFBAC5D2D7CABBAB9FA527
:105B0000A2A7ABC7CBC5ABA1A09794969EB3ABA3FE
:105B1000A9A29897979698A7A2A2A4A5A8ADABB65C
:105B2000BAC1C9D0D8D7D8D5E0E7EDEFECF5F0F69B
:105B3000F9F303FDFF090F130B15192A363B313515
:105B4000443C34333133363A0C2C46265C474725E7
:105B50003451505B5553594D4E4C4B4A47505C5F46
:105B60005B54524C4F5C5251504B536158454C4B17
:105B700046514B4538473E433329241C1317151D06
:105B80001824FF04DDF325EE00280905C4E20F20E8
:105B900023F233391E0B120C02121C111C1DF021B2
:105BA0003D39453A291D3128354B41382D302625C0
:105BB0002F1D1F283A101B2B110A170E132C2A1702
:105BC000171C1C1C1F110A0702FBFF08F9FCEBEC59
:105BD000E7E6F3E0D1BABFBCBDE0D3CCB698A0AE47
:105BE000AD94A3A4A4AFBDD5E1EED3C0CEF5EBC276
:105BF000E3E5CEBDB9CBCAC7C9BFBCC4BDBAC1B647
:105C0000E70DE6F2E1D0E6E0D6CEC6DAB9E13E3401
:105C1000DCEA114F550A291E0D0411FDDDE4FD27B4
:105C200010102D1D121EF5E8F62237284C51334F67
:105C30001C0C4852461F5A536D68234F3741686801
:105C40004E64716E717167726F71624345482A10BC
:105C50002F2422221308E8FA09E7EB04102F6174BD
:105C600033FA1ED00107081D40763E4BFEDB1603BB
:105C7000EDD6E923463D2A351F19EA334D2B75141D
:105C800003EE0E01F00F15F4BA8DAB046F6601E759
:105C900012FCD9FBFAE4A58F90AAD1C0E61E171C0E
:105CA000590FECDFFA1B08313D37362F2A3754578E
:105CB000604247615C2C3C5A706B534E6B4F45649D
:105CC000615C68565147240924484D5A4F554F513D
:105CD0004D3914F1F5FC25332D314A291F343E3B53
:105CE0002E16E4CDB7C5FADD0519191AE7E8E2F377
:105CF000EFDEF3F8D7A18E908D8E8D8E8E8F8E90E5
:105D00008F90919191919394949496949898A2EBFA
:105D1000B1949C98969CC8D30D092D4D28294833E1
:105D2000221E08FF26323D52133A451332271348EC
:105D3000484B4647130818FF261E192D161D2D1017
:105D4000231CF5EFFCE5DCDBC5D3E4DD1C3B02F4F2
:105D5000FAE4FBE3F1CCBDC5BEBDA9989EA899A805
:105D6000B4A7A7928F9E9E9D929DB2D5DAC2CCF524
:105D7000CBCCAAC0E6DED7E4E6E8D6E5DCD7D7EBA5
:105D8000EAEAE2D5D6B9C9D5DBE7FDECDFD5CECC62
:105D9000D0B4BEDDD7F3180DEAEEF4F1DED9C8D2E7
:105DA000FAE4E2D5D50505EADFF6E7E6E8E6F1F53F
:105DB000D6F2EBF2F0151A0D0EE5DDDBE525EBEB87
:105DC000222500FA0309F900EF100BEBF601080891
:105DD000E2EB2E2A1016210916123B334C33565390
:105DE0002904211A292D2C30421207E71122415D86
:105DF000673820300D19342C1CF4051B574D5842C0
:105E000015353E3B33434B5B4C6C6C71666D5C3FB0
:105E10004E2F0D4B14383C575E4F3F28525C48FFC5
:105E2000432C485A565F4D4B534B5360595C5E525E
:105E30004A4F4B4C584E42435241082742392F3368
:105E400017072047362620183206EA190D2D33345D
:105E500032130E082DF7DEDAF301DD08241C2E4C78
:105E60002C222510100811151E271B0A061B2714AB
:105E7000132723192A1837170809F3FF1D031F28B2
:105E80001101E9E1030CE106F70622FF25676738F7
:105E9000FC22F1BAEF1A4C1A3240335929125B1D19
:105EA0000E083D4F253936346574271E0619240720
:105EB00014FC4C5C1D254931313A10F6F4FC566C4B
:105EC0003E4719447367422F38383C270803032D97
:105ED000364A463A21FAE1E1E3201C0E02405A72AA
:105EE00052281F0FF0EC02E8EF4930514F1C1F22DF
:105EF0003B735A1A0037313C4178272DDFFD4B3C6C
:105F000058426225333F685F1C010A3E2FFDF3EFC4
:105F1000242430140EE8ED1506FA275F5850353B5F
:105F20005748F7E409DF010FE8E80D23373237441B
:105F300001261E1DF5F21D022C09F6F5CDC0EB0958
:105F400015F8FEF72E241A1308120501393B1926FD
:105F50001F1806EBFACBA7C99191BC2B1B14FBD9D8
:105F6000EAF2CDB4A4A2958BBAD2B5ACAEBBA49CD8
:105F70008BA9C2D3CF99BACAC6CDD7EDC5B6C7D9FA
:105F8000B1BEA4B3D3D2CFC7DAFD0607E7C9CFBDF0
:105F9000AFAAE5DCC8DBC2CDD4E3D1B2DAE5C5E314
:105FA00000ECE1082728F4CBC5D9DFEACED4BAF457
:105FB00019040E2D21E5F30C1A5006130BF1FAF912
:105FC000E2E4EC0ED1EDF913202C0D364E252A0813
:105FD000E0D7C4EFE1FBF90E303A5838465213B718
:105FE0000847105619112AE2462CFEFAFE312E13EC
:105FF00044433D6C706E726F706E6D505D1BD9F2D4
:10600000216E6E69594246792C404628293B472A21
:10601000131F593C0F10185C373D23DAD3A8939512
:10602000BAC6DCA2DFEEAA9D9FCDDAD09DB9EBD334
:10603000DDD9CFCBFAECC8FAF2D3FD1104E322E8A4
:10604000F1E6FFE0D5E7F8D80A30F1FDE10F392994
:106050001F2E0C11462A1C1B251A00183D3F3E1608
:10606000FE10291C0F140E193E2BF1C1AEC8EBF027
:10607000DEF125342D1E2C3C4A2AFFE1DADB0E012D
:10608000EC0F1D0DF114080700F8C1F91A07E0D74D
:10609000C9102C13361AFD1003E5DC01F8223E3935
:1060A0003A38130E04020BDAD3F3121E06FBED018D
:1060B00028114C5D1CF6EAE6D1D8EC0E4053405A4C
:1060C000521F2A26FD08374C604E562E0F27332CC0
:1060D00030553CF60B370D0F3425272E2D383A2B33
:1060E0000A202230594727D8061502254E634B4314
:1060F000532A333D26111C18181D2325FFE5E1FC0A
:1061000022284C141909F4342F032A5D3E3C2F0A2F
:10611000FB1E495424375B24EBD7ECECF6303758A0
:106120006D3B30555C2EFEE63467555A2111DED3A7
:106130003D5D351F1DEE58270B2221EAD92C34E88E
:10614000FC2F1F3A2B4E452CF7F81024221E1B1053
:106150002712454F1D343422DED2A7BBDD1209F7CA
:1061600011F0B6CCBFB3BECCCFBBD0ACE4D9D7C056
:10617000BE988F8D98ABA4C6EDCFACC6C7BCB5F5A5
:10618000DEB1B48F8F9FBBD7CDD3CDC5E4F9EDDDA4
:10619000EFFAF1E3E1DEECEB13FFECE3CFB1C2DDAC
:1061A0000606EF0C2C3B2C41402A321D0A0C182508
:1061B0001F041E03D0E706111623333C24121514C6
:1061C00005E0D1E50C20271F2316141D27171409FD
:1061D0001C0C03191907DBDE1B2107100A0610052A
:1061E00011140FFE0CF1CEB2B7BABFB0C6DD202934
:1061F000000C01FAF2EDD3D2DFC7DAD18AACA79353
:10620000969AF5ECB8CECCCEBFC4E2D5E8AFA1A942
:10621000AFC2BB90B18FA1C7BDC9D4D6E6030301FD
:10622000D6D7C3D3EEE7D6C9A4998ABDDDB8D3DAF1
:10623000FC122325211D36210BEFDAE9BDCDE4CF79
:10624000F2FB1C0ECEDDE7F1F7E0F80F1BEFD5D522
:10625000EDF2B8DBE10B1EFA0C0D15121D1E13FD3D
:10626000ECF0041902F9EAF201D8C4C9EA24312297
:106270001EF8F507172019EFEEE0DDF0CEC6FF217E
:10628000200BE6EFFB1C1505E9E0E2F600F7F3DF73
:10629000DCBDE80D0C00F6E6D80308E8F5E4C6C955
:1062A000C3CFCAEE1C222604DAE401F4C8ED0A1AB0
:1062B000F8B3D9E3F319363D2F1D13091EF6EFC9C4
:1062C000EA132E4D5D6F55FA0F36432D0F252752D9
:1062D0002200FD104327E1151309131E1817122180
:1062E0005F440AFA1DFB0A1E1CFEF9E2DEFA010FEA
:1062F0000C0B5B72605A6F412B41422918EFDD1382
:106300001818FB0F3223FF2D4C0520432E1808EBE5
:1063100002FC041306F9F3F30502E7EC22282D280A
:10632000F51136284C4634220F0906E5C5DBEBE3B0
:106330000F4D6A6F19ED36350F4A59532B366222CD
:10634000150B12273B3E361BF42370616458542E04
:106350003139695737556221F60112060F06292196
:1063600038262205DD182D3F070A2BFAFBF6FF0819
:1063700018E7F11D273104332C271F06FA12373D89
:106380002B11373F0CF804F407CFA2C1F6E8E3F174
:1063900004FE3034D8A4B9FD221EFC161D03EF0BF9
:1063A0001BFFC5ECE4053311061CF901EC101FECD2
:1063B000F9180A1A1E1B250A446F482D1904EACB46
:1063C000CDFE040CFDEF16292609E916412C170213
:1063D000DFCDCBD6E1FAFE070F0AF81928291F0AEC
:1063E00008FE11281CFAE6CADAF7F9FE021D0AF8BF
:1063F000FA100B2E1800EEECDDE5E3162107F7ECA2
:106400000206FA07F4DFEEDEE4F90C0900F0F1F61B
:10641000EAE2E0DDD6D0D0C9C5C1BFC9C0C5C6C695
:10642000E4FFF6E4DBD4C0CACDE4C0A494AAD9EA60
:10643000F7E2E8E9C2CAB8C7CFB7B0B5C9E5E7EB3C
:10644000D1CEC4B2C2D8D1C8BAB5CADDC0C0C2B2FA
:10645000DE1A1AF7E4EAEDCDB6C7D8E9FAF5050574
:106460000A0C180EF0DCE8EDD1D0CEE2E1EAF91822
:10647000330BD8E0E2DFE5F1F7FEE40AFCFF300C75
:106480000614FA1F2C111010F7EBDF051A1C150F5C
:106490001304FBFEFEE8DAD7E202F2CAE7EEDAEF17
:1064A0000608E8CDE9ED00DF919DEEFBECEFECF0A6
:1064B000E4C5C604E5E609E2CDE8CEA4C3DCDEBE51
:1064C000D8EFDDE9D7CFD5F9EEE8DDD39B9EE3F435
:1064D000DCDEE600EDF3F0E5F6DAD5EAD0D5F7E755
:1064E000D1C5CCE307FCFB0BF8E6E0D4CDCFD7E970
:1064F000E8F9FB010F0303EBEEFBEEED030B0EF5EA
:10650000FE0613232E1208FCF60C0806122727138A
:106510000E2A2B17140AFFE1E8F80C2930171A2667
:10652000161303EBEC0B201F09FB0B2414081C1E95
:10653000EDCDED2209030FF51B0CF0222D311019C2
:106540003B2BFFFD0900EE0606160BFF0F2D26065E
:10655000060B1C13E4F3E101FFF200DBE0F1FCF7B2
:10656000061110141500D7F7D9E63A2203F9F6F60A
:10657000F2E5D7E5F61E26100A0C00E8E90D181B17
:106580001C290AE5F5F4D1D4E6F2F400F0FD0C166E
:10659000303235293D2AFCE5F4120FF8101C131592
:1065A00011F3F316211A10183D27130F0A0E13ECDE
:1065B000F1F906FDF6E1D6DFDCEA011B3C3201E031
:1065C000EFECDAE6FED5CBD2ECEAED0409FF0302EC
:1065D000E7F400F8E0C6C2D0E2DAF2FF03EDF50C12
:1065E000FAE6E4E6FB150F0608F8E7EAF6ECECFD40
:1065F000FF031406F7FAEA010304120B0AF1090F6C
:10660000F8122104F9EDE3FDF2F90E0F1D16F0EC7E
:106610000CF5EAE5D8D1EBF5E6072216F1F0F4E83F
:10662000EAE7E7F0FB2B1D03F60FFAEAE20011059B
:10663000FCF8FDF9F0FF18E3DCFD1E0BE5EEF0F3CE
:10664000E2F6F9050B1E2705EFECF0E90102DFDAAF
:10665000F8F1061905E8EFFE00FBF6CDD4DAE5F710
:10666000EEC2D1D9E1E2E5C6EC0A0106E1D5DCE2F1
:10667000F5F1F2EDEEF3FC03040A1E11EDE1DCE2AC
:10668000F7F1EFFD04F1FF02F8EDE4EFEDF8F8F3B8
:10669000F8FCFD02FCE6E4F2F5DDE1F4F4FFF9F2CA
:1066A000FE06F2E6E8F6F0F5F2E9E7E7FA0108F8A7
:1066B000F2F2F403FCF5F8EE000A00F60A030A0908
:1066C000F1061101F1FD0806161D060B1108170849
:1066D00017160606ECE6FEFFFCF607FEF4FCF3FCDC
:1066E000FF0C2917FB0801F1F7FBF5FFF900F8DCB7
:1066F000EEF8FD09F5F1F302FAE5E0E7F0F2F1FC5E
:10670000080400F7F6E2E60BF8E9D4DDEEECE80069
:1067100006ECF80DFAFBF0F10C0904F3EBF4FAF5D2
:10672000FF00EEE9C7DAE3C0D1F2F3EBE3D7E1DF34
:10673000C6BCDAE4CDD1DEDDF2F4F3FB06DEE0F830
:10674000F8F6FAFDEEE7F0010105000309FDEEF0B1
:10675000EEE4E2ECFD06F9F8EDE0EDF6E6E5FA111F
:106760001A201F0908EBE8FAEEEBE4F901FC03F943
:10677000FB05FCFFF7F604FCFAF402F5E8FBE9FC84
:10678000F9E7EEEFE8F7F6F0E2E7EFF0DBE404F725
:10679000F1F9F1E6E7D4CDD6EEF9F8F1E1FB030823
:1067A0001108E3D3E4E1E1F0FBFBF8E8E805FAE7E0
:1067B000F4E3EAEEE9E0DCE3EFFDFDF3FDF0E8F9F8
:1067C000F4FFECF9F4E0F1F30EFDE209200DF60020
:1067D0000100FBE5F3EFDDEDF7F3ECFC090A09FA44
:1067E00001171C16F9E8F1FC01FDFFF7011511EE88
:1067F000EDFE0A0E02E4F6040D09FAFEFDFB191780
:1068000001ECFE0AFB010525332D23190E0F0506A9
:10681000050D0F0A06F7E9F7E4F6FC04FFFCFE0499
:10682000120201060B09F7F7FDFBF5FAFD11F2FF65
:106830002B272410FF08141A01F3D7D9F3F5EAFD2A
:106840000403110DF6E5E0DAEA0700F9FE02F3F8B9
:10685000F6F0FC010803FE0308010F0C0E04E7EE3E
:10686000EEECE7F8EFFA0B0FFEE9DDDAD9FCFBF10D
:10687000FBE6DEDDE3FD03FF0F02F5FE0B04F0F4A3
:10688000DCE3FCF5F5120E0A06F3EFF31614FD0E29
:10689000FAF6EED7D6E2ED0E1B080506FE10140D33
:1068A0000E06F8FE0B1112EDEA06FFFDF8E7FA00FE
:1068B000FEF7F707FFF5F7D9E3CCD0F50F170E0C6D
:1068C000040109F5EAE5ECEDF0FA0203FDFCF2E95A
:1068D000DFEE0013FDF21724190807FCFE0BFEF192
:1068E00003FCF8FF06FE01FE03131614FF03130F4B
:1068F00017100E1605100BF2FEF6F800FFF804084C
:106900000709010902FAFDF9E8F6ECF002F60708BA
:1069100008FF01FDF601FD050D0A0E0B01FDFCF15E
:10692000F5F0F6FEFFFEF4F2F2F8FBFDFCF9F9EEED
:10693000F9F9FE05FD03050907040C030504F8EC4D
:10694000E6E1E4EEEDF5FEE9F1F2E4F1F2F5F7F758
:10695000FCF3F2F9E5EDEDF4F9F9FD0410151D185D
:106960000E07FEF7F7F4F3ECF0EAEFF2EBF1F0F5D7
:10697000FDF2FE140E0FF2F6EDE3FBF3FB09010846
:1069800003F9F0F2E2D6E4F5FA020D14120B161A2E
:106990000FFFF701192C15FC050F0716101314092A
:1069A00006FCF6FB020504F6ECFF0905FBF60812EF
:1069B00018181905030405010F160D07050A0C0127
:1069C000F5FB08FE05FDF6FCFDFF02F6F80607ECF8
:1069D000EEF8F2EAF2E8EFFEFCEDE4E8F3F8F2F1AB
:1069E000F6F902FCFBEFE9E3EE010304FEFFFBF71F
:1069F000F1EDF3F6EFE8E4E0DED8E5EAEEF2E6E406
:106A0000EDE8E5E6E7EAEAE5E0EBEDEAEAECEEF2EE
:106A1000FB01F9EBEFF7FBFCFFFEF9F0ECF2F8F30A
:106A2000F0EDEEF8030201FCFCFFFE00FEFCF0ECD2
:106A3000FBFFF6F1F3FDFCF7F3F6F3ECFCF5F7FEE4
:106A4000F3F0F9F9E8EDFF090C0BFEF9FAFA020789
:106A500002FCFE07FFF8FCFF06010309070502FF21
:106A600001FA010BFD000401090AFEFDF5F404061C
:106A7000FEFE02FCEF010604FAF1F6060F0C02FF1F
:106A80000802F1EC00110E09FDF5FCF9081108F6F9
:106A9000E8E3E2EEEBF0FEF6F1F50001F7F4FB01BE
:106AA000EEEFFDEFECF0EBF402FDF0F4FBF5F0FCA3
:106AB000F4ECF2FAF3FE0E0A01E9E3EEF1EDEDEB90
:106AC000F2FCFEF9FB0200000B0702FEF5F5040DD7
:106AD000160D00F7FB070A0300FFF6FA0105071081
:106AE000100C04FD04090AFCF2F7FE06010A171156
:106AF000100D06070406FF08090201FB0508070B35
:106B000005FBFF0305050603FDF7F3FA0804050876
:106B1000FE090BFDFC010508F9F3F6EAF1F7020E98
:106B200006FAF7FCF9E5E5F8F7EEF5F2F1EFE7F133
:106B3000FBF9FCF9F5E4ECF2EFF3F7EDDDE1DDD67E
:106B4000E6EEEFEBF6FD070E01080A0A080B0A0055
:106B50000F0EFFFEF1F3F5EEFC090BF3F0FC0B0A50
:106B6000F6F2F0EF050A01FA060604FCF40308ED5C
:106B7000E6FE0401F9F30417120DFEF8F3E9EBED5C
:106B8000F3F4FEFFEFECF4F9F0E8EDF5F3F8F5FAC5
:106B9000FCF8F4F1FF09FDFB030F09020703050DE3
:106BA0000BFAFBFDF7F1F7F6FE0605FAEDEBEEF258
:106BB000F7F3EDF7F3E5EEFB04FEFF080707080720
:106BC0000707F7F2FBF3EDEEFD0D05F8F7060704F6
:106BD00002F5F4EEFB090A0507030302F8F7FD0AC4
:106BE0000E0B0605000902FE0610100B0B0D06FC2D
:106BF0000206090A0B0F110C030502020203080D1D
:106C00000800F9F2F5F2F2F7FC06FCF3EBF1F3F908
:106C1000FDFDF7F0F2F1FD04FCFE0602070AFBECB5
:106C2000F0F8010A0E09081303F1F9F1E3EEF2F3AB
:106C300004100506FBECEEEDE2E1E6F5FBF4EEEB0D
:106C4000F3F2EAF0FCFAF501FEFA01F5FA110B088D
:106C5000090705FBFC0203EFE6E6E2EEF9F2F8FABB
:106C6000F70406F5F3FCFAFAFAFAF5FB0CFDF4FA70
:106C7000060C100B000F0C080B050D100E1619104A
:106C80000B09080F140B080AF9E3E7F3F9FFF1F910
:106C900000020C0E0802FAFD060D060508F4E7F2E4
:106CA000FD0606FFFFFEF5F4FF0C0602FAF6F8FB00
:106CB000F1E7F1F1FCFAF0F502FBF8FCFDFD060648
:106CC000010503F8FBF8F1F5FEFDF4F2F3F8FEF729
:106CD000F901FCFAFB060A100F06F1F1F1F10707C2
:106CE00000F6F5FE0502F8FA06080B07020B070886
:106CF00009110E06FDFBFEF9F6F7F2FD030603018E
:106D0000FF03FF050B0402FEEEEDFD0304080B0874
:106D1000FDFAFE0002FAFDFCFE00FFF7F2FFFAEAC0
:106D2000E9F5FCFC0202FF03060C06FDFAF8F9FD8A
:106D30000200FC0606F9FAFD030100FAF6F3F7EE8D
:106D4000F2FBF7FB0505030E0F05010602FDFEF839
:106D5000F0F70506FF00FE050C0C07030B0C0A04F8
:106D6000040A06000005080C0E0C0D10040004FBBC
:106D7000F5FD040E0E0705070605050503000205CF
:106D800004FCF8FBFEFBFAFCFBF3F3FDFDF6F8F860
:106D9000F8F7F4F4F8FEFEF7F1F1F0F1F5F7F8FB8F
:106DA000F8F90001FEF7FA030303FFFCFDFAFAFE0F
:106DB00002FEFFFDF5F7FAF9FBF9F2F4F3F1F6F84C
:106DC000FAFDFEFFFCFBF7FE05FEFBFEFCFCFD00F2
:106DD00002FF02FCFF0307100BFDF7FB0200FAFBAA
:106DE000FDFDFFFF0200F9F9F5F5F4FA01FDFEF8EB
:106DF000F2F8040805FDFF01F9F6000804FCFBF9B0
:106E0000FCFCFB0000F7F4F2F1F3FCFCF7FA00FDE8
:106E10000101F8FBFFF9F0F901060913130B020257
:106E200005FBF9FCFD0002F9F4F5FB04FFFDFAFA9D
:106E3000F9F7FF0202FC030A0A05020203F9F6FE53
:106E400002070B0402FC0208FC0201FFFAFC040D1D
:106E50000B0000FDF4FAFDFAF4FC0004050204073F
:106E60000B08020000000301020500F9FCFD040408
:106E7000FF010500FFFBF6F6F8F70002FF00010333
:106E800001FDFAF9FDFBF3FB00FDF9FCFBFD040835
:106E9000040000FDFF00FCFA03070501FAF6FC02FE
:106EA0000505FF0204060501FF00FC020601FD02C4
:106EB00000FFFEFBFAFBF8F9F6FA0102050B07FFEB
:106EC000FBFA0200FDFCFBFBFAF9F5FB0000FB00FE
:106ED000FF01020304FCFCFDFD0307040200FF01A7
:106EE000FF040908FFFD00FE0000FAFCFD0003029C
:106EF000FF00FCFCFCF9FCFF010302FF0000FFFDAA
:106F0000FDFCFAFBFE02FCF7F5F5F9F9F6FAFDFBDC
:106F1000FAFDFCFAFB03070700FCF900020101007F
:106F2000000506070802FEFDFD01FF0100FCFDFE55
:106F3000030202FF01FFFC02020301000205040339
:106F400006040601FF030000FEFF01000504020223
:106F50000301FF0101FDFDFBF9FAFAFCFD0003024C
:106F6000FFF9FD0200FF010203FD0000FDFDFDFD34
:106F7000FAFA00FDFDFCF9F7F8F7FBFE000300004C
:106F800000010301FCF9FBFE01FEFDFDFAFC01FE20
:106F9000FDFAFD0000FDF9F8FDFEFDFBF8FAF7FC37
:106FA000FDFD0300FC00FFFFFAF9F7FAFD0000FE0B
:106FB00003FF00FD000202FFFAFE02FE00FF0000D8
:106FC00002020304010305040301FDFEFC00FFFBB4
:106FD000FBFCFEFEFD0000FE00FFFBFBFC00FFFBD8
:106FE000FAFAFCFCF9F8F7FBFBFDFEFEFFFEFCFEE7
:106FF000FFFE00FD01FFFDFBF9FD00FF00020303A2
:10700000030201FDFEFE010200FFFFFEFFFEFDFF89
:10701000FFFE00010201FFFD00020101FFFFFD0173
:10702000FFFFFF01000000010201FFFDFDFDFCFC70
:10703000FDFE01FF0000FFFFFDFBFBFDFDFDFDFD73
:10704000FCFEFEFEFEFEFDFDFDFEFFFEFD0101005D
:10705000FE0000FF0000FF00FF00FF0000FFFF0038
:10706000FCFF00FDFDFDFDFE01FF01FEFF00FF0036
:10707000FEFD00FEFDFE01FFFDFE01FFFEFBFBFF2E
:107080000102FF020301FF0002030203020302FFE9
:10709000FF01FDFDFAFAFAFCFDFDFDFCFFFF00001B
:1070A000FDFD00FF01030100FEFDFDFD000000FDF0
:1070B000FE02030302030000FEFDFE0000FEFD00D1
:1070C00000FFFF01FFFDFE0000FF01FEFE01FF01CA
:1070D000FFFDFDFDFDFDFD0300FDFDFE01FFFFFBCE
:1070E000FAFEFC0000FCFDFAFDFF00FCFEFDFEFDCB
:1070F000FEFDFEFCFAF8FAFDFDFAFBFDFDFDFF01C9
:10710000FF01FF01FF01FF01FF01FF01FF01FF017F
:10711000FF01FF01FF01FFFD000102FF01FFFEFD76
:10712000FDFE01FCFE0000FF01FF01FF01FF01FE6B
:10713000FE01FF01030201020000FDFF01FF00004C
:10714000FFFF0000FF01FEFE000000FDFEFDFEFD52
:1071500000FFFF01FF0000FDFDFDFDFDFE01FF0141
:1071600002000000020301FF00FDFF01FDFDFDFF25
:1071700001FF0000FEFDFFFF01FF01FF000303020E
:107180000301FF0001FF0201FF01FF01FF000201F7
:10719000FF00FF0000FF00FEFDFF01FF01FEFDFDFF
:1071A000FDFDFDFDFE01FFFF0000FF00FC0000FEF5
:1071B000FDFEFF00FFFF01FF01FFFDFEFC0000FDE3
:1071C000FDFDFDFDFDFDFDFF01FF01FFFDFFFEFDDE
:1071D000FEFDFE00FEFFFDFE01FF0102FF01FFFFBD
:1071E000FF01FF00FDFF0000FDFFFF01FE00FFFDAE
:1071F00001FF00FF01FF01FF01FF01FF01FF01FF90
:1072000001FF0000FF01FF01FEFE01FCFDFDFEFD90
:10721000FEFDFEFDFEFC00FEFF0000FFFDFEFDFD8D
:10722000FDFEFDFE01FF0002080000F600085A0105
:10723000084E01084B0108460108410108370108C2
:107240002D010500FF0002030000EC0008320108D8
:107250001E01080A01083201081E010500FF000294
:10726000030000F600083E010302010302010302CD
:1072700001030201030201040A01030201030201E6
:1072800003020103020103020104020103020103DC
:107290000201030201030201040A010302010302C5
:1072A00001030201030201040501030201030201BB
:1072B00003020103020104020103020103020103AC
:1072C0000201030201050000FF00020201060001A5
:1072D00000E000FF0002020106000100E000FF00E4
:1072E000000026720000000000000045720000004F
:1072F000000000005E7200000000000000C9720083
:10730000000000000000D472000000000274400081
:1073100000C219C21902365A0000F017F017020213
:1073200001020F10020203041112020205061314D7
:107330000202070815160202090A171802020B0CAE
:10734000191A02020D0E1B1C140801010101010192
:107350000101010101020304010101010101010117
:1073600001010101010101010506070801010101F7
:10737000010101010101010101010101090A0B0CD7
:107380000101010101010101010101010101010DE1
:107390000E0F100101010101010111121314151644
:1073A0001718191A1B1C1D1E1F202122010123243E
:1073B00025262728292A2B2C2D2E2F303132333405
:1073C0003501363738393A3B3C3D3E3F4041424338
:1073D00044454647484901014A4B4C4D4E4F505198
:1073E00052535455565758595A5B060A015C5D5E14
:1073F0005F606162636465666768696A6B6C6D6E25
:107400006F707172737475767778797A7B7C7D7E14
:107410007F808182830184850101010186870101CA
:1074200001018889010101011011131415171819A0
:107430001A1B1C1D1E1E1F1F1F1F1F1E1E1D1C1C76
:107440001B19181716141311100E0D0B0A08070636
:107450000504030201010000000000010102020313
:1074600004050708090B0C0E0305060706050302B1
:107470000100010200122A3C54667808182E425876
:107480006C7F0D1F32495C73848040201008040219
:1074900050524F544543542020434F4D504F4E457A
:1074A0004E5453210020202020452E532E442E20C0
:1074B00041545441434B0020202020202020564599
:1074C0005220312E3000202320323030382C434CD3
:1074D000415920434F5747494C4C00504342205399
:1074E0004D4F4B4544212047414D45204F56455275
:1074F0002100574156453A002020202020202020FE
:10750000202020202020202020202020002020209B
:107510005245414348454420574156453A20202092
:107520002020200047414D452F50524F4752414D9A
:107530003A20434C415920434F5747494C4C202A4D
:1075400020415544494F3A20414C454320424F5534
:1075500052515545202A204D4F56452043524F53F6
:107560005348414952205749544820442D504144E2
:1075700020414E44204649524520594F5552204DF6
:107580004F56532041542054484520535041524BAC
:10759000532057495448204120414E442042204224
:1075A0005554544F4E532E20204649524520544F97
:1075B0004F204F4654454E20414E4420594F55527E
:1075C000204D4F56532057494C4C204F564552485A
:1075D00045415420414E44204D55535420434F4F74
:1075E0004C20444F574E2E2E2E202020202020208D
:1075F000202020202020202020202020202020208B
:10760000202020202020202020202020202020009A
:1076100011241FBECFEFD0E1DEBFCDBF14BE88E185
:107620000FB6F89480936000109260000FBE11E0D6
:10763000A0E0B1E0EEEFF8ED02C005900D92A43AA3
:10764000B107D9F71FE0A4EAB1E001C01D92AE3D39
:10765000B107E1F7F894E1E2FCE080E090E020E897
:1076600002C02193019632E08C309307D4F381E27B
:107670009CE090932E0E80932D0E10922F0EE2E33D
:10768000FEE080E090E003C0108201963A968430DC
:107690009105D4F31092810015BCE0E0F1E080E0A8
:1076A00090E02EEF02C02193019680399105DCF322
:1076B0009093630E8093620E80E00E944853E0E056
:1076C000F7E080E090E050ED20EC31E041E00EC0CA
:1076D00010821182009719F45093020701C01282A0
:1076E000348323831782408701963F968F3091051C
:1076F0007CF39093630E8093620E91E09093F90B6C
:107700008FEF87B984B980E88AB98CE081B983EFBB
:1077100082B91092FA0B86E08093FB0B10928500E1
:107720001092840083E0809389008DE88093880024
:1077300089E08093810082E080936F0082E484BDC1
:1077400017BC95BD83E88093B0001092B30090936E
:10775000B10081E185B978940E943C540E94A167F0
:107760000C947D6C0C940000DC52E652F452FF51F4
:10777000EBEDC8950000EA95E1F700C000C040912C
:107780000507509106074ABD5BBDC0910B07D0911C
:107790000C0740900D0750900E0790900707F0904F
:1077A0000207E0900A0770910107672F677088242D
:1077B00000EDA02EA4EEB7E075D00027E101D301C3
:1077C00008B9F1E0E091F40B119311931193119327
:1077D00011931193E091F50B119311931193119360
:1077E00011931193E091F60B11931193119311934F
:1077F00011931193E091F70B11931193119311933E
:1078000011931193E091F80B11931193119311932C
:107810001193119363957395FA94A9F483940FE0EF
:10782000809EF001E050F94F058016800ABC1BBC19
:10783000C385D485458456849780F280E284718123
:10784000672F677008C00000000000000000000003
:1078500009E00A95F1F7791509F4E20109F47727AF
:1078600009F46627AA9441F0683019F000C000C0FE
:10787000A3CF6627A096A0CFC895C8950E94CD52E9
:107880004091FB0B405D4093FB0B11E00091FD0B21
:1078900001270093FD0BE1E0E093FC0BE2E0E093B5
:1078A000360008952898E0912D0EF0912E0E01914A
:1078B0002EE0ED32F20721E23CE00093B30008F045
:1078C000F901E0932D0EF0932E0E1E01C090E207F9
:1078D000D090E30780E323E036E0D1E040EA56E0D1
:1078E00098E00D91099F112D0F71FA01029FE00D93
:1078F000F11D0281C081F601089FE00DF11D139F6B
:10790000E00DF11DC093F40B0590099205900992CA
:1079100005900992059009920590099205900992A7
:107920000D91099F112D0F71FA01029FE00DF11DBC
:107930000281C081F601089FE00DF11D139FE00D4B
:10794000F11DC093F50B05900992059009920590E1
:107950000992059009920D91289A05900992059037
:107960000992099F112D0F71FA01029FE00DF11D7F
:107970000281C081F601089FE00DF11D139FE00D0B
:10798000F11DC093F60B05900992059009920590A0
:1079900009920590099205900992059009920D911E
:1079A000099F112D0F71FA01029FE00DF11D028157
:1079B000C081F601089FE00DF11D139FE00DF11D40
:1079C000C093F70B059009920590099205900992D2
:1079D0000590099205900992059009920D91099FD1
:1079E000112D0F71FA01029FE00DF11D0281C0817E
:1079F000F601089FE00DF11D139FE00DF11DC093EE
:107A0000F80B05900992059009920590099205904E
:107A100009920590099205900992E1013D01DE016C
:107A20001EEF4AB55BB5639FC0013A2F307ECE2D65
:107A3000CC0FDD27C057DE4FE991F881C6E0D1E0D9
:107A4000CC9020E3C29EA395AF71A32B040E151E0C
:107A5000080E191E0994F001C895C895C895C895D7
:107A60000591D990D1120D2D08B9CC900591D990DE
:107A7000D1120D2D08B9C29E0591D990D1120D2DAC
:107A800008B9040E151E0591D990D1120D2D08B913
:107A9000080E191E0591D990D1120D2D08B9A39584
:107AA000AF710591D990D1120D2D08B9A32BF0011A
:107AB0000591D990D1120D2D08B9CC900591D9908E
:107AC000D1120D2D08B9C29E0591D990D1120D2D5C
:107AD00008B9040E151E0591D990D1120D2D08B9C3
:107AE000080E191E0591D990D1120D2D08B9A39534
:107AF000AF710591D990D1120D2D08B9A32BF001CA
:107B00000591D990D1120D2D08B9CC900591D9903D
:107B1000D1120D2D08B9C29E0591D990D1120D2D0B
:107B200008B9040E151E0591D990D1120D2D08B972
:107B3000080E191E0591D990D1120D2D08B9A395E3
:107B4000AF710591D990D1120D2D08B9A32BF00179
:107B50000591D990D1120D2D08B9CC900591D990ED
:107B6000D1120D2D08B9C29E0591D990D1120D2DBB
:107B700008B9040E151E0591D990D1120D2D08B922
:107B8000080E191E0591D990D1120D2D08B9A39593
:107B9000AF710591D990D1120D2D08B9A32BF00129
:107BA0000591D990D1120D2D08B9CC900591D9909D
:107BB000D1120D2D08B9C29E0591D990D1120D2D6B
:107BC00008B9040E151E0591D990D1120D2D08B9D2
:107BD000080E191E0591D990D1120D2D08B9A39543
:107BE000AF710591D990D1120D2D08B9A32BF001D9
:107BF0000591D990D1120D2D08B9CC900591D9904D
:107C0000D1120D2D08B9C29E0591D990D1120D2D1A
:107C100008B9040E151E0591D990D1120D2D08B981
:107C2000080E191E0591D990D1120D2D08B9A395F2
:107C3000AF710591D990D1120D2D08B9A32BF00188
:107C40000591D990D1120D2D08B9CC900591D990FC
:107C5000D1120D2D08B9C29E0591D990D1120D2DCA
:107C600008B9040E151E0591D990D1120D2D08B931
:107C7000080E191E0591D990D1120D2D08B9A395A2
:107C8000AF710591D990D1120D2D08B9A32BF00138
:107C90000591D990D1120D2D08B9CC900591D990AC
:107CA000D1120D2D08B9C29E0591D990D1120D2D7A
:107CB00008B9040E151E0591D990D1120D2D08B9E1
:107CC000080E191E0591D990D1120D2D08B9A39552
:107CD000AF710591D990D1120D2D08B9A32BF001E8
:107CE0000591D990D1120D2D08B9CC900591D9905C
:107CF000D1120D2D08B9C29E0591D990D1120D2D2A
:107D000008B9040E151E0591D990D1120D2D08B990
:107D1000080E191E0591D990D1120D2D08B9A39501
:107D2000AF710591D990D1120D2D08B9A32BF00197
:107D30000591D990D1120D2D08B9CC900591D9900B
:107D4000D1120D2D08B9C29E0591D990D1120D2DD9
:107D500008B9040E151E0591D990D1120D2D08B940
:107D6000080E191E0591D990D1120D2D08B9A395B1
:107D7000AF710591D990D1120D2D08B9A32BF00147
:107D80000591D990D1120D2D08B9CC900591D990BB
:107D9000D1120D2D08B9C29E0591D990D1120D2D89
:107DA00008B9040E151E0591D990D1120D2D08B9F0
:107DB000080E191E0591D990D1120D2D08B9A39561
:107DC000AF710591D990D1120D2D08B9A32BF001F7
:107DD0000591D990D1120D2D08B9CC900591D9906B
:107DE000D1120D2D08B9C29E0591D990D1120D2D39
:107DF00008B9040E151E0591D990D1120D2D08B9A0
:107E0000080E191E0591D990D1120D2D08B9A39510
:107E1000AF710591D990D1120D2D08B9A32BF001A6
:107E20000591D990D1120D2D08B9CC900591D9901A
:107E3000D1120D2D08B9C29E0591D990D1120D2DE8
:107E400008B9040E151E0591D990D1120D2D08B94F
:107E5000080E191E0591D990D1120D2D08B9A395C0
:107E6000AF710591D990D1120D2D08B9A32BF00156
:107E70000591D990D1120D2D08B9CC900591D990CA
:107E8000D1120D2D08B9C29E0591D990D1120D2D98
:107E900008B9040E151E0591D990D1120D2D08B9FF
:107EA000080E191E0591D990D1120D2D08B9A39570
:107EB000AF710591D990D1120D2D08B9A32BF00106
:107EC0000591D990D1120D2D08B9CC900591D9907A
:107ED000D1120D2D08B9C29E0591D990D1120D2D48
:107EE00008B9040E151E0591D990D1120D2D08B9AF
:107EF000080E191E0591D990D1120D2D08B9A39520
:107F0000AF710591D990D1120D2D08B9A32BF001B5
:107F10000591D990D1120D2D08B9CC900591D99029
:107F2000D1120D2D08B9C29E0591D990D1120D2DF7
:107F300008B9040E151E0591D990D1120D2D08B95E
:107F4000080E191E0591D990D1120D2D08B9A395CF
:107F5000AF710591D990D1120D2D08B9A32BF00165
:107F60000591D990D1120D2D08B9CC900591D990D9
:107F7000D1120D2D08B9C29E0591D990D1120D2DA7
:107F800008B9040E151E0591D990D1120D2D08B90E
:107F9000080E191E0591D990D1120D2D08B9A3957F
:107FA000AF710591D990D1120D2D08B9A32BF00115
:107FB0000591D990D1120D2D08B9CC900591D99089
:107FC000D1120D2D08B9C29E0591D990D1120D2D57
:107FD00008B9040E151E0591D990D1120D2D08B9BE
:107FE000080E191E0591D990D1120D2D08B9A3952F
:107FF000AF710591D990D1120D2D08B9A32BF001C5
:108000000591D990D1120D2D08B9CC900591D99038
:10801000D1120D2D08B9C29E0591D990D1120D2D06
:1080200008B9040E151E0591D990D1120D2D08B96D
:10803000080E191E0591D990D1120D2D08B9A395DE
:10804000AF710591D990D1120D2D08B9A32BF00174
:108050000591D990D1120D2D08B9CC900591D990E8
:10806000D1120D2D08B9C29E0591D990D1120D2DB6
:1080700008B9040E151E0591D990D1120D2D08B91D
:10808000080E191E0591D990D1120D2D08B9A3958E
:10809000AF710591D990D1120D2D08B9A32BF00124
:1080A0000591D990D1120D2D08B9CC900591D99098
:1080B000D1120D2D08B9C29E0591D990D1120D2D66
:1080C00008B9040E151E0591D990D1120D2D08B9CD
:1080D000080E191E0591D990D1120D2D08B9A3953E
:1080E000AF710591D990D1120D2D08B9A32BF001D4
:1080F0000591D990D1120D2D08B9CC900591D99048
:10810000D1120D2D08B9C29E0591D990D1120D2D15
:1081100008B9040E151E0591D990D1120D2D08B97C
:10812000080E191E0591D990D1120D2D08B9A395ED
:10813000AF710591D990D1120D2D08B9A32BF00183
:108140000895F0013196CC9000C000C000C000C07E
:108150000591D990D1120D2D08B9C29E0591D990E3
:10816000D1120D2D08B9040E151E0591D990D1120A
:108170000D2D08B9080E191E0591D990D1120D2D9B
:1081800008B9A395AF710591D990D1120D2D08B9F9
:10819000A32BF0010591D990D1120D2D08B9CC90E7
:1081A0000591D990D1120D2D08B9C29E0591D99093
:1081B000D1120D2D08B9040E151E0591D990D112BA
:1081C0000D2D08B9080E191E0591D990D1120D2D4B
:1081D00008B9A395AF710591D990D1120D2D08B9A9
:1081E000A32BF0010591D990D1120D2D08B9CC9097
:1081F0000591D990D1120D2D08B9C29E0591D99043
:10820000D1120D2D08B9040E151E0591D990D11269
:108210000D2D08B9080E191E0591D990D1120D2DFA
:1082200008B9A395AF710591D990D1120D2D08B958
:10823000A32BF0010591D990D1120D2D08B9CC9046
:108240000591D990D1120D2D08B9C29E0591D990F2
:10825000D1120D2D08B9040E151E0591D990D11219
:108260000D2D08B9080E191E0591D990D1120D2DAA
:1082700008B9A395AF710591D990D1120D2D08B908
:10828000A32BF0010591D990D1120D2D08B9CC90F6
:108290000591D990D1120D2D08B9C29E0591D990A2
:1082A000D1120D2D08B9040E151E0591D990D112C9
:1082B0000D2D08B9080E191E0591D990D1120D2D5A
:1082C00008B9A395AF710591D990D1120D2D08B9B8
:1082D000A32BF0010591D990D1120D2D08B9CC90A6
:1082E0000591D990D1120D2D08B9C29E0591D99052
:1082F000D1120D2D08B9040E151E0591D990D11279
:108300000D2D08B9080E191E0591D990D1120D2D09
:1083100008B9A395AF710591D990D1120D2D08B967
:10832000A32BF0010591D990D1120D2D08B9CC9055
:108330000591D990D1120D2D08B9C29E0591D99001
:10834000D1120D2D08B9040E151E0591D990D11228
:108350000D2D08B9080E191E0591D990D1120D2DB9
:1083600008B9A395AF710591D990D1120D2D08B917
:10837000A32BF0010591D990D1120D2D08B9CC9005
:108380000591D990D1120D2D08B9C29E0591D990B1
:10839000D1120D2D08B9040E151E0591D990D112D8
:1083A0000D2D08B9080E191E0591D990D1120D2D69
:1083B00008B9A395AF710591D990D1120D2D08B9C7
:1083C000A32BF0010591D990D1120D2D08B9CC90B5
:1083D0000591D990D1120D2D08B9C29E0591D99061
:1083E000D1120D2D08B9040E151E0591D990D11288
:1083F0000D2D08B9080E191E0591D990D1120D2D19
:1084000008B9A395AF710591D990D1120D2D08B976
:10841000A32BF0010591D990D1120D2D08B9CC9064
:108420000591D990D1120D2D08B9C29E0591D99010
:10843000D1120D2D08B9040E151E0591D990D11237
:108440000D2D08B9080E191E0591D990D1120D2DC8
:1084500008B9A395AF710591D990D1120D2D08B926
:10846000A32BF0010591D990D1120D2D08B9CC9014
:108470000591D990D1120D2D08B9C29E0591D990C0
:10848000D1120D2D08B9040E151E0591D990D112E7
:108490000D2D08B9080E191E0591D990D1120D2D78
:1084A00008B9A395AF710591D990D1120D2D08B9D6
:1084B000A32BF0010591D990D1120D2D08B9CC90C4
:1084C0000591D990D1120D2D08B9C29E0591D99070
:1084D000D1120D2D08B9040E151E0591D990D11297
:1084E0000D2D08B9080E191E0591D990D1120D2D28
:1084F00008B9A395AF710591D990D1120D2D08B986
:10850000A32BF0010591D990D1120D2D08B9CC9073
:108510000591D990D1120D2D08B9C29E0591D9901F
:10852000D1120D2D08B9040E151E0591D990D11246
:108530000D2D08B9080E191E0591D990D1120D2DD7
:1085400008B9A395AF710591D990D1120D2D08B935
:10855000A32BF0010591D990D1120D2D08B9CC9023
:108560000591D990D1120D2D08B9C29E0591D990CF
:10857000D1120D2D08B9040E151E0591D990D112F6
:108580000D2D08B9080E191E0591D990D1120D2D87
:1085900008B9A395AF710591D990D1120D2D08B9E5
:1085A000A32BF0010591D990D1120D2D08B9CC90D3
:1085B0000591D990D1120D2D08B9C29E0591D9907F
:1085C000D1120D2D08B9040E151E0591D990D112A6
:1085D0000D2D08B9080E191E0591D990D1120D2D37
:1085E00008B9A395AF710591D990D1120D2D08B995
:1085F000A32BF0010591D990D1120D2D08B9CC9083
:108600000591D990D1120D2D08B9C29E0591D9902E
:10861000D1120D2D08B9040E151E0591D990D11255
:108620000D2D08B9080E191E0591D990D1120D2DE6
:1086300008B9A395AF710591D990D1120D2D08B944
:10864000A32BF0010591D990D1120D2D08B9CC9032
:108650000591D990D1120D2D08B9C29E0591D990DE
:10866000D1120D2D08B9040E151E0591D990D11205
:108670000D2D08B9080E191E0591D990D1120D2D96
:1086800008B9A395AF710591D990D1120D2D08B9F4
:10869000A32BF0010591D990D1120D2D08B9CC90E2
:1086A0000591D990D1120D2D08B9C29E0591D9908E
:1086B000D1120D2D08B9040E151E0591D990D112B5
:1086C0000D2D08B9080E191E0591D990D1120D2D46
:1086D00008B9A395AF710591D990D1120D2D08B9A4
:1086E000A32BF0010591D990D1120D2D08B9CC9092
:1086F0000591D990D1120D2D08B9C29E0591D9903E
:10870000D1120D2D08B9040E151E0591D990D11264
:108710000D2D08B9080E191E0591D990D1120D2DF5
:1087200008B9A395AF710591D990D1120D2D08B953
:10873000A32BF0010591D990D1120D2D08B9CC9041
:108740000591D990D1120D2D08B9C29E0591D990ED
:10875000D1120D2D08B9040E151E0591D990D11214
:108760000D2D08B9080E191E0591D990D1120D2DA5
:1087700008B9A395AF710591D990D1120D2D08B903
:10878000A32BF0010591D990D1120D2D08B9CC90F1
:108790000591D990D1120D2D08B9C29E0591D9909D
:1087A000D1120D2D08B9040E151E0591D990D112C4
:1087B0000D2D08B9080E191E0591D990D1120D2D55
:1087C00008B9A395AF710591D990D1120D2D08B9B3
:1087D000A32BF0010591D990D1120D2D08B9CC90A1
:1087E0000591D990D1120D2D08B9C29E0591D9904D
:1087F000D1120D2D08B9040E151E0591D990D11274
:108800000D2D08B9080E191E0591D990D1120D2D04
:1088100008B9A395AF710591D990D1120D2D08B962
:10882000A32BF0010591D990D1120D2D08B9CC9050
:108830000895F0013296CC90C29E00C000C000C0E6
:108840000591D990D1120D2D08B9040E151E059170
:10885000D990D1120D2D08B9080E191E0591D99085
:10886000D1120D2D08B9A395AF710591D990D112F0
:108870000D2D08B9A32BF0010591D990D1120D2D22
:1088800008B9CC900591D990D1120D2D08B9C29E8E
:108890000591D990D1120D2D08B9040E151E059120
:1088A000D990D1120D2D08B9080E191E0591D99035
:1088B000D1120D2D08B9A395AF710591D990D112A0
:1088C0000D2D08B9A32BF0010591D990D1120D2DD2
:1088D00008B9CC900591D990D1120D2D08B9C29E3E
:1088E0000591D990D1120D2D08B9040E151E0591D0
:1088F000D990D1120D2D08B9080E191E0591D990E5
:10890000D1120D2D08B9A395AF710591D990D1124F
:108910000D2D08B9A32BF0010591D990D1120D2D81
:1089200008B9CC900591D990D1120D2D08B9C29EED
:108930000591D990D1120D2D08B9040E151E05917F
:10894000D990D1120D2D08B9080E191E0591D99094
:10895000D1120D2D08B9A395AF710591D990D112FF
:108960000D2D08B9A32BF0010591D990D1120D2D31
:1089700008B9CC900591D990D1120D2D08B9C29E9D
:108980000591D990D1120D2D08B9040E151E05912F
:10899000D990D1120D2D08B9080E191E0591D99044
:1089A000D1120D2D08B9A395AF710591D990D112AF
:1089B0000D2D08B9A32BF0010591D990D1120D2DE1
:1089C00008B9CC900591D990D1120D2D08B9C29E4D
:1089D0000591D990D1120D2D08B9040E151E0591DF
:1089E000D990D1120D2D08B9080E191E0591D990F4
:1089F000D1120D2D08B9A395AF710591D990D1125F
:108A00000D2D08B9A32BF0010591D990D1120D2D90
:108A100008B9CC900591D990D1120D2D08B9C29EFC
:108A20000591D990D1120D2D08B9040E151E05918E
:108A3000D990D1120D2D08B9080E191E0591D990A3
:108A4000D1120D2D08B9A395AF710591D990D1120E
:108A50000D2D08B9A32BF0010591D990D1120D2D40
:108A600008B9CC900591D990D1120D2D08B9C29EAC
:108A70000591D990D1120D2D08B9040E151E05913E
:108A8000D990D1120D2D08B9080E191E0591D99053
:108A9000D1120D2D08B9A395AF710591D990D112BE
:108AA0000D2D08B9A32BF0010591D990D1120D2DF0
:108AB00008B9CC900591D990D1120D2D08B9C29E5C
:108AC0000591D990D1120D2D08B9040E151E0591EE
:108AD000D990D1120D2D08B9080E191E0591D99003
:108AE000D1120D2D08B9A395AF710591D990D1126E
:108AF0000D2D08B9A32BF0010591D990D1120D2DA0
:108B000008B9CC900591D990D1120D2D08B9C29E0B
:108B10000591D990D1120D2D08B9040E151E05919D
:108B2000D990D1120D2D08B9080E191E0591D990B2
:108B3000D1120D2D08B9A395AF710591D990D1121D
:108B40000D2D08B9A32BF0010591D990D1120D2D4F
:108B500008B9CC900591D990D1120D2D08B9C29EBB
:108B60000591D990D1120D2D08B9040E151E05914D
:108B7000D990D1120D2D08B9080E191E0591D99062
:108B8000D1120D2D08B9A395AF710591D990D112CD
:108B90000D2D08B9A32BF0010591D990D1120D2DFF
:108BA00008B9CC900591D990D1120D2D08B9C29E6B
:108BB0000591D990D1120D2D08B9040E151E0591FD
:108BC000D990D1120D2D08B9080E191E0591D99012
:108BD000D1120D2D08B9A395AF710591D990D1127D
:108BE0000D2D08B9A32BF0010591D990D1120D2DAF
:108BF00008B9CC900591D990D1120D2D08B9C29E1B
:108C00000591D990D1120D2D08B9040E151E0591AC
:108C1000D990D1120D2D08B9080E191E0591D990C1
:108C2000D1120D2D08B9A395AF710591D990D1122C
:108C30000D2D08B9A32BF0010591D990D1120D2D5E
:108C400008B9CC900591D990D1120D2D08B9C29ECA
:108C50000591D990D1120D2D08B9040E151E05915C
:108C6000D990D1120D2D08B9080E191E0591D99071
:108C7000D1120D2D08B9A395AF710591D990D112DC
:108C80000D2D08B9A32BF0010591D990D1120D2D0E
:108C900008B9CC900591D990D1120D2D08B9C29E7A
:108CA0000591D990D1120D2D08B9040E151E05910C
:108CB000D990D1120D2D08B9080E191E0591D99021
:108CC000D1120D2D08B9A395AF710591D990D1128C
:108CD0000D2D08B9A32BF0010591D990D1120D2DBE
:108CE00008B9CC900591D990D1120D2D08B9C29E2A
:108CF0000591D990D1120D2D08B9040E151E0591BC
:108D0000D990D1120D2D08B9080E191E0591D990D0
:108D1000D1120D2D08B9A395AF710591D990D1123B
:108D20000D2D08B9A32BF0010591D990D1120D2D6D
:108D300008B9CC900591D990D1120D2D08B9C29ED9
:108D40000591D990D1120D2D08B9040E151E05916B
:108D5000D990D1120D2D08B9080E191E0591D99080
:108D6000D1120D2D08B9A395AF710591D990D112EB
:108D70000D2D08B9A32BF0010591D990D1120D2D1D
:108D800008B9CC900591D990D1120D2D08B9C29E89
:108D90000591D990D1120D2D08B9040E151E05911B
:108DA000D990D1120D2D08B9080E191E0591D99030
:108DB000D1120D2D08B9A395AF710591D990D1129B
:108DC0000D2D08B9A32BF0010591D990D1120D2DCD
:108DD00008B9CC900591D990D1120D2D08B9C29E39
:108DE0000591D990D1120D2D08B9040E151E0591CB
:108DF000D990D1120D2D08B9080E191E0591D990E0
:108E0000D1120D2D08B9A395AF710591D990D1124A
:108E10000D2D08B9A32BF0010591D990D1120D2D7C
:108E200008B9CC900591D990D1120D2D08B9C29EE8
:108E30000591D990D1120D2D08B9040E151E05917A
:108E4000D990D1120D2D08B9080E191E0591D9908F
:108E5000D1120D2D08B9A395AF710591D990D112FA
:108E60000D2D08B9A32BF0010591D990D1120D2D2C
:108E700008B9CC900591D990D1120D2D08B9C29E98
:108E80000591D990D1120D2D08B9040E151E05912A
:108E9000D990D1120D2D08B9080E191E0591D9903F
:108EA000D1120D2D08B9A395AF710591D990D112AA
:108EB0000D2D08B9A32BF0010591D990D1120D2DDC
:108EC00008B9CC900591D990D1120D2D08B9C29E48
:108ED0000591D990D1120D2D08B9040E151E0591DA
:108EE000D990D1120D2D08B9080E191E0591D990EF
:108EF000D1120D2D08B9A395AF710591D990D1125A
:108F00000D2D08B9A32BF0010591D990D1120D2D8B
:108F100008B9CC900591D990D1120D2D08B9C29EF7
:108F20000895F0013396CC90C29E040E151E00C029
:108F300000C00591D990D1120D2D08B9080E191E47
:108F40000591D990D1120D2D08B9A395AF71059156
:108F5000D990D1120D2D08B9A32BF0010591D9900C
:108F6000D1120D2D08B9CC900591D990D1120D2DAB
:108F700008B9C29E0591D990D1120D2D08B9040EE1
:108F8000151E0591D990D1120D2D08B9080E191E84
:108F90000591D990D1120D2D08B9A395AF71059106
:108FA000D990D1120D2D08B9A32BF0010591D990BC
:108FB000D1120D2D08B9CC900591D990D1120D2D5B
:108FC00008B9C29E0591D990D1120D2D08B9040E91
:108FD000151E0591D990D1120D2D08B9080E191E34
:108FE0000591D990D1120D2D08B9A395AF710591B6
:108FF000D990D1120D2D08B9A32BF0010591D9906C
:10900000D1120D2D08B9CC900591D990D1120D2D0A
:1090100008B9C29E0591D990D1120D2D08B9040E40
:10902000151E0591D990D1120D2D08B9080E191EE3
:109030000591D990D1120D2D08B9A395AF71059165
:10904000D990D1120D2D08B9A32BF0010591D9901B
:10905000D1120D2D08B9CC900591D990D1120D2DBA
:1090600008B9C29E0591D990D1120D2D08B9040EF0
:10907000151E0591D990D1120D2D08B9080E191E93
:109080000591D990D1120D2D08B9A395AF71059115
:10909000D990D1120D2D08B9A32BF0010591D990CB
:1090A000D1120D2D08B9CC900591D990D1120D2D6A
:1090B00008B9C29E0591D990D1120D2D08B9040EA0
:1090C000151E0591D990D1120D2D08B9080E191E43
:1090D0000591D990D1120D2D08B9A395AF710591C5
:1090E000D990D1120D2D08B9A32BF0010591D9907B
:1090F000D1120D2D08B9CC900591D990D1120D2D1A
:1091000008B9C29E0591D990D1120D2D08B9040E4F
:10911000151E0591D990D1120D2D08B9080E191EF2
:109120000591D990D1120D2D08B9A395AF71059174
:10913000D990D1120D2D08B9A32BF0010591D9902A
:10914000D1120D2D08B9CC900591D990D1120D2DC9
:1091500008B9C29E0591D990D1120D2D08B9040EFF
:10916000151E0591D990D1120D2D08B9080E191EA2
:109170000591D990D1120D2D08B9A395AF71059124
:10918000D990D1120D2D08B9A32BF0010591D990DA
:10919000D1120D2D08B9CC900591D990D1120D2D79
:1091A00008B9C29E0591D990D1120D2D08B9040EAF
:1091B000151E0591D990D1120D2D08B9080E191E52
:1091C0000591D990D1120D2D08B9A395AF710591D4
:1091D000D990D1120D2D08B9A32BF0010591D9908A
:1091E000D1120D2D08B9CC900591D990D1120D2D29
:1091F00008B9C29E0591D990D1120D2D08B9040E5F
:10920000151E0591D990D1120D2D08B9080E191E01
:109210000591D990D1120D2D08B9A395AF71059183
:10922000D990D1120D2D08B9A32BF0010591D99039
:10923000D1120D2D08B9CC900591D990D1120D2DD8
:1092400008B9C29E0591D990D1120D2D08B9040E0E
:10925000151E0591D990D1120D2D08B9080E191EB1
:109260000591D990D1120D2D08B9A395AF71059133
:10927000D990D1120D2D08B9A32BF0010591D990E9
:10928000D1120D2D08B9CC900591D990D1120D2D88
:1092900008B9C29E0591D990D1120D2D08B9040EBE
:1092A000151E0591D990D1120D2D08B9080E191E61
:1092B0000591D990D1120D2D08B9A395AF710591E3
:1092C000D990D1120D2D08B9A32BF0010591D99099
:1092D000D1120D2D08B9CC900591D990D1120D2D38
:1092E00008B9C29E0591D990D1120D2D08B9040E6E
:1092F000151E0591D990D1120D2D08B9080E191E11
:109300000591D990D1120D2D08B9A395AF71059192
:10931000D990D1120D2D08B9A32BF0010591D99048
:10932000D1120D2D08B9CC900591D990D1120D2DE7
:1093300008B9C29E0591D990D1120D2D08B9040E1D
:10934000151E0591D990D1120D2D08B9080E191EC0
:109350000591D990D1120D2D08B9A395AF71059142
:10936000D990D1120D2D08B9A32BF0010591D990F8
:10937000D1120D2D08B9CC900591D990D1120D2D97
:1093800008B9C29E0591D990D1120D2D08B9040ECD
:10939000151E0591D990D1120D2D08B9080E191E70
:1093A0000591D990D1120D2D08B9A395AF710591F2
:1093B000D990D1120D2D08B9A32BF0010591D990A8
:1093C000D1120D2D08B9CC900591D990D1120D2D47
:1093D00008B9C29E0591D990D1120D2D08B9040E7D
:1093E000151E0591D990D1120D2D08B9080E191E20
:1093F0000591D990D1120D2D08B9A395AF710591A2
:10940000D990D1120D2D08B9A32BF0010591D99057
:10941000D1120D2D08B9CC900591D990D1120D2DF6
:1094200008B9C29E0591D990D1120D2D08B9040E2C
:10943000151E0591D990D1120D2D08B9080E191ECF
:109440000591D990D1120D2D08B9A395AF71059151
:10945000D990D1120D2D08B9A32BF0010591D99007
:10946000D1120D2D08B9CC900591D990D1120D2DA6
:1094700008B9C29E0591D990D1120D2D08B9040EDC
:10948000151E0591D990D1120D2D08B9080E191E7F
:109490000591D990D1120D2D08B9A395AF71059101
:1094A000D990D1120D2D08B9A32BF0010591D990B7
:1094B000D1120D2D08B9CC900591D990D1120D2D56
:1094C00008B9C29E0591D990D1120D2D08B9040E8C
:1094D000151E0591D990D1120D2D08B9080E191E2F
:1094E0000591D990D1120D2D08B9A395AF710591B1
:1094F000D990D1120D2D08B9A32BF0010591D99067
:10950000D1120D2D08B9CC900591D990D1120D2D05
:1095100008B9C29E0591D990D1120D2D08B9040E3B
:10952000151E0591D990D1120D2D08B9080E191EDE
:109530000591D990D1120D2D08B9A395AF71059160
:10954000D990D1120D2D08B9A32BF0010591D99016
:10955000D1120D2D08B9CC900591D990D1120D2DB5
:1095600008B9C29E0591D990D1120D2D08B9040EEB
:10957000151E0591D990D1120D2D08B9080E191E8E
:109580000591D990D1120D2D08B9A395AF71059110
:10959000D990D1120D2D08B9A32BF0010591D990C6
:1095A000D1120D2D08B9CC900591D990D1120D2D65
:1095B00008B9C29E0591D990D1120D2D08B9040E9B
:1095C000151E0591D990D1120D2D08B9080E191E3E
:1095D0000591D990D1120D2D08B9A395AF710591C0
:1095E000D990D1120D2D08B9A32BF0010591D99076
:1095F000D1120D2D08B9CC900591D990D1120D2D15
:1096000008B9C29E0591D990D1120D2D08B9040E4A
:10961000151E0895F0013496CC90C29E040E151EBE
:10962000080E191E00C00591D990D1120D2D08B950
:10963000A395AF710591D990D1120D2D08B9A32B27
:10964000F0010591D990D1120D2D08B9CC9005915A
:10965000D990D1120D2D08B9C29E0591D990D11281
:109660000D2D08B9040E151E0591D990D1120D2D9E
:1096700008B9080E191E0591D990D1120D2D08B9FF
:10968000A395AF710591D990D1120D2D08B9A32BD7
:10969000F0010591D990D1120D2D08B9CC9005910A
:1096A000D990D1120D2D08B9C29E0591D990D11231
:1096B0000D2D08B9040E151E0591D990D1120D2D4E
:1096C00008B9080E191E0591D990D1120D2D08B9AF
:1096D000A395AF710591D990D1120D2D08B9A32B87
:1096E000F0010591D990D1120D2D08B9CC900591BA
:1096F000D990D1120D2D08B9C29E0591D990D112E1
:109700000D2D08B9040E151E0591D990D1120D2DFD
:1097100008B9080E191E0591D990D1120D2D08B95E
:10972000A395AF710591D990D1120D2D08B9A32B36
:10973000F0010591D990D1120D2D08B9CC90059169
:10974000D990D1120D2D08B9C29E0591D990D11290
:109750000D2D08B9040E151E0591D990D1120D2DAD
:1097600008B9080E191E0591D990D1120D2D08B90E
:10977000A395AF710591D990D1120D2D08B9A32BE6
:10978000F0010591D990D1120D2D08B9CC90059119
:10979000D990D1120D2D08B9C29E0591D990D11240
:1097A0000D2D08B9040E151E0591D990D1120D2D5D
:1097B00008B9080E191E0591D990D1120D2D08B9BE
:1097C000A395AF710591D990D1120D2D08B9A32B96
:1097D000F0010591D990D1120D2D08B9CC900591C9
:1097E000D990D1120D2D08B9C29E0591D990D112F0
:1097F0000D2D08B9040E151E0591D990D1120D2D0D
:1098000008B9080E191E0591D990D1120D2D08B96D
:10981000A395AF710591D990D1120D2D08B9A32B45
:10982000F0010591D990D1120D2D08B9CC90059178
:10983000D990D1120D2D08B9C29E0591D990D1129F
:109840000D2D08B9040E151E0591D990D1120D2DBC
:1098500008B9080E191E0591D990D1120D2D08B91D
:10986000A395AF710591D990D1120D2D08B9A32BF5
:10987000F0010591D990D1120D2D08B9CC90059128
:10988000D990D1120D2D08B9C29E0591D990D1124F
:109890000D2D08B9040E151E0591D990D1120D2D6C
:1098A00008B9080E191E0591D990D1120D2D08B9CD
:1098B000A395AF710591D990D1120D2D08B9A32BA5
:1098C000F0010591D990D1120D2D08B9CC900591D8
:1098D000D990D1120D2D08B9C29E0591D990D112FF
:1098E0000D2D08B9040E151E0591D990D1120D2D1C
:1098F00008B9080E191E0591D990D1120D2D08B97D
:10990000A395AF710591D990D1120D2D08B9A32B54
:10991000F0010591D990D1120D2D08B9CC90059187
:10992000D990D1120D2D08B9C29E0591D990D112AE
:109930000D2D08B9040E151E0591D990D1120D2DCB
:1099400008B9080E191E0591D990D1120D2D08B92C
:10995000A395AF710591D990D1120D2D08B9A32B04
:10996000F0010591D990D1120D2D08B9CC90059137
:10997000D990D1120D2D08B9C29E0591D990D1125E
:109980000D2D08B9040E151E0591D990D1120D2D7B
:1099900008B9080E191E0591D990D1120D2D08B9DC
:1099A000A395AF710591D990D1120D2D08B9A32BB4
:1099B000F0010591D990D1120D2D08B9CC900591E7
:1099C000D990D1120D2D08B9C29E0591D990D1120E
:1099D0000D2D08B9040E151E0591D990D1120D2D2B
:1099E00008B9080E191E0591D990D1120D2D08B98C
:1099F000A395AF710591D990D1120D2D08B9A32B64
:109A0000F0010591D990D1120D2D08B9CC90059196
:109A1000D990D1120D2D08B9C29E0591D990D112BD
:109A20000D2D08B9040E151E0591D990D1120D2DDA
:109A300008B9080E191E0591D990D1120D2D08B93B
:109A4000A395AF710591D990D1120D2D08B9A32B13
:109A5000F0010591D990D1120D2D08B9CC90059146
:109A6000D990D1120D2D08B9C29E0591D990D1126D
:109A70000D2D08B9040E151E0591D990D1120D2D8A
:109A800008B9080E191E0591D990D1120D2D08B9EB
:109A9000A395AF710591D990D1120D2D08B9A32BC3
:109AA000F0010591D990D1120D2D08B9CC900591F6
:109AB000D990D1120D2D08B9C29E0591D990D1121D
:109AC0000D2D08B9040E151E0591D990D1120D2D3A
:109AD00008B9080E191E0591D990D1120D2D08B99B
:109AE000A395AF710591D990D1120D2D08B9A32B73
:109AF000F0010591D990D1120D2D08B9CC900591A6
:109B0000D990D1120D2D08B9C29E0591D990D112CC
:109B10000D2D08B9040E151E0591D990D1120D2DE9
:109B200008B9080E191E0591D990D1120D2D08B94A
:109B3000A395AF710591D990D1120D2D08B9A32B22
:109B4000F0010591D990D1120D2D08B9CC90059155
:109B5000D990D1120D2D08B9C29E0591D990D1127C
:109B60000D2D08B9040E151E0591D990D1120D2D99
:109B700008B9080E191E0591D990D1120D2D08B9FA
:109B8000A395AF710591D990D1120D2D08B9A32BD2
:109B9000F0010591D990D1120D2D08B9CC90059105
:109BA000D990D1120D2D08B9C29E0591D990D1122C
:109BB0000D2D08B9040E151E0591D990D1120D2D49
:109BC00008B9080E191E0591D990D1120D2D08B9AA
:109BD000A395AF710591D990D1120D2D08B9A32B82
:109BE000F0010591D990D1120D2D08B9CC900591B5
:109BF000D990D1120D2D08B9C29E0591D990D112DC
:109C00000D2D08B9040E151E0591D990D1120D2DF8
:109C100008B9080E191E0591D990D1120D2D08B959
:109C2000A395AF710591D990D1120D2D08B9A32B31
:109C3000F0010591D990D1120D2D08B9CC90059164
:109C4000D990D1120D2D08B9C29E0591D990D1128B
:109C50000D2D08B9040E151E0591D990D1120D2DA8
:109C600008B9080E191E0591D990D1120D2D08B909
:109C7000A395AF710591D990D1120D2D08B9A32BE1
:109C8000F0010591D990D1120D2D08B9CC90059114
:109C9000D990D1120D2D08B9C29E0591D990D1123B
:109CA0000D2D08B9040E151E0591D990D1120D2D58
:109CB00008B9080E191E0591D990D1120D2D08B9B9
:109CC000A395AF710591D990D1120D2D08B9A32B91
:109CD000F0010591D990D1120D2D08B9CC900591C4
:109CE000D990D1120D2D08B9C29E0591D990D112EB
:109CF0000D2D08B9040E151E0591D990D1120D2D08
:109D000008B9080E191E0895F0013596CC90C29E30
:109D1000040E151E080E191EA395AF710591D9905A
:109D2000D1120D2D08B9A32BF0010591D990D112B4
:109D30000D2D08B9CC900591D990D1120D2D08B9EF
:109D4000C29E0591D990D1120D2D08B9040E151E91
:109D50000591D990D1120D2D08B9080E191E059143
:109D6000D990D1120D2D08B9A395AF710591D99055
:109D7000D1120D2D08B9A32BF0010591D990D11264
:109D80000D2D08B9CC900591D990D1120D2D08B99F
:109D9000C29E0591D990D1120D2D08B9040E151E41
:109DA0000591D990D1120D2D08B9080E191E0591F3
:109DB000D990D1120D2D08B9A395AF710591D99005
:109DC000D1120D2D08B9A32BF0010591D990D11214
:109DD0000D2D08B9CC900591D990D1120D2D08B94F
:109DE000C29E0591D990D1120D2D08B9040E151EF1
:109DF0000591D990D1120D2D08B9080E191E0591A3
:109E0000D990D1120D2D08B9A395AF710591D990B4
:109E1000D1120D2D08B9A32BF0010591D990D112C3
:109E20000D2D08B9CC900591D990D1120D2D08B9FE
:109E3000C29E0591D990D1120D2D08B9040E151EA0
:109E40000591D990D1120D2D08B9080E191E059152
:109E5000D990D1120D2D08B9A395AF710591D99064
:109E6000D1120D2D08B9A32BF0010591D990D11273
:109E70000D2D08B9CC900591D990D1120D2D08B9AE
:109E8000C29E0591D990D1120D2D08B9040E151E50
:109E90000591D990D1120D2D08B9080E191E059102
:109EA000D990D1120D2D08B9A395AF710591D99014
:109EB000D1120D2D08B9A32BF0010591D990D11223
:109EC0000D2D08B9CC900591D990D1120D2D08B95E
:109ED000C29E0591D990D1120D2D08B9040E151E00
:109EE0000591D990D1120D2D08B9080E191E0591B2
:109EF000D990D1120D2D08B9A395AF710591D990C4
:109F0000D1120D2D08B9A32BF0010591D990D112D2
:109F10000D2D08B9CC900591D990D1120D2D08B90D
:109F2000C29E0591D990D1120D2D08B9040E151EAF
:109F30000591D990D1120D2D08B9080E191E059161
:109F4000D990D1120D2D08B9A395AF710591D99073
:109F5000D1120D2D08B9A32BF0010591D990D11282
:109F60000D2D08B9CC900591D990D1120D2D08B9BD
:109F7000C29E0591D990D1120D2D08B9040E151E5F
:109F80000591D990D1120D2D08B9080E191E059111
:109F9000D990D1120D2D08B9A395AF710591D99023
:109FA000D1120D2D08B9A32BF0010591D990D11232
:109FB0000D2D08B9CC900591D990D1120D2D08B96D
:109FC000C29E0591D990D1120D2D08B9040E151E0F
:109FD0000591D990D1120D2D08B9080E191E0591C1
:109FE000D990D1120D2D08B9A395AF710591D990D3
:109FF000D1120D2D08B9A32BF0010591D990D112E2
:10A000000D2D08B9CC900591D990D1120D2D08B91C
:10A01000C29E0591D990D1120D2D08B9040E151EBE
:10A020000591D990D1120D2D08B9080E191E059170
:10A03000D990D1120D2D08B9A395AF710591D99082
:10A04000D1120D2D08B9A32BF0010591D990D11291
:10A050000D2D08B9CC900591D990D1120D2D08B9CC
:10A06000C29E0591D990D1120D2D08B9040E151E6E
:10A070000591D990D1120D2D08B9080E191E059120
:10A08000D990D1120D2D08B9A395AF710591D99032
:10A09000D1120D2D08B9A32BF0010591D990D11241
:10A0A0000D2D08B9CC900591D990D1120D2D08B97C
:10A0B000C29E0591D990D1120D2D08B9040E151E1E
:10A0C0000591D990D1120D2D08B9080E191E0591D0
:10A0D000D990D1120D2D08B9A395AF710591D990E2
:10A0E000D1120D2D08B9A32BF0010591D990D112F1
:10A0F0000D2D08B9CC900591D990D1120D2D08B92C
:10A10000C29E0591D990D1120D2D08B9040E151ECD
:10A110000591D990D1120D2D08B9080E191E05917F
:10A12000D990D1120D2D08B9A395AF710591D99091
:10A13000D1120D2D08B9A32BF0010591D990D112A0
:10A140000D2D08B9CC900591D990D1120D2D08B9DB
:10A15000C29E0591D990D1120D2D08B9040E151E7D
:10A160000591D990D1120D2D08B9080E191E05912F
:10A17000D990D1120D2D08B9A395AF710591D99041
:10A18000D1120D2D08B9A32BF0010591D990D11250
:10A190000D2D08B9CC900591D990D1120D2D08B98B
:10A1A000C29E0591D990D1120D2D08B9040E151E2D
:10A1B0000591D990D1120D2D08B9080E191E0591DF
:10A1C000D990D1120D2D08B9A395AF710591D990F1
:10A1D000D1120D2D08B9A32BF0010591D990D11200
:10A1E0000D2D08B9CC900591D990D1120D2D08B93B
:10A1F000C29E0591D990D1120D2D08B9040E151EDD
:10A200000591D990D1120D2D08B9080E191E05918E
:10A21000D990D1120D2D08B9A395AF710591D990A0
:10A22000D1120D2D08B9A32BF0010591D990D112AF
:10A230000D2D08B9CC900591D990D1120D2D08B9EA
:10A24000C29E0591D990D1120D2D08B9040E151E8C
:10A250000591D990D1120D2D08B9080E191E05913E
:10A26000D990D1120D2D08B9A395AF710591D99050
:10A27000D1120D2D08B9A32BF0010591D990D1125F
:10A280000D2D08B9CC900591D990D1120D2D08B99A
:10A29000C29E0591D990D1120D2D08B9040E151E3C
:10A2A0000591D990D1120D2D08B9080E191E0591EE
:10A2B000D990D1120D2D08B9A395AF710591D99000
:10A2C000D1120D2D08B9A32BF0010591D990D1120F
:10A2D0000D2D08B9CC900591D990D1120D2D08B94A
:10A2E000C29E0591D990D1120D2D08B9040E151EEC
:10A2F0000591D990D1120D2D08B9080E191E05919E
:10A30000D990D1120D2D08B9A395AF710591D990AF
:10A31000D1120D2D08B9A32BF0010591D990D112BE
:10A320000D2D08B9CC900591D990D1120D2D08B9F9
:10A33000C29E0591D990D1120D2D08B9040E151E9B
:10A340000591D990D1120D2D08B9080E191E05914D
:10A35000D990D1120D2D08B9A395AF710591D9905F
:10A36000D1120D2D08B9A32BF0010591D990D1126E
:10A370000D2D08B9CC900591D990D1120D2D08B9A9
:10A38000C29E0591D990D1120D2D08B9040E151E4B
:10A390000591D990D1120D2D08B9080E191E0591FD
:10A3A000D990D1120D2D08B9A395AF710591D9900F
:10A3B000D1120D2D08B9A32BF0010591D990D1121E
:10A3C0000D2D08B9CC900591D990D1120D2D08B959
:10A3D000C29E0591D990D1120D2D08B9040E151EFB
:10A3E0000591D990D1120D2D08B9080E191E0591AD
:10A3F000D990D1120D2D08B9A395AF710895289861
:10A400000E94A55AE7E1EA95F1F7289A10D1E0E019
:10A41000F6E0F3D0E0FF4ED0E0FF02C00E94AC595E
:10A420000895129A0C9414520C94165212984427C0
:10A430005527662777278CE00C941E520C942052E7
:10A440000C9422520C9424520C9426520C942852B0
:10A45000440F551F00994160660F771F0199616095
:10A46000139A0C9433520C94355213980C9438521E
:10A470000C943A520C943C520C943E528A9541F7FB
:10A4800040955095609570955F707F704093010C7A
:10A490005093020C6093030C7093040C9BE04830C3
:10A4A000590711F40E9430546830790711F40E9462
:10A4B00030540895EF93E091FB0BE53EE0F5E53174
:10A4C000D0F12F923F924F925F926F927F928F9234
:10A4D0009F92AF92BF92CF92DF92EF92FF920F9333
:10A4E0001F932F933F934F935F936F937F938F931C
:10A4F0009F93AF93BF93CF93DF930E94B83BDF91BD
:10A50000CF91BF91AF919F918F917F916F915F910B
:10A510004F913F912F911F910F91FF90EF90DF90FE
:10A52000CF90BF90AF909F908F907F906F905F90F3
:10A530004F903F902F90EF910895FF93EF93EFB7D7
:10A54000EF93E0918400EE50E13000F0E23000F053
:10A55000E33000F0E43000F0E53000F0E63000F0E9
:10A56000E73000F0E83000F0E93000F005D0EF917E
:10A57000EFBFEF91FF9118950F921F92E8E6F7E772
:10A580000090FA0B000C1124E00DF11D05901490C1
:10A59000F00109951F900F90089528980E94A55AE0
:10A5A000E5E1EA95F1F7E091FB0BEA95E093FB0B0F
:10A5B000289A00000000089528980E94CE5A289AF0
:10A5C0000000E1E0F6E019D02BD0089528980E9411
:10A5D000CE5AE0EB0000EA95E9F700000000289A67
:10A5E000F6E0E2E00AD0089528980E94CE5A289A10
:10A5F0000000E3E0FDEF01D008950090FB0B0A940A
:10A6000010905F0011FC0F2E0092FB0B0090FA0BD4
:10A6100011FC0E2E0092FA0BE0E011FCE1E008952F
:10A62000E3E0E0938900EDE8E09388000895E7E037
:10A63000E0938900EBE1E09388000895E0EEF4E018
:10A64000A0ECB1E066276D933197E9F711240895E6
:10A650009927772720E2629F080E191EA0ECB1E02F
:10A66000A00DB11D4C93112408950895992720E25F
:10A67000629F080E191EA0ECB1E0A00DB11D509113
:10A68000000C450F4C93112408958093000C0895FD
:10A690008093E10708958093E2079093E30708957C
:10A6A000EF92FF920F931F93CF93DF93E0E0F7E0D9
:10A6B00020E0822F60814181EF93FF932F930E94CE
:10A6C000AD602F91FF91EF913F9623952F3088F346
:10A6D00055272FE0662775E084EE97E0E0E0F7E08D
:10A6E00030854281EC01579FC00DD11D540F44238A
:10A6F00049F0317039F0699369936993699369936B
:10A700004A95C9F73F962A9559F731E02091E1071C
:10A71000213011F43091F90B00EA16E0780123E0C2
:10A72000A5E0B0E241E0F701329FE00DF11D0081AC
:10A7300011811030E9F1183DD8F50030C9F10A381F
:10A74000B8F560E0712F760F783068F1783D58F5F4
:10A750007850EC017A9FC00DD11D0880002021F4B3
:10A760006B9F030E08821FC00980002021F46B9F9D
:10A77000030E098218C00A80002021F46B9F030E8B
:10A780000A8211C00B80002021F46B9F030E0B8204
:10A790000AC00C80002039F46B9F030E0C82032E3C
:10A7A0000A940092F90B259673956395683050F2E0
:10A7B0003395303208F031E04395403208F4B3CF9E
:10A7C0007091F90B703208F071E07093F90B552716
:10A7D0002FE0662775E0E0E0F7E030854281EC018C
:10A7E000579FC00DD11D540F442349F0317039F4E7
:10A7F000699369936993699369934A95C9F73F96F9
:10A800002A9559F71124DF91CF911F910F91FF9055
:10A81000EF9008958093FE0B9093FF0B0895809125
:10A82000FC0B089511241092FC0B0895882329F441
:10A830008091010C9091020C08958091030C9091ED
:10A84000040C089580E891E080936100909361008A
:10A85000089580E890E080936100909361000895EE
:10A8600028E088E190E00FB6F894A8958093600006
:10A870000FBE2093600008950F931F9303E318E029
:10A88000C8010E94D75480E790E090930607809318
:10A8900005070E941E538FE090E00E948062C8016D
:10A8A0000E94D75441E06FEF80E00E94735800ECA3
:10A8B00017E0A8016CE088E00E94336283E090E03A
:10A8C0000E94806244EF57E06CE088E00E943362AF
:10A8D00082E090E00E948062A8016CE088E00E9423
:10A8E000336280E590E00E9480620E941E5384E102
:10A8F00090E00E9480621F910F91089590E025E101
:10A9000030E0829FF001839FF00D929FF00D1124A3
:10A91000EA59F14F6187089560935B0E089590E0C6
:10A9200025E130E0829FF001839FF00D929FF00DB2
:10A930001124EA59F14F12861182089590E025E121
:10A9400030E0829FF001839FF00D929FF00D112463
:10A95000EA59F14F81E0828B089590E025E130E0E3
:10A96000829FF001839FF00D929FF00D1124EA5910
:10A97000F14F6087089590E025E130E0829FF0017B
:10A98000839FF00D929FF00D1124EA59F14F6483DB
:10A99000089590E025E130E0829FF001839FF00D63
:10A9A000929FF00D1124EA59F14F65830895909319
:10A9B000BD0E8093BC0E8FE68093C20E1092200CC9
:10A9C000E6E6FEE021E09FEF88E120831782968390
:10A9D00013861182858375963EE0EA3BF307A9F75B
:10A9E00008951092670E10927C0E1092910E1092A4
:10A9F000A60E01969093C60E8093C50E9093650E99
:10AA00008093640E9093C90E8093C80E1092C40E6A
:10AA10001092C30E1092BB0E1092BA0E1092BE0E80
:10AA200081E08093200C1092C10E1092C00E089508
:10AA30008091640E9091650E0E94F154089580916A
:10AA40006F0E87FD03C08AEF80936F0E8091840E96
:10AA500087FD03C08AEF8093840E8091990E87FD55
:10AA600003C08AEF8093990E8091AE0E87FD03C0DC
:10AA70008AEF8093AE0E1092200C089581E08093AF
:10AA8000200C0895DC01ED91FC911197AF014F5F0F
:10AA90005F4F11965C934E93E4912E2F30E0E7FFC9
:10AAA00013C02F7730703695322F22273795279590
:10AAB000FA014F5F5F4FE4918E2F8F77280F311D82
:10AAC000E7FDF1CF4D935C93C90108958093C20EC9
:10AAD000089508950E9494590895EF92FF920F935C
:10AAE0001F93CF93DF93182F062FE42EF22EC82F3B
:10AAF000D0E085E190E0C89FF001C99FF00DD89F9C
:10AB0000F00D1124EA59F14F8285882321F08181CB
:10AB1000882309F0A5C0FF2091F485E190E0C89F4B
:10AB2000F001C99FF00DD89FF00D1124EA59F14FA3
:10AB3000128A8185882309F093C0178291C013304F
:10AB400049F51092530E89E0089FC001112420910D
:10AB5000BC0E3091BD0E280F391FF9013196459179
:10AB600054915093550E4093540EF90135968591AA
:10AB70009491840F951F9093570E8093560EF90170
:10AB8000379685919491480F591F5093590E4093D1
:10AB9000580E04C060E0812F0E9494596E2D812FC1
:10ABA0000E9480590F3799F485E190E0C89FF00129
:10ABB000C99FF00DD89FF00D1124EA59F14F8091F3
:10ABC000BF0E868780EC9EE0948B838B30C089E03B
:10ABD000089FC0011124E091BC0EF091BD0EE80F5A
:10ABE000F91F3396459154914115510571F485E152
:10ABF00090E0C89FF001C99FF00DD89FF00D11247F
:10AC0000EA59F14F148A138A12C0FA01249185E19E
:10AC100090E0C89FF001C99FF00DD89FF00D11245E
:10AC2000EA59F14F26874F5F5F4F548B438B85E185
:10AC300090E0C89FF001C99FF00DD89FF00D11243E
:10AC4000EA59F14F17861186038711828FEF8087AB
:10AC5000F782E282108A81E08287128A118A148246
:10AC6000DF91CF911F910F91FF90EF900895CF92B8
:10AC7000DF92FF920F931F93CF93DF93EEE6FEE0F8
:10AC80008181282F332727FD30958081280F311DA2
:10AC90002F3F310519F014F02FEF30E0C90137FFD5
:10ACA00002C080E090E0808375964EE0E23CF407BD
:10ACB00039F78091200C882309F019C135C1E09142
:10ACC000C50EF091C60E9F012F5F3F4F3093C60E09
:10ACD0002093C50E44914F3F69F5A9014F5F5F4F27
:10ACE0005093C60E4093C50EF90184918F3219F42A
:10ACF0001092200C0AC1863009F0EAC0FA013196A0
:10AD0000CF0101969093C60E8093C50EE491E33572
:10AD100029F49093C90E8093C80EDAC0E53409F087
:10AD2000D7C08091C80E9091C90E9093C60E8093A3
:10AD3000C50ECEC047FF02C04093BE0E542F5F70B9
:10AD4000842F90E0807F9070803B910529F1803CBA
:10AD5000910579F18039910509F042C0C901019648
:10AD6000F901449101969093C60E8093C50E019708
:10AD7000FC012491852F90E08C9FF0018D9FF00DB8
:10AD80009C9FF00D1124EA59F14F8081882309F42A
:10AD90009FC0220F638552C0C9010196F9014491F9
:10ADA00001969093C60E8093C50E0197FC012491E5
:10ADB00053C02F5F3F4F3093C60E2093C50E2150D6
:10ADC0003040F9012491852F90E08C9FF0018D9FF8
:10ADD000F00D9C9FF00D1124EA59F14F238778C0A4
:10ADE0008091BE0E582F5F7090E0807F9070803B06
:10ADF000910541F1803C910509F45EC080399105CF
:10AE000009F066C02F5F3F4F3093C60E2093C50EEA
:10AE100021503040F9012491852F90E08C9FD00182
:10AE20008D9FB00D9C9FB00D1124AA59B14F8C91EC
:10AE3000882309F44DC0220F1B966C91852F0E9428
:10AE40006D5546C02F5F3F4F3093C60E2093C50E01
:10AE500021503040F9012491473071F4852F90E062
:10AE60008C9FF0018D9FF00D9C9FF00D1124EA59ED
:10AE7000F14F220F26832CC04C3571F4852F90E0C2
:10AE80008C9FF0018D9FF00D9C9FF00D1124EA59CD
:10AE9000F14F220F24831CC04436D1F4852F90E05B
:10AEA0008C9FF0018D9FF00D9C9FF00D1124EA59AD
:10AEB000F14F220F25830CC0852F90E08C9FF0016D
:10AEC0008D9FF00D9C9FF00D1124EA59F14F43879F
:10AED00085EC9EE00E944255969587959093C40E0E
:10AEE0008093C30E1092BB0E1092BA0E02C0C5E141
:10AEF000D0E06091BA0E7091BB0E8091C30E90911C
:10AF0000C40E6817790709F4DACE6F5F7F4F70932C
:10AF1000BB0E6093BA0E8091C00E9091C10E019647
:10AF20009093C10E8093C00E02E31EE0C7E6DEE000
:10AF3000FF24BFEFCB2ED12C8989882309F05EC076
:10AF40008A899B89892B09F456C09E858D8598171F
:10AF500008F04CC050C08A852A893B898F37E9F4B4
:10AF6000D9018D91BB8BAA8B8F3F01F1F9016181D2
:10AF70001196BB8BAA8BE82FF0E0EE0FFF1FE45C6D
:10AF8000F74F0190F081E02D8F2D0995EA89FB891B
:10AF900081918D87FB8BEA8B28C0A9014F5F5F4FA2
:10AFA0005B8B4A8BF90184918F3F21F418821B8AB5
:10AFB0001A8A21C04F5F5F4F5B8B4A8B41505040D4
:10AFC000FA01649190E0880F991F845C974FFC010F
:10AFD000259134918F2DF9010995EA89FB893196E4
:10AFE000FB8BEA8B3197E491ED871E869E858D85DC
:10AFF000981709F4B0CF8E858F5F8E878985882357
:10B0000019F420E030E05DC08F858F3F11F08F5F35
:10B010008F879E81992309F44EC02F81222309F442
:10B020004AC08D81882309F446C04091C20E442352
:10B0300009F441C0899FC001112480509F4F892F7E
:10B04000992730E0BC01629FC001639F900D729F01
:10B05000900D112480509F4F892F9927242F30E085
:10B06000FC01E29FC001E39F900DF29F900D11241F
:10B0700080509F4F292F33278B818823F1F0EA815D
:10B08000F0E0E050FA44E491E058E89FC001112458
:10B0900080509F4F892F9927A601481B590B429F2B
:10B0A000C001439F900D529F900D112480509F4FDF
:10B0B000292F332702C020E030E08A819C81890F4C
:10B0C0008A83F8012083F394065F1F4F6596F4E0AE
:10B0D000FF1609F031CFDF91CF911F910F91FF90B3
:10B0E000DF90CF9008951F93CF93DF93382F562F83
:10B0F00089E0389FB0011124C091BC0ED091BD0EE3
:10B10000C60FD71FCE010396FC01A591B491FE0195
:10B1100084918150823010F413E01DC080917C0E28
:10B120008823B1F08091870E831711F4442381F4B2
:10B130008091910E882371F080919C0E831711F4F9
:10B14000442341F490918B0E8091A00E891710F446
:10B1500011E001C012E0C12FD0E0FD01249185E192
:10B1600090E0C89FF001C99FF00DD89FF00D112409
:10B17000EA59F14F26871196B48BA38B178680E589
:10B18000828357838FEF80871186128A108A81E02D
:10B190008287118A348781831482133029F51092B3
:10B1A000530E2091BC0E3091BD0E260F371FF901B2
:10B1B0003196459154915093550E4093540EF90198
:10B1C000359685919491840F951F9093570E809397
:10B1D000560EF901379685919491480F591F509357
:10B1E000590E4093580E04C060E0812F0E9494597C
:10B1F00085E190E0C89FF001C99FF00DD89FF00D48
:10B200001124EA59F14F6281812F0E948059DF9108
:10B21000CF911F910895FF920F931F93082FF62E41
:10B220000E94805910E085E190E0089FF001099F9D
:10B23000F00D189FF00D1124EA59F14FF2821F9181
:10B240000F91FF900895962F482F50E025E130E0B0
:10B25000429FF001439FF00D529FF00D1124EA59D7
:10B26000F14F6281691B62830E9480590895482FC3
:10B2700050E025E130E0429FF001439FF00D529FE6
:10B28000F00D1124EA59F14F9281690F62830E94F7
:10B290008059089500000000000000000000000038
:10B2A000000000000000000000000000000000009E
:10B2B000000000000000000000000000000000008E
:10B2C000000000000000000000000000000000007E
:10B2D000000000000000000000000000000000006E
:10B2E000000000000000000000000000000000005E
:10B2F000000000000000000000000000000000004E
:10B3000099277727E0E0F0EC660F771FE60FF71F2D
:10B31000A591B491E2E3FEE02AE0289FE00DF11D43
:10B32000A183B2831124089599277727E2E3FEE0F1
:10B330002AE0289FE00DF11D76EB760F758311242E
:10B34000089599277727E2E3FEE02AE0289FE00DA1
:10B35000F11D6083112408952F933F934F935F93C2
:10B360006F937F938F939F93AF93BF9378941124A0
:10B370000E9450530E9411520E9437562F923F92C2
:10B380004F925F926F927F928F929F92AF92BF92F5
:10B39000CF92DF92EF92FF920F931F93CF93DF93A1
:10B3A00000902F0E002019F4A1E2BCE002C0A7E239
:10B3B000BDE001E0002600922F0E02E00093300E67
:10B3C0005091500E6091540E7091550E8091530E15
:10B3D0004090510E5090520E66248090580E9090DE
:10B3E000590EA090560EB090570E1D01C3E8840D63
:10B3F000651D761D6815790508F0B501FB014491BE
:10B4000045031D92840D651D761D6815790508F0AC
:10B41000B501FB01449145031D92CA9541F7D10145
:10B420002090330E3090340E4090360E5090370EF0
:10B430006090350E1091320E70903D0E80903E0E51
:10B4400090903F0EA090400EB090410E20913C0E87
:10B45000C090470ED090480EE0904A0EF0904B0EF0
:10B460000091490E3091460E9FEFCC91DD27C7FD2C
:10B47000DFEF620C431CF2014491410300240008F9
:10B48000C10DD01D970CA81CF50144914203002466
:10B490000008C10DD01D0C0DED1CF70144914303B4
:10B4A00000240008C10DD01D0024C038D0050CF0C8
:10B4B000CFE70A94C038D0050CF4C0E8C058CD934B
:10B4C0009A9509F0D2CF4091300E4A954093300EB4
:10B4D00097E009F0CACF6092350E4092360E9092F6
:10B4E0003F0EA092400E0093490EE0924A0E5093F8
:10B4F000500E6093540E7093550E8093530EDF914F
:10B50000CF911F910F91FF90EF90DF90CF90BF9060
:10B51000AF909F908F907F906F905F904F903F90F3
:10B520002F9099278091FA0B77276091FB0B1124BC
:10B530000E946955BF91AF919F918F917F916F91BB
:10B540005F914F913F912F9108950C94A75A0C94BD
:10B55000A95A0F931F932ABDE0912D0EF0912E0E44
:10B56000019100000093B3000EE0ED32F00710F4FB
:10B570000000000010F0E1E2FCE0E0932D0EF093FB
:10B580002E0EC895C895C895C895C895C895000051
:10B59000000000002AB51F910F9108950000E0916E
:10B5A000FB0BE0FFD6CFE1E1EA95F1F700000000E8
:10B5B00008950000000000000000000000000000EE
:10B5C000000000000000000000000000000000007B
:10B5D000000000000000000000000000000000006B
:10B5E000000000000000000000000000000000005B
:10B5F000000000000000000000000000000000004B
:10B60000000306090C101316191C1F2225282B2EC7
:10B61000313336393C3F414447494C4E51535558DC
:10B620005A5C5E60626466686A6B6D6F7071737499
:10B63000757678797A7A7B7C7D7D7E7E7E7F7F7F52
:10B640007F7F7F7F7E7E7E7D7D7C7B7A7A79787638
:10B6500075747371706F6D6B6A68666462605E5C4E
:10B660005A585553514E4C494744413F3C39363363
:10B67000312E2B2825221F1C191613100C09060326
:10B6800000FDFAF7F4F0EDEAE7E4E1DEDBD8D5D22D
:10B69000CFCDCAC7C4C1BFBCB9B7B4B2AFADABA8F8
:10B6A000A6A4A2A09E9C9A9896959391908F8D8C1B
:10B6B0008B8A888786868584838382828281818142
:10B6C0008181818182828283838485868687888A3C
:10B6D0008B8C8D8F9091939596989A9C9EA0A2A406
:10B6E000A6A8ABADAFB2B4B7B9BCBFC1C4C7CACDD1
:10B6F000CFD2D5D8DBDEE1E4E7EAEDF0F4F7FAFDEE
:10B70000808182838485868788898A8B8C8D8E8FC1
:10B71000909192939495969798999A9B9C9D9E9FB1
:10B72000A0A1A2A3A4A5A6A7A8A9AAABACADAEAFA1
:10B73000B0B1B2B3B4B5B6B7B8B9BABBBCBDBEBF91
:10B74000C0C1C2C3C4C5C6C7C8C9CACBCCCDCECF81
:10B75000D0D1D2D3D4D5D6D7D8D9DADBDCDDDEDF71
:10B76000E0E1E2E3E4E5E6E7E8E9EAEBECEDEEEF61
:10B77000F0F1F2F3F4F5F6F7F8F9FAFBFCFDFEFF51
:10B78000000102030405060708090A0B0C0D0E0F41
:10B79000101112131415161718191A1B1C1D1E1F31
:10B7A000202122232425262728292A2B2C2D2E2F21
:10B7B000303132333435363738393A3B3C3D3E3F11
:10B7C000404142434445464748494A4B4C4D4E4F01
:10B7D000505152535455565758595A5B5C5D5E5FF1
:10B7E000606162636465666768696A6B6C6D6E6FE1
:10B7F000707172737475767778797A7B7C7D7E7FD1
:10B8000000020406080A0C0E10121416181A1C1E48
:10B8100020222426282A2C2E30323436383A3C3E38
:10B8200040424446484A4C4E50525456585A5C5E28
:10B8300060626466686A6C6E70727476787A7C7E18
:10B840007F7D7B79777573716F6D6B6967656361F8
:10B850005F5D5B59575553514F4D4B4947454341E8
:10B860003F3D3B39373533312F2D2B2927252321D8
:10B870001F1D1B19171513110F0D0B0907050301C8
:10B88000FFFDFBF9F7F5F3F1EFEDEBE9E7E5E3E1B8
:10B89000DFDDDBD9D7D5D3D1CFCDCBC9C7C5C3C1A8
:10B8A000BFBDBBB9B7B5B3B1AFADABA9A7A5A3A198
:10B8B0009F9D9B99979593918F8D8B898785838188
:10B8C00080828486888A8C8E90929496989A9C9E88
:10B8D000A0A2A4A6A8AAACAEB0B2B4B6B8BABCBE78
:10B8E000C0C2C4C6C8CACCCED0D2D4D6D8DADCDE68
:10B8F000E0E2E4E6E8EAECEEF0F2F4F6F8FAFCFE58
:10B900007F7F7F7F7F7F7F7F7F7F7F7F7F7F7F7F47
:10B910007F7F7F7F7F7F7F7F7F7F7F7F7F7F7F7F37
:10B920007F7F7F7F7F7F7F7F7F7F7F7F7F7F7F7F27
:10B930007F7F7F7F7F7F7F7F7F7F7F7F7F7F7F7F17
:10BC00000309131E28313A40464C5054585B5E617C
:10BC1000636567696B6C6E6F70717273747576773C
:10BC2000777879797A7A7B7B7C7C7C7D7D7D7E7E62
:10BC30007E7E7F7F7F7F7F7F7F7F7F7F7F7F7F7F16
:10BC40007F7F7F7F7F7F7F7F7F7F7F7F7F7E7E7E07
:10BC50007E7D7D7D7C7C7C7B7B7A7A797978777739
:10BC6000767574737271706F6E6C6B696765636102
:10BC70005E5B5854504C46403A31281E130903006D
:10BC8000C6CCD5DBDFE3E5E7E9EAEBECEDEEEFEF81
:10BC9000F0F0F0F1F1F1F1F2F2F2F2F2F2F2F2F38D
:10BCA000F3F3F3F3F3F3F3F3F3F3F3F3F3F3F3F364
:10BCB000F3F3F3F3F3F3F3F3F3F3F3F3F3F3F3F354
:10BCC000F3F3F3F3F3F3F3F3F3F3F3F3F3F3F3F344
:10BCD000F3F3F3F3F3F3F3F3F3F3F3F3F3F3F3F334
:10BCE000F2F2F2F2F2F2F2F2F1F1F1F1F0F0F0EF41
:10BCF000EFEEEDECEBEAE9E7E5E3DFDBD5CCC60000
:10BD000000283D42302D2C2B2C2D2E2F3032333558
:10BD100037393B3D3F414345484A4C4E50535557B8
:10BD2000595B5D5F61636567696B6C6E707173749D
:10BD3000757778797A7B7C7D7D7E7E7F7F7F7F7F44
:10BD40007F7F7F7F7F7F7E7E7D7D7C7B7A7978772A
:10BD500075747371706E6C6B69676563615F5D5B51
:10BD600059575553504E4C4A484543413F3D3B3946
:10BD700037353332302F2E2D2C2B2C2D30423D28B1
:10BD800000E9E5FED4D7D7D7D6D4D2D0CECCCAC816
:10BD9000C6C3C1BFBDBAB8B6B4B1AFADABA9A7A554
:10BDA000A3A19F9E9C9A999795949391908F8D8C27
:10BDB0008B8A898888878685858484848383838326
:10BDC0008383838383848484858586878888898A1E
:10BDD0008B8C8D8F909193949597999A9C9E9FA10F
:10BDE000A3A5A7A9ABADAFB1B4B6B8BABDBFC1C327
:10BDF000C6C8CACCCED0D2D4D6D7D7D7D4FEE5E9E0
:10BE0000F9F8F9F5EBE1DDDEE0E2E4E5E6E5E4E2B0
:10BE1000DED9D2CAC1B7ACA299918A8683818080CB
:10BE20008182838586888A8C8D8F90929395969750
:10BE300098999A9B9B9C9D9D9D9E9E9E9F9F9F9F38
:10BE40009F9F9F9E9E9E9D9D9D9C9B9B9A99989730
:10BE500096959392908F8D8C8A8886858382818037
:10BE6000808183868A9199A2ACB7C1CAD2D9DEE219
:10BE7000E4E5E6E5E4E2E0DEDDE1EBF5F9F8F90022
:10BE80000708070B151F2322201E1C1B1A1B1C1E34
:10BE900022272E363F49545E676F767A7E7F7F7FFA
:10BEA0007F7E7D7B7A7876747371706E6D6B6A6954
:10BEB000686766656564646363626262616161614B
:10BEC0006161616262626363636465656667686934
:10BED0006A6B6D6E7071737476787A7B7D7E7F7F0E
:10BEE0007F7F7E7A766F675E54493F362E27221E0B
:10BEF0001C1B1A1B1C1E2022231F150B07080700E2
:10BF00001F313D444E5354565A5F64696E747679BE
:10BF10007C7F7F7F7F7F7F7F7F7F7F7F7F7F7F7F34
:10BF20007F7F7F7F7F7F7F7F7F7F7F7F7F7F7F7F21
:10BF30007F7F7F7F7F7F7F7F7F7F7F7F7F7F7F7F11
:10BF40007F7F7F7F7F7F7F7F7F7F7F7F7F7F7F7F01
:10BF50007F7F7F7F7F7F7F7F7F7F7F7F7F7F7F7FF1
:10BF60007F7F7F7F7F7F7F7F7F7F7F7F7F7F7F7FE1
:10BF70007F7F7F7F7F7F7F7F7F7F7F7C7871684C33
:10BF80002C1C120C0A0B0A05FDF3E9DFD4CAC0B75A
:10BF9000AEA69E97918B86858280808080808080EF
:10BFA0008080808080808080808080808080808091
:10BFB0008080808080808080808080808080808081
:10BFC0008080808080808080808080808080808071
:10BFD0008080808080808080808080808080808061
:10BFE0008080808080808080808080808080808051
:10BFF000808080808087919DACC4CBD4DDF2FAFA3A
:10C0000022002400260028002B002D0030003300E1
:10C01000360039003D004000440048004C0051000B
:10C0200056005B00600066006C00730079008100C0
:10C03000880090009900A200AC00B600C100CC00BE
:10C04000D800E500F3000101100121013201440193
:10C0500057016C0181019801B001CA01E50102029A
:10C060002102410264028802AE02D70203033003B8
:10C0700061039403CB03050442048304C704100541
:10C080005D05AF0505066106C20629079607090882
:10C09000830805098E09200ABA0A5D0B0A0CC10C37
:10C0A000840D510E2B0F121007110A121D1340148C
:10C0B0007415BA1614188319071BA31C571E2420C5
:10C0C0000E22142439267F28E82A752D29300633BC
:10C0D0000F364539AD3C49401B442848734CFE504F
:10C0E000CF55EA5A51600C661D6C8B725A7992805A
:10C0F00037885090E598FDA19FABD3B5A3C0000051
:10C100001F93CF93DF93FA01549131961491C52F69
:10C11000D0E09F012F5F3F4F70E095E0660F771FE3
:10C120009A95E1F7680F711D40E00BC084918D93E3
:10C130009F5F31969517D0F34F5F2C0F3D1F605EC8
:10C140007F4F411730F4DB01A054BE4FF90190E05E
:10C15000F1CFDF91CF911F910895382F603CD0F43B
:10C1600070E0660F771FCB018E5A974FFC01249128
:10C170006D5A774FFB016491832F90E0FC0174E0CE
:10C18000EE0FFF1F7A95E1F7E81BF90BE050F94F2E
:10C1900021876287832F90E0FC0154E0EE0FFF1FA0
:10C1A0005A95E1F7E81BF90BE050F94F818523819F
:10C1B0003481280F311D368725874695469546954B
:10C1C000842F90E045E0880F991F4A95E1F7280FEA
:10C1D000391F3487238708958F929F92AF92BF9221
:10C1E000CF92DF92EF92FF920F931F93CF93DF9343
:10C1F000882E962E5A016901F02E00E010E080EEA4
:10C20000F80E0CC04F2D6E2D882D8C0F0E943653CA
:10C210002196CA15DB05B4F30F5F1F4F0C151D05E2
:10C220002CF4C0E0D0E0E02EE90CF3CFDF91CF9109
:10C230001F910F91FF90EF90DF90CF90BF90AF9044
:10C240009F908F90089540520E9436530895FF9218
:10C250000F931F93CF93DF938C01F62EEA01FE011B
:10C2600044912196442349F0802F0F5F1F4F4F7751
:10C2700040526F2D0E943653F2CFDF91CF911F9124
:10C280000F91FF900895FF920F931F93182F062F81
:10C29000F42E42954F704A3010F4405F01C0495E61
:10C2A000602F812F0E9436534F2D4F70812F8F5F4B
:10C2B0004A3010F4405F01C0495E602F0E9436533F
:10C2C0001F910F91FF900895FF920F931F93F82EE7
:10C2D000162F042F452F0E944361402F612F8F2D71
:10C2E0008E5F0E9443611F910F91FF900895EF921E
:10C2F000FF920F931F93F62E042F182FF8E0EF2EC6
:10C30000E80E07FF02C041E101C040E16F2D812F1F
:10C310000E9436531F5F1E1511F0000FF2CF1F91C0
:10C320000F91FF90EF900895FF920F931F93CF937B
:10C33000DF93F62E042FEC0110E0002311F41123FB
:10C3400039F4802F6AE00E94B76B905F492F01C0DB
:10C3500040E06F2D8C2F0E9436531F5F21971330C2
:10C3600031F0802F6AE00E94B76B082FE6CFDF9193
:10C37000CF911F910F91FF900895CF92DF92EF928E
:10C38000FF920F931F93CF93DF93C62E79018A01FB
:10C39000EC01DD24E114F1040105110511F4DD20A7
:10C3A00059F4C801B7012AE030E040E050E00E94B3
:10C3B000D66B462F405F01C040E06C2D8C2F0E9451
:10C3C0003653D394219786E0D81669F0C801B70197
:10C3D0002AE030E040E050E00E94D66BC901DA016B
:10C3E0007C018D01D7CFDF91CF911F910F91FF90ED
:10C3F000EF90DF90CF9008957F928F929F92AF92AF
:10C40000BF92CF92DF92EF92FF920F931F93CF9341
:10C41000DF93782E862E5A016901780100E010E042
:10C420000CC0A701692D872D8C0F0E9428532196DF
:10C43000CA15DB05B4F30F5F1F4F0C151D052CF457
:10C44000C0E0D0E0902E980CF3CFDF91CF911F91F8
:10C450000F91FF90EF90DF90CF90BF90AF909F90A3
:10C460008F907F9008957F928F929F92AF92BF920C
:10C47000CF92DF92EF92FF920F931F93CF93DF93B0
:10C48000782E862EEA01FA01C590D490FA013296F0
:10C49000A590B49000E016C0FC01EE0DFF1D329691
:10C4A000EE0FFF1FEC0FFD1F45915491692D812F59
:10C4B000870D0E9428531F5F812F90E08C159D05EA
:10C4C0005CF30F5F802F90E08A159B055CF48C9DD8
:10C4D00070018D9DF00C9C9DF00C112410E0902EAD
:10C4E000980CEACFDF91CF911F910F91FF90EF90C1
:10C4F000DF90CF90BF90AF909F908F907F900895E6
:10C500000F931F93CF93DF938C01C0E0D0E007C05F
:10C510000E940F548823E1F30E9412542196C01701
:10C52000D107B4F3DF91CF911F910F9108958091BE
:10C530009F0187FD09C08A5F8093FC068F5F80930F
:10C54000FF06855080939F0180919F0183313CF0CD
:10C550008FEF80939F018093FB068093FE060895E2
:10C56000982F87FF05C083E98093400584E904C0C4
:10C570008AE8809340058BE88093410596FF05C0CB
:10C5800085E98093430586E904C08DE880934305DF
:10C590008EE88093440595FF02C087E901C08FE8CB
:10C5A0008093470594FF05C088E980934A0589E98F
:10C5B00004C080E980934A0581E980934B0593FF8D
:10C5C00002C087E901C08FE880934E0592FF05C045
:10C5D00085E98093510586E904C08DE88093510573
:10C5E0008EE88093520591FF05C083E9809354053E
:10C5F00084E904C08AE8809354058BE8809355054C
:10C600000895EAECFEE0A6EAB6E04FEF5FEF85851D
:10C610008F3128F48230E0F4813011F503C08F317E
:10C62000F9F419C084858823B1F081508487808112
:10C63000918120853185820F931F91838083828130
:10C64000938122853385820F931F9383828308C051
:10C650008F5F858705C0158651834083538342834E
:10C6600081818C93838111968C931197858581307C
:10C6700031F0823038F0869586958695815E1296E7
:10C680008C9312973E9613968FE0EA33F80709F0E1
:10C69000BECF80913B0F882319F0815080933B0FD0
:10C6A000089580E58093020721E02093080780E643
:10C6B0008093110780E893E090931307809312070B
:10C6C000209317072093200740E055E0509322075E
:10C6D000409321072093260720932F07509331077B
:10C6E000409330072093350720932E0720933E0771
:10C6F0005093400740933F072093440762E06093C4
:10C700003D0720934D0750934F0740934E072093CA
:10C71000530783E080934C0720935C0750935E0798
:10C7200040935D072093620734E030935B072093CA
:10C730006B0750936D0740936C072093710785E05A
:10C7400080936A0720937A0750937C0740937B0776
:10C750002093800786E08093790720938907509380
:10C760008B0740938A0720938F0787E08093880781
:10C770002093980780E295E090939A078093990719
:10C7800020939E072093A7079093A9078093A8075B
:10C790002093AD072093A6076093B6079093B80740
:10C7A0008093B7072093BC076093B5073093C50704
:10C7B0009093C7078093C6072093CB073093C40795
:10C7C00080E18093D40780E495E09093D60780932E
:10C7D000D5072093DA0782ED99E0909306078093BE
:10C7E00005079093150780931407E3E2F7E084ECC4
:10C7F00092E3918380833F9627E0E73DF207C9F7F4
:10C8000082ED99E0918380830895FF920F931F93A7
:10C81000CF93DF93F82EE7EDFEE0C0E0D0E080811B
:10C82000882309F0A0C0CE01880F991FDC0123E006
:10C83000AA0FBB1F2A95E1F7A81BB90BA653B14F4E
:10C8400081E01D968C931D97FE0103E0EE0FFF1F04
:10C850000A95E1F7EC1BFD0BEE0FFF1FE453F14FC0
:10C8600080E094EC9183808380913A0F04EC10E097
:10C87000081B11094091DD0FFF2061F480E098E072
:10C880008D939C93242F30E02850304080E0922FED
:10C89000B8010EC080E090E88D939C9320E830E0D2
:10C8A000241B310966277727601B710B80E0922FCC
:10C8B0000E94C36B20173107ACF4CE01880F991F7B
:10C8C000FC01A3E0EE0FFF1FAA95E1F7E81BF90BAF
:10C8D000E653F14F80E09FEF9387828760877187EF
:10C8E000048738C0CE01880F991FFF2069F4FC012E
:10C8F00073E0EE0FFF1F7A95E1F7E81BF90BE653A3
:10C90000F14F80E091E00CC0FC0163E0EE0FFF1FEF
:10C910006A95E1F7E81BF90BE653F14F80E09FEFD2
:10C9200091878087CE01880F991FFC0143E0EE0FAD
:10C93000FF1F4A95E1F7E81BF90BE653F14F80E042
:10C94000902FB9010E94C36B709561957F4F7387DB
:10C95000628724878EE180933B0F41E060E782E0AD
:10C960000E94735806C021963E96C830D10509F042
:10C9700056CFDF91CF911F910F91FF900895BF92F5
:10C98000CF92DF92EF92FF920F931F93CF93DF939B
:10C990000AEC1EE055E4E52E5FE0F52E42E0B42EF1
:10C9A000CC24CA94DC2CF8018585882309F43FC087
:10C9B000CCE3DFE0F70180818823A1F1F801218138
:10C9C0002D5F5381898183504B8128175CF1332778
:10C9D00027FD3095992787FD909509968217930733
:10C9E0000CF1252F2C5F842F84502817DCF033277F
:10C9F00027FD3095992787FD90950C968217930710
:10CA00008CF01986B58688819981918380838A818B
:10CA10009B8193838283D982C88241E060EA81E06E
:10CA20000E9473582A96FFE0CC3DDF0719F6025F9B
:10CA30001F4F8AE090E0E80EF91E9FE00A331907C5
:10CA400009F0B1CFDF91CF911F910F91FF90EF903F
:10CA5000DF90CF90BF9008950F931F93CF93DF93F4
:10CA600080E00E941654EC0193FF5AC080919E0111
:10CA70008130F1F410929E0182ED99E090930607C7
:10CA80008093050700E010E02AE030E040E250E04B
:10CA900060E070E080E090E00E94FC6110925A0E2D
:10CAA000109200074AEE53E760E087E10E94806041
:10CAB00080913B0F8823A1F580915C0E853048F072
:10CAC0008AE080935C0E41E060EA80E00E94735847
:10CAD00012C08F5F80935C0E80919C0187FD08C01F
:10CAE0000E94A76B63E070E00E94C36B019719F48A
:10CAF00080E00E94056480915E0E882389F4109284
:10CB00005F0E81E080935E0E00E010E021E030E0F7
:10CB100046E150E068E170E081E090E00E94FC6155
:10CB2000C3FF5AC080919E018130F1F410929E01A2
:10CB300082ED99E0909306078093050700E010E0EE
:10CB40002AE030E040E250E060E070E080E090E019
:10CB50000E94FC6110925A0E109200074AEE53E7B1
:10CB600060E087E10E94806080913B0F8823A1F5FF
:10CB700080915D0E853048F08AE080935D0E41E043
:10CB800060EA80E00E94735812C08F5F80935D0E50
:10CB900080919C0181FD08C00E94A76B63E070E05A
:10CBA0000E94C36B019719F481E00E940564809193
:10CBB0005E0E882389F410925F0E81E080935E0EF2
:10CBC00000E010E021E030E046E150E068E170E094
:10CBD00081E090E00E94FC61C7FF0AC080913A0F9B
:10CBE000825080933A0F893018F488E080933A0F8E
:10CBF000C6FF0AC080913A0F8E5F80933A0F803C47
:10CC000018F080EC80933A0FC5FF0AC08091DD0FC9
:10CC100081508093DD0F873018F486E08093DD0F1C
:10CC2000C4FF0AC08091DD0F8F5F8093DD0F8538D0
:10CC300018F084E88093DD0FD093610EC093600EEE
:10CC400080E0DF91CF911F910F9108950F931F9373
:10CC5000CF93DF93E5E4FFE000E010E080818823DC
:10CC600009F07BC0E801CC0FDD1FC80123E0880F6D
:10CC7000991F2A95E1F7C80FD91FC45CD04F84E1F2
:10CC8000898720915A0E84E990E0821B91091882CD
:10CC90008983F801EE0FFF1FEE0FFF1FE00FF11F5A
:10CCA000EE0FFF1FE25CF04F2091010780E590E05E
:10CCB000821B9109108281830E94A76B62E370E05E
:10CCC0000E94C36B9D838C830E94A76B62E370E01C
:10CCD0000E94C36B88969F838E8380915F0E8F30F6
:10CCE00048F00E94A76B62E370E00E94C36BCC9691
:10CCF0009F838E830E94A76B80FF14C0F801EE0F04
:10CD0000FF1FC801A3E0880F991FAA95E1F7E80F5C
:10CD1000F91FE45CF04F84819581909581959F4F38
:10CD2000958384830E94A76BF80173E0EE0FFF1FC9
:10CD30007A95E1F7000F111FE00FF11FE45CF04F4F
:10CD400064E670E00E94C36B8E5C80872FEF43E245
:10CD500065E083E00E946D5507C00F5F1F4F3A9654
:10CD60000031110509F07ACFDF91CF911F910F911A
:10CD70000895982F80919F018F3FB9F5923011F45B
:10CD80008EE717C0943011F48CE613C0983011F47C
:10CD900087E50FC0903111F482E40BC0903211F49A
:10CDA0008DE207C0903411F488E103C0903819F483
:10CDB00086E08093DC0F9091DC0F9093FA0626ECCE
:10CDC0002093FB0686E08093FC069A5F9093FD0615
:10CDD0002093FE0687E08093FF062FEF4EE166E08A
:10CDE00083E00E946D5510929F0108959F92AF922B
:10CDF000BF92CF92DF92EF92FF920F931F93CF9348
:10CE0000DF93CCE3DFE00EEB16E054E1952EAA248D
:10CE1000AA94BA2C8985882309F478C088819981DD
:10CE20002C813D81820F931F998388838E819F81FE
:10CE30002A813B81820F931F9B838A83892F9927A5
:10CE4000893C910508F43BC04981642F70E020E0E3
:10CE500030E0F901EE57FB488491F901E558FB48B1
:10CE60005491841710F0451758F490E00197681713
:10CE70007907ECF4852F90E0029768177907BCF0EA
:10CE800027573B48F9012491822F809590919C016E
:10CE9000892380939C0190919D01891769F0822FCD
:10CEA0000E94B96680919C0180939D0105C02F5F0F
:10CEB0003F4F2730310569F61986B982A882E9808B
:10CEC000FF24F6E0EF16F10438F48C819D819095F3
:10CED00081959F4F9D838C83C980DD2483E8C8168C
:10CEE000D10438F08C819D81909581959F4F9D83D1
:10CEF0008C8380915B0E90E083709070892B31F46D
:10CF000089858F5F8987803209F499868981F80144
:10CF100080838B818183898582832A960D5F1F4F51
:10CF2000FFE0CC3DDF0709F075CFDF91CF911F9176
:10CF30000F91FF90EF90DF90CF90BF90AF909F90B8
:10CF400008952F923F924F925F926F927F928F92AD
:10CF50009F92AF92BF92CF92DF92EF92FF920F9388
:10CF60001F93DF93CF93CDB7DEB767970FB6F894D3
:10CF7000DEBF0FBECDBF0E941E53549A5B9A8FED49
:10CF800092E70E94D75480ED0E94665584E398E3AF
:10CF90000E944B5380E00E9448530E94516300E07E
:10CFA00010E024E030E046E150E06BE070E080E02B
:10CFB00090E00E94FC618AE90E94455345EA54E7EB
:10CFC00060E170E081E090E00E94276147EB54E768
:10CFD00061E170E081E090E00E94276146EC54E757
:10CFE00063E170E081E090E00E9427612FEF43E26F
:10CFF00065E083E00E946D5584EB90E00E948062C2
:10D0000024E030E046E150E06BE070E080E090E04A
:10D010000E94FC6102E910E021E030E046E150E0CE
:10D020006DE170E080E090E00E94FC6148E453E72D
:10D030006EE081E00E9480604AEE53E760E087E1A5
:10D040000E94806080919C010E94B06240E954E798
:10D0500068E170E081E090E00E9427619E012F5F0F
:10D060003F4F3B8B2A8BF901CE010D969D8B8C8B0C
:10D070008E2F9A89891B81932C893D89E217F307AA
:10D08000B9F788E48093DD0F84E680933A0F10921D
:10D09000A50689E08093F10620ED2093F20695E243
:10D0A0009093F30681E88093F4062093F50690931D
:10D0B000F6066624FF24DD245524CC24188A24E0B7
:10D0C000E22E32E03F8781E08E87AA24A39498EC79
:10D0D000292E1D86332488EC482E882402E3B02EA6
:10D0E000FE013B96FF8BEE8B4B990DC023988FE092
:10D0F00090E00E94806201C05C9A4B99FDCF4B9BEF
:10D10000FECF5C98239A80915E0E8823F1F4D3942D
:10D11000F9E5FD1510F4DD2403C02DE22D1548F0CE
:10D1200040E954E768E170E081E090E00E94276107
:10D130000CC000E010E021E030E046E150E068E1A2
:10D1400070E080E090E00E94FC6180915E0E823091
:10D1500009F0ACC0D39439E53D1510F4DD2403C0CB
:10D160008DE28D1548F04BED54E768E170E080E00A
:10D1700090E00E9427610CC000E010E021E030E068
:10D1800046E150E068E170E080E090E00E94FC61E0
:10D190004DE055E769E170E080E090E00E94276192
:10D1A00040915F0E69E170E081E190E00E9494613E
:10D1B000442009F07BC09EEF90939C0100E010E0BA
:10D1C00022E030E046E150E06AE170E080E090E08B
:10D1D0000E94FC6110925E0EECE3FFE0118620E0FD
:10D1E0003CE83183208380E090ED938382833A96FC
:10D1F0009FE0EC3DF90791F70E94F666E7EDFEE04F
:10D200002FE120833E963FE0E734F307C9F70E9401
:10D21000016311C081E090E00E94806280915A0E0B
:10D220008F5F80935A0E813C10F010925A0E8091BD
:10D230005A0E8093000780915A0E882359F788E090
:10D2400080935A0E8093000791E090939E01E2EB49
:10D25000F0E2F0930607E09305071092010700E261
:10D2600010E02AE030E040E250E060E070E080E072
:10D2700090E00E94FC6181E090E00E948062109248
:10D280005F0E88E790E00E94806248EF54E769E112
:10D2900070E080E090E00E94276177246624FF24FC
:10D2A00012E0A12E33248824B2E3BB2E81E090E06B
:10D2B0000E94806280915B0E8F5F80935B0EF98984
:10D2C000FF5FF98B0E9401630E94F6660E94BF64B3
:10D2D0000E9401630E94F6660E94BF640E9401637F
:10D2E0000E94F6660E94BF6480919C018C7749F48D
:10D2F00080915E0E813029F422E020935E0EA8EC2E
:10D300004A2E80915E0E823031F480915A0E88232D
:10D3100011F410929E013989333009F056C00E94F1
:10D320009762C39486E08C1508F4CC2480919C010C
:10D33000809581FF0AC046E0C49EA0011124425E90
:10D340005C486AE184E10E94806080919C01809544
:10D3500082FF0AC046E0C49EA0011124425E5C48E0
:10D360006AE181E10E94806080919C01809584FF48
:10D370000AC046E0C49EA0011124425E5C486AE1F6
:10D380008AE00E94806080919C01809586FF0AC09F
:10D3900046E0C49EA0011124425E5C486AE183E03D
:10D3A0000E94806080919C0187FD0AC046E0C49E77
:10D3B000A0011124425E5C486AE180E00E94806026
:10D3C00080919C010E94B062198A53949EE1591683
:10D3D00009F043C080915C0E882319F0815080933E
:10D3E0005C0E80915D0E882319F0815080935D0E54
:10D3F00080915C0E853018F08170865D01C08B5D78
:10D400008093F30680915D0E853018F08170865D03
:10D4100001C08B5D8093F6068394E4E1E815E0F4A7
:10D4200080915F0E8F5F80935F0E42EF54E768E15B
:10D4300070E088E090E00E94276140915F0E68E113
:10D4400070E08EE090E00E949461FEEFBF0E24E059
:10D450002B1508F026C127C1552435E0831641F469
:10D4600048EF54E768E170E088E090E00E942761AF
:10D4700080915B0E8F728F32B9F40E94A76B80FD92
:10D4800007C0E39485E08E1548F4F5E0EF2E06C062
:10D49000EA9492E09E1510F0E3E0EE2EEE2DE250BD
:10D4A000EF87FE2DF350FE878EE197E0DE011196A7
:10D4B000ED91F0E0E859FB4824912E19FC012083FE
:10D4C0000F962E893F89A217B30791F738893F5FDE
:10D4D000388BEB85F0E0E859FB48E491E6958E2F18
:10D4E0009F85891B8093B407E695FE85EF1BE0932B
:10D4F000C307353079F4FE01319680818F5F8083D8
:10D500008C3008F0108231962C893D89E217F307A0
:10D51000A1F7188A939480919E018823E1F432E068
:10D520009316B1F480915A0E8F5F80935A0E813C0E
:10D5300010F010925A0EE0915A0EE0930007F0E0BE
:10D54000EF73F070E85DFB48E491E09301079924E4
:10D5500072E0A72E87C09A1409F084C08D858823B5
:10D56000C1F480915A0E885F80935A0EE2EBF0E28C
:10D57000F0930607E093050700E210E02AE030E0B0
:10D5800040E250E060E070E080E090E00E94FC61EA
:10D590007724332081F56394F5E0F61568F47394ED
:10D5A000EF2DF0E0EC5DFA48F3948491E72DF0E084
:10D5B000E05AFD4F808366242FE1F216D1F03FE35D
:10D5C000F316B9F08FE5F816A1F09FE7F91689F088
:10D5D000EFE9FE1671F0FFEBFF1659F02FEDF21692
:10D5E00041F03AEE3F1538F47724FF243324339486
:10D5F00002C077247A9480915A0E8F5F80935A0EDE
:10D60000803C10F010925A0E80915A0E80930007C1
:10D6100091E0391611F5882301F510929E01E2ED93
:10D62000F9E0F0930607E093050700E010E02AE038
:10D6300030E040E250E060E070E080E090E00E9486
:10D64000FC614AEE53E760E087E10E948060992424
:10D65000AA24A394F1E0FD8705C09924AA24A394E9
:10D6600021E02D8780919E01882361F42A9451F452
:10D670000E9426660E94A76B6B2D70E00E94C36B10
:10D680002B2C280E8091DD0F8093A30680913A0FFA
:10D690008093A406442019F40E942C6525CD4A9459
:10D6A00023CD65E0B62E55248824E2CEA0E0B0E07C
:10D6B000ECE5FBE60C944E6CEC01A880B980CA80C6
:10D6C000DB80A114B104C104D10441F484E2A82E8A
:10D6D00089EDB82E8BE5C82E87E0D82EC601B5019E
:10D6E0002DE133EF41E050E00E942B6C27EA31E45A
:10D6F00040E050E00E940C6C7B018C01C601B5013A
:10D700002DE133EF41E050E00E942B6CCA01B901DA
:10D710002CEE34EF4FEF5FEF0E940C6C6E0D7F1D0F
:10D72000801F911F97FF04C0615070408040904857
:10D73000688379838A839B839B013F77C901CDB737
:10D74000DEB7EAE00C946A6C0E94566B089580EA9A
:10D7500091E00E94566B0895A0E0B0E08093A00194
:10D760009093A101A093A201B093A3010895991BE6
:10D7700079E004C0991F961708F0961B881F7A95C8
:10D78000C9F78095089597FB092E07260AD077FDE3
:10D7900004D02ED006D000201AF4709561957F4FEA
:10D7A0000895F6F7909581959F4F0895A1E21A2E5E
:10D7B000AA1BBB1BFD010DC0AA1FBB1FEE1FFF1F35
:10D7C000A217B307E407F50720F0A21BB30BE40B85
:10D7D000F50B661F771F881F991F1A9469F76095CC
:10D7E0007095809590959B01AC01BD01CF01089586
:10D7F000AA1BBB1B51E107C0AA1FBB1FA617B70777
:10D8000010F0A61BB70B881F991F5A95A9F7809592
:10D810009095BC01CD010895629FD001739FF001E6
:10D82000829FE00DF11D649FE00DF11D929FF00DB0
:10D83000839FF00D749FF00D659FF00D9927729FE7
:10D84000B00DE11DF91F639FB00DE11DF91FBD0172
:10D85000CF011124089597FB092E05260ED057FD00
:10D8600004D0A4DF0AD0001C38F4509540953095C0
:10D8700021953F4F4F4F5F4F0895F6F79095809554
:10D88000709561957F4F8F4F9F4F08952F923F92D4
:10D890004F925F926F927F928F929F92AF92BF92C0
:10D8A000CF92DF92EF92FF920F931F93CF93DF936C
:10D8B000CDB7DEB7CA1BDB0B0FB6F894DEBF0FBEC9
:10D8C000CDBF09942A88398848885F846E847D8416
:10D8D0008C849B84AA84B984C884DF80EE80FD8018
:10D8E0000C811B81AA81B981CE0FD11D0FB6F8948E
:0ED8F000DEBF0FBECDBFED010895F894FFCF4F
:10D8FE00000000000000000000000000000000001A
:10D90E000000000000000000000000000000000009
:10D91E0000000000000000000000000000000000F9
:10D92E0000000000000000000000000000000000E9
:10D93E0000000000000000000000000000000000D9
:10D94E0000000000000000000000000000000000C9
:10D95E0000000000000000000000000000000000B9
:10D96E0000000000000000000000000000000000A9
:10D97E000000000000000000000000000000000099
:10D98E002B3DA140194491470A4B844EFEFE01FFE8
:04D99E000100000084
:00000001FF
